:020000040800F2
:10000000005000207D4C01081D4D01086536010897
:100010001D4D01081D4D01081D4D01080000000087
:100020000000000000000000000000001D4D01085D
:100030001D4D0108000000001D4D0108D7DF00081C
:100040001D4D01081D4D01081D4D01081D4D0108E4
:100050001D4D01081D4D010801B80008FDB700083D
:100060001D4D01081D4D01081D4D01081D4D0108C4
:100070001D4D01081D4D010815CC00081D4D01083E
:1000800089F700081D4D01081D4D01081D4D01088F
:100090001D4D01081D4D01081D4D0108F9B700084F
:1000A0001D4D010869DB00081D4D010879DB0008C2
:1000B00059DB000849DB000839DB00084944000827
:1000C0004D44000841440008454400081D4D010806
:1000D0001D4D01080DCC000805CC0008FDCB000823
:1000E000E5DF00081D4D01081D4D0108000000005E
:1000F0000000000000000000000000000000000000
:0C01000000000000000000005FF808F1A3
:100110002DE9F04F754B764EA3B03360002373602A
:1001200012F03CF818B912F05BF80AF009FC0AF07A
:10013000A9FC704A704C1378704D43F001031370A2
:1001400000230A930B930C934FF4E0130D93236851
:10015000A87B43F480332360A36943F01003A361B9
:10016000236803F400330B930A9B01330A930B9B20
:100170001BB90A9BB3F5A06FF2D123685E4913F453
:10018000003301D0022315E00A6842F001020A6040
:100190000A93236803F002030B930A9B01330A932B
:1001A0000B9B1BB90A9BB3F5A06FF2D123689B0789
:1001B00039D501230C93524B52491A6842F0100270
:1001C0001A601A6822F003021A601A6842F00202EA
:1001D0001A606368636063686360636843F48063A4
:1001E0006360494B1A68043B22F070425A60474AE8
:1001F0001160616821F47C116160596841F000412F
:100200005960D96821F40041D9609B681F0449BF37
:100210003F4B4FF4E01313604FF480130D930C9B8E
:10022000012B01D117E0FEE7022B18D168B10D9B1D
:10023000B3F5801F02D14FF4A01305E00D9BB3F579
:10024000E01F02D14FF400130D930D9963680B4327
:1002500043F4803302E0636843F46013636023680F
:1002600043F0807323602168234B8901FBD55968D3
:1002700021F003015960596841F002015960636837
:100280001D4903F00C03082BF9D14B68DFF88C8073
:1002900003F00C03042B03D0082B03D0194B12E0FE
:1002A000136810E04B684868C3F38343C70303F146
:1002B000020301D4174905E0496811F4003F1168B1
:1002C00018BF49084B43C8F8003063681249C3F3AC
:1002D00003130B44197ED8F80030CB40C8F8003027
:1002E0001368084A93421BD101221DE027A1000890
:1002F00030090020B833002000100240EC29002013
:100300000020024000127A00041001402400002066
:10031000001BB70000093D00649C01085C00002040
:100320008A4A934202D10222894B1A70DFF878A2DE
:10033000884BDFF878C2CAF80C30A3690DF1880B3E
:1003400043F00103A361636A834FB360636A60464D
:1003500043F080736362A3694FF0000943F01C030C
:10036000A3614FF6FF732BF82C3D5946CDF80CC016
:100370008DF85E900FF013FB384659460FF00FFBD7
:10038000594676480FF00BFB754A5846536843F0C0
:100390000073536008F030FC724A179B4946B3FB68
:1003A000F2F3714A714813600C2216F082FFD8F8FC
:1003B00000304FF47A72B3FBF2F36D4A013B5360A5
:1003C000F0238AF823300723C2F808901360AB6843
:1003D000DFF8DC91DFF8DC81C9F8003098E80F0025
:1003E0008BE80F00A3694FF0100A43F00803A361E4
:1003F000A369179843F00803A36108233B6118A978
:10040000C7F810A00FF0CBFA19981AA90FF0C7FA85
:10041000D9F80020100713D5564B93F89021012AE4
:100420000ED8554993F89121896811F0805300F056
:10043000F28505E04F4B002283F891210AF0E4FC9D
:1004400064200DF0BEFDA0224C48002116F031FFC3
:10045000E369002243F00703E361A36943F4006307
:1004600043F00C03A361444B4FF0000803F10C016F
:1004700002F8018001320E2AF5D1FF229A76DA764F
:100480001A775A773E4B3F4A41461A603E483C2213
:10049000D9F8004016F00DFF4146C4F3801705233C
:1004A0003A4ADFF8E4E0885C0C224A4302F80E0086
:1004B00047B91E3801289FBFFF2003F1FF3302F820
:1004C0000E00DBB201310529EAD1314A95F805A0C9
:1004D0001370304B304983F800A0304B264A33620A
:1004E000C0330B602E4BA10603EBCA035B7848BFF9
:1004F00001235362002340F2DC512A4A22F81310F0
:100500000133082BF7D110A800211C2216F0D1FED0
:1005100014F4007CDFF8A09004F400684ED0A3042B
:100520000AD4B8F1000F0AD095F8842109F10C0320
:10053000012A08BF4B4604E0CDF8109002E009F113
:100540000C030493CDF858B03AE000BF001BB7008D
:10055000E33300200005FA05000C014000100140C3
:100560000000014040420F003C2500208012002086
:1005700010E000E0EC290020300900205025002088
:10058000E4120020D22B0020E8120020B4C00108A1
:1005900065100020400400206C260020002A002066
:1005A000BCC00108CE0F002000ED00E000080140B3
:1005B0008C2900208C9C0108649C0108CDF810C097
:1005C000BAF10E0F04D00AF0EF0ABAF1080F02D107
:1005D00001238DF852300120CDF814C007F02EFF12
:1005E000DDF814C018B14088003018BF0120C4F3F2
:1005F00040038DF84630C4F3403300F001008DF81D
:100600004030C4F3C0338DF845008DF848708DF844
:100610004330B8F1000F07D095F8848108F1FF3717
:10062000D7F1000848EB0708C4F300438DF84930C0
:100630001CF1000318BF01238DF84A30736AB5F826
:100640004801003318BF01238DF84B30C4F3005329
:100650008DF84C30B5F84A31ADF85600ADF8503051
:10066000E004B5F8563148BFBA48ADF84E30C4F38F
:10067000804348BFB0F850018DF84730B5F8543189
:1006800048BFADF85600B3F5FA7FADF8543084BFDB
:100690000023ADF8563095F8CC31AF4886F82830B5
:1006A000002386F8293043709DF8523004F0010190
:1006B000002BC4F3C0028DF844808DF841108DF8F2
:1006C00042200CBF0023022301B902B1013309EB20
:1006D0008309D9F838309A1E1A33079300230692FB
:1006E0000593069B33F8024F06934FF6FF739C4227
:1006F00000F08E819DF84520E3B2240AE5B21AB1DC
:100700009A1E012A40F27F819DF8482032B1934918
:100710001A018958924A914200F075819DF849006A
:1007200030B18E491A0189588D4A914200F06B818F
:100730009DF8462052B18949039E01EB03114A6896
:10074000B24203D10A89102A00F05D819DF843204E
:1007500052B18249039E01EB03114A68B24203D1B0
:100760000A89022A00F04F819DF8442052B17B494A
:100770007C4E01EB03114A68B24203D10A89022A76
:1007800000F04181169E7EB1744F326807EB03176B
:100790007968914208D13A89B188914200F0338159
:1007A000F188914200F02F81022C02D19DF8402067
:1007B00003E0012C04D19DF84120002A00F02381A0
:1007C0009DF84B20654C1E015AB19DF8522042B94C
:1007D000A3F10802012A04D8A25963498A4208BF3A
:1007E00004259DF84C20344452B19DF852203AB96A
:1007F00010B10C3B012B01E0043B032B40F2EB80DA
:10080000012D48D1594FDFF854A1FF2387F87030EC
:1008100087F871300AEB06035A7B586803F1080920
:100820001B894FF00008ADF85C3017A9022387F848
:100830007480C7F880408DF85F308DF85E2087F8AF
:100840002C80C7F83080C7F83480C7F83880C7F8E4
:100850006C8087F8728087F873800FF0A0F85AF8E0
:10086000060099F8021042460AF017FE204641465B
:100870002A460CF01FF93E4BC7F88C80C7F884302D
:100880003C4B2046C7F8883007F1840107F1880205
:100890000CF058F9B7E0022D4CD19DF814204FF020
:1008A0001C0C0CFB02FC314B002703EB0C080893DB
:1008B0009DF814304FF0010988F87530274B88F8FF
:1008C00076709A19517B506802F1080A12898DF8E6
:1008D0005E1088F87E7017A988F87490C8F8804078
:1008E000CDF824C0ADF85C208DF85F500FF057F8BC
:1008F0001A4B9AF8021098593A460AF0CEFD204653
:1009000039464A460CF0D6F81B49089BDDF824C04E
:10091000C8F8841019496344C8F8881003F18401A9
:10092000C8F88C7020460A1D0CF00CF9059B4B444E
:10093000059368E0032D4CD19DF847300B4D104EC8
:1009400003B395F82A70204608214FF6FF72002362
:1009500033E000BFEC290020590900206CBE0108DB
:1009600000040040000C0140002C01403009002030
:1009700009AF0008E9AF0008D5B40008DFAE0008F1
:10098000D4270020BDF8542095F82A70B2F5FA7FDC
:10099000BDF856300BD986492046B1FBF2F208214A
:1009A00092B20AF0CFFD834B46F827000AE0824955
:1009B0002046B1FBF2F2012192B20AF0C3FD7F4B57
:1009C00046F82700C36095F82A30013385F82A30AD
:1009D00019E0042D17D1BDF84E20774B784D93FBCD
:1009E000F2F22046BDF85030012192B295F829600C
:1009F0000AF0A8FD95F8293005EB86060133C6F804
:100A0000540185F82930069B079A93427FF469AE1A
:100A10006B4D6C4B95F82920002485F874216A4AA7
:100A20001C7016789846A6F11702022A19D82B6A6C
:100A30000021185903EB040913F0D0F810B16B6AC8
:100A40005BBB25E0614F99E80F00274487E80F0062
:100A500098F8003010340133C02C88F80030E6D10B
:100A6000EDE75B4B13F836E003EBC603D3F804C0A5
:100A700088F800E0BCF1000FE1D07445DFDA534F95
:100A800023011F4463440FCB013487E80F00F4E7D0
:100A9000504F3B68DA0424D41DE04F4B4F4A13F803
:100AA000360003EBC6035C681070002CF0D0002306
:100AB0008342EDDAC3EBC3016218D2F800C0DFF85D
:100AC00044E1013341F80EC001EB0E079188B98073
:100AD0009279BA71ECE706F0EF03082B404B25D171
:100AE00026E098F80030012BF5D93E4C04EB0313B7
:100AF00003F1100810344445EDD054F8100C4FF0B9
:100B00007C5112F0D7FE4FF07C5144F8100C54F891
:100B1000140C12F0CFFE4FF07C5144F8140C54F832
:100B20000C0C12F0C7FE44F80C0CE3E70E2E08D1B3
:100B30001A78182E42F010021A7008D10DF0D4FC69
:100B400005E01A78192E22F010021A70F5E70DF060
:100B5000AFFC3B68244C5B035EBF244B01221A7040
:100B6000234B24481A78994642F004021A70224A0C
:100B700011789046022934BF142310238DF85E307B
:100B80004FF002038DF85F30A3694FF4805243F0B9
:100B90000403ADF85C2038BF0026A36128BF0126FE
:100BA00017A90EF0FCFE154B76B3154A2DE000BFD9
:100BB00000127A0009B0000840420F00F9AF0008A7
:100BC00030090020D0270020400400207C030020B2
:100BD000BCC001088C290020A4A70108F82500202A
:100BE000A81000208403002000100240A808002064
:100BF000B833002000080140E3330020C833002050
:100C000089DB0008F9250020714A00201A600DF0E8
:100C1000F7F9704B704E93E80300A3698BE803006B
:100C200043F00803A361179818A90EF0B8FEE36912
:100C3000304643F48043E3612369594643F48043DB
:100C4000236118238DF85E304FF42043ADF85C30FB
:100C500003238DF85F300EF0A2FE04224FF4804390
:100C6000304659468DF85E2003924FF4805AADF815
:100C70005C300EF094FE1023304659468DF85E30FD
:100C8000ADF85CA00EF08BFE2369322043F4804364
:100C90002361236923F480432361504B198801F4B5
:100CA000415141F4457141F003011980998B21F4C0
:100CB00000610904090C998307211982198889B2F6
:100CC00041F0400119809F23C6F810A08DF83C30F8
:100CD00000238DF83D308DF83E308DF83F300DF01B
:100CE00070F9039AC6F814A058460FA911F0DEFD5A
:100CF000C6F810A09DF85E309DF85D201B0243EA07
:100D000002439DF85F201343354A934215D03220A9
:100D10000DF057F9C6F814A0F52011F0FDFDFF20E5
:100D200011F0FAFD7028C6F810A006D198F800302E
:100D3000022B02BF2B4B03221A7098F80030032BB2
:100D40000CBF1F20022007F0FCFA98F80030032B9C
:100D500003D001200FF074F807E0022007F06EFBCB
:100D60000028F6D04388002BF3D03E684FF0100BDC
:100D700006F40043039306F4006305931A4B002125
:100D800018465A46069398F8008016F092FA4FF6E5
:100D9000FF72069BADF83C2002224FF0000A16EAD3
:100DA00002018DF83E208DF83FA01E4620D022A9DA
:100DB00021F84CBD0D4808F0CBF80423337007220E
:100DC000012386F801A0B370F2709A4611E000BFCB
:100DD0009DDB0008AC9C0108000C0140003800407D
:100DE00015202000E33300203C15002000080140BE
:100DF0008A46B8F1010F12D9202222A921F84C2DE0
:100E00009F4808F0A5F8052201233272B3720AF157
:100E10000102072386F809A0F3725FFA82FA039BA6
:100E20008BB122A9022221F84C2D954808F090F8A8
:100E300001220AEB0201072386F805A03271B27184
:100E4000F3715FFA81FA059B93B1022222A921F87E
:100E50004C2D8C4808F07CF8092201233273B373BF
:100E60000AF10102072386F80DA0F3735FFA82FAF4
:100E70006268854842F4404262606269DFF8088235
:100E800042F001026261A26942F40072A26107F0BD
:100E90003BFE7E4A002417927D4ABAF1010F189258
:100EA00094BF224680221C924FF480721D924FF410
:100EB00080621E92202240461F9217A94FF40052D2
:100EC00020921994CDF868A01B94219407F0FEFDA0
:100ED000D8F800206F4942F00102C8F800204A68A3
:100EE000BAF1010F22F4702294BF0020012022F4F5
:100EF000807242EA00224A608868674A0AF1FF333A
:100F0000024042F4602242F002028A60CA6ADBB206
:100F100022F4700242EA0353CB6201233219917822
:100F2000002963D0305D591C0928C9B2D278DFF896
:100F300064C112D9A0F10A0EDCF80CA00EEB4E0E23
:100F40004FF0070808FA0EF82AEA080802FA0EF22B
:100F500048EA0202CCF80C200FE0DCF8108000EB2D
:100F6000400A4FF0070E0EFA0AFE28EA0E0E02FAA9
:100F70000AF24EEA0202CCF81020062BDFF814E148
:100F800010D8013BDEF8342003EB83034FF01F0C35
:100F90000CFA03FC22EA0C0200FA03F31343CEF826
:100FA000343022E00C2B10D8073BDEF8302003EB66
:100FB00083034FF01F0C0CFA03FC22EA0C0200FA28
:100FC00003F31343CEF830300FE0A3F10D02DEF847
:100FD0002C8002EB82021F23934028EA030C00FAC4
:100FE00002F34CEA0303CEF82C300B460434102CE9
:100FF00094D1284B9A6842F480729A609A6842F0C1
:1010000001029A609A6842F008029A609968214A3F
:101010000C0743D5FAE7013A092A3FF611AAD8F896
:101020002C0004935946C7F814A0CBF8000003988D
:101030000EF0B5FC039B3C201A46082313610CF00C
:10104000C0FF049BC7F810A01F4695F891319F423E
:10105000BFF6F0A9039BDFF82CA04FF00808CAF8F0
:1010600010807820C3F814800CF0A0FF039BCAF80E
:1010700014807820C3F810800CF098FF0137E4E763
:1010800000080140000C0140080002404C240140CF
:101090004C15002000240140FDF7F1FF936843F058
:1010A00004039360BF4B9E6816F00406FAD1BE4C51
:1010B0009A68B4F85C0142F4A0029A60002840F0FB
:1010C0002186B4F95E31002B40F01C86B4F9603102
:1010D000002B40F017863B6898031FD5C8200CF002
:1010E00070FFAE200EF017FE08B10EF019FE85F865
:1010F0007501C8200CF065FFAC4B0021C5F87831B4
:10110000AB4D0C22284616F0D4F80223EB7008F001
:10111000EFFB0CF02FFFA74B0344AB60A64DB4F8D8
:101120000CE02B68B4F8640194F8631194F86B2117
:10113000B3F95630CDF800E094F80FE0CDF804E0B4
:1011400005F032FF10B903200CF0B6FF99F800301B
:10115000102243F0020389F80030984B4FF00A0840
:101160005A6108221A61DFF854921920D9F80C301C
:1011700008F1FF3883F01003C9F80C30D9F80C30AF
:1011800083F00803C9F80C300CF01BFF01200CF0B1
:1011900037FF19200CF015FF00200CF031FF18F07C
:1011A000FF08E0D10823C9F810304FF0100A844B33
:1011B000C9F810A01A68984612F0080F09D0814BA0
:1011C000C9F814A01B6898477F4B0122C9F810A0EA
:1011D0001A707E4BDFF81C921B68187B12F016FB0E
:1011E0007B4912F067FB09F087FA8246B9F80000E4
:1011F00012F00CFB514612F05DFB16F067FA754BCE
:101200001880B9F8000012F001FB0146724812F094
:1012100005FC724912F002FC714B6D491860714B6C
:10122000186912F047FB704912F044FB6F4BFF2125
:1012300018606F4B1A22184616F03BF8DFF8B8E139
:10124000002273460270D8F80020012112F0020F2C
:101250008EF800101FBF417003218EF8001002218C
:1012600018BF8170510741BF9EF8001001F1010EB7
:1012700083F800E04FF0030E48BF00F801E012F0E1
:101280000A0F0ED01A7804218154511CC9B24FF0B4
:10129000050E00F801E0D11C02321970D2B206210D
:1012A000815439688F0641BF1A78571C1F70072771
:1012B00048BF87540A0608D51A7809278754971C0F
:1012C00001321F70D2B20A2787546779082F01D0E4
:1012D0000E2F08D11A7802F1010E83F800E04FF0CA
:1012E0000B0E00F802E01A7811F4803F4FF00C0C5E
:1012F00000F802C002F1010E1CBFDFF8FCC0023290
:101300005FFA8EFE83F800E01FBF8CF80020384A99
:101310004FF00E0C02F80EC04A0748BF1A784FF083
:10132000120C41BF02F1010E83F800E04FF0100EE5
:1013300000F802E01A7811F4806F02F1010E5FFAF2
:101340008EFE83F800E000F802C00ED094F810C2C0
:10135000BCF1000F09D0DFF8A0C002328CF80020E9
:10136000234A4FF0130C02F80EC01A7811F4007FD4
:101370004FF0140C00F802C002F1010E1CBFDFF8A0
:1013800078C002325FFA8EFE83F800E01FBF8CF84F
:101390000020174A4FF0150C02F80EC0182F41D14B
:1013A0002CE000BF00240140EC290020742B002019
:1013B000D0260020404B4C00E00F0020000C0140E4
:1013C000A4100020B8120020E0120020782600208F
:1013D00035FA8E3C9C2600200AE81C4100401C4641
:1013E000FC01002010120020BD3786357426002035
:1013F000AD0F00201C000020AC0F00201A784FF029
:10140000160E00F802E002F1010E5FFA8EFE4FF0B8
:10141000170C00F80EC002F1030E0232D2B283F8AC
:1014200000E087540A0341BF1A78511C1970192330
:1014300048BF835400219822A14815F03AFF05F0D7
:101440002AFDA04AA04BA1491A6000234B800B71D2
:10145000B4F896019E490A6081B29E4A22F81310A0
:101460000133122BF9D19C4F3B681B0740F1DB8005
:1014700094F89031062B00F2D080DFE803F00404EA
:10148000345A718D8D009549954A012B0A60DFF819
:10149000BCE2944894490AD14FF0030C8EF800C086
:1014A0004FF0070E0B7080F800E00C2307E00223DA
:1014B0008EF800300323037000230B700723137092
:1014C0008A4A8B4B40201A6007F092F8002800F0FF
:1014D000A48001234FF0000B90F9000040218DE81B
:1014E0000808844A39E012F091F9834912F0E2F9D0
:1014F000824912F0D5F812F0C9FB0023804A42F865
:1015000023000133122BF9D1794A7E494020116022
:10151000734A137007F06CF800287ED001234FF057
:10152000070A90F9000040218DE80804764A774BBD
:101530006DE0774A6E4B40201A60694B10221A709A
:1015400007F056F8002868D001234FF0000990F901
:1015500000008DE808026F4A40214FF4E13356E065
:101560006D4A634B40201A605D4B08221A7007F0E9
:101570003FF8002851D001234FF0000C90F90000F3
:1015800040218DE80810654A4FF4E13306F006FF6C
:10159000634BC3F87C013CE051490C22062BDFF879
:1015A000B0C1DFF8B0E15F480A7010D000238CF8BA
:1015B00000308EF8003003705B4B1B2119705B4BC1
:1015C0004FF4E1391A705A4B05221A700EE00021CF
:1015D00001708CF800108EF800105349212008701B
:1015E0005249DFF874910A70514A1370514A404BC6
:1015F00040201A6006F0FCFF78B101234FF0000E86
:1016000090F900008DE808404B464B4A402106F017
:10161000C5FE003018BF012028B9082009F05EF986
:10162000334B00221A603B682D4A13F4804F1FBFD2
:101630000821117041482E4918BF086042F201018B
:10164000194051B12A493E480860980444BF082116
:101650001170D90744BF0C21117011781B06A1F13C
:101660000401517040F1B880364B2D484FF0000A0C
:10167000DFF8E890C0F880315146152200F5C270BD
:10168000039389F801A0C9F804A0C9F808A015F0CF
:1016900010FE039BDFF8C8B0053B5046CBF8003086
:1016A0000BF079FF284B02201B68C9F80C3006F0BC
:1016B0009FFFDE46002855D1802009F00FF984E015
:1016C0006C110020742B0020C00E0020A8330020D5
:1016D000E8150020C82900208C290020DC0000200B
:1016E000EC150020E00000208B130020018800088A
:1016F000E415002075890008CDCCCC3F0000B04433
:101700001C140020558800087D8A0008A08601006E
:10171000418800080D8A000829880008C18900084E
:101720003009002084140020861400208913002032
:101730008714002055870008A188000885880008C4
:1017400091880008D22B0020B0290020D80000206A
:101750008A1300208514002090D003001802002076
:101760003802002090F805C099F80130CC490C22CD
:1017700002FB03125278624504D00133DBB2042B22
:10178000F4D9002389F80130DEF8003099F80120FF
:101790001B7890F90000002B4FF00C0303FB0213A1
:1017A00014BF4FF0030E4FF0010E00225B78CDF80E
:1017B00000E00192022106F0F1FDBA4B186000280A
:1017C0003FF47AAF01200BF0E6FE2868B64B00F537
:1017D000C5721A600BF086FF3B68980555D5B34A71
:1017E000B34D049B4FF010092B609369B14843F04F
:1017F00001039361049B0EA91B888DF83A90ADF804
:10180000383002238DF83B300EF0C9F82B68A94818
:101810005B880EA9ADF8383004238DF83A300EF00D
:10182000BEF82B680120197A0EF0A4F82B68A24AA2
:101830005B684FF0000A536117A88DF861904FF074
:10184000010917938DF860A08DF8629007F042FBB4
:101850002B680FA85B7A8DF83EA08DF83C300323EF
:101860008DF83D308DF83F9011F002F8934B944A7B
:101870001B683C3B1360D8F800304FF0FF3243F058
:101880001003C8F800308F4B1A608F4B8F4A904D71
:101890001360904A803313603B684FF00008D9030F
:1018A00085F8008040F1B88010F080F840F22A3CC2
:1018B000DFF854B2DFF8F4A14FF001096246584650
:1018C0004146CDF80CC085F8009015F0F2FCDAF82E
:1018D0001830814843F00403CAF818304023ADF8AB
:1018E000383018238DF83B300EA903238DF83A3099
:1018F00007F02EFBDAF81C30784943F00203CAF8EF
:101900001C30774B774D1B68AAF6947AB3FBF1F342
:101910002988013B21F45C710904090C29809BB2E0
:101920001D21A9852B85A5F814902B8C23F001038C
:101930001B041B0C2B842B8CA888298B23F00203FF
:1019400021F0730109041B04090C1B0C41F0600118
:1019500080B243EA0903A8802983A5F834802B8448
:101960002B8B23F008031B041B0C43F008032B8371
:10197000B5F844306FEA43436FEA53439BB2A5F88E
:101980004430DAF8A83F43EA0903CAF8A83F5046B2
:1019900007F0BAF8544BDDF80CC0179380231C9362
:1019A0004FF48073CDF860B01D934FF0100B4FF4DF
:1019B0000053504617A92093CDF86C80CDF878805D
:1019C000CDF87C80CDF88480CDF864B0CDF868C0C7
:1019D00007F07CF8AB890FA89BB243F40073AB818E
:1019E000DAF8003043F00203CAF800308DF83CB05A
:1019F0008DF83D908DF83E808DF83F9010F038FFC7
:101A00003A4B1A683A4B43F826200136202EF7D17C
:101A10000DF0D2FE0DF0D0FE3B685A0540F18F80EC
:101A2000344D354BD5F8C4840420C3F8008006F04B
:101A3000DFFD0421C5F8C80406F0B6FD2F4B85F87C
:101A4000CC040820C3F8008006F0D2FD0821C5F8B8
:101A5000D00406F0A9FD2A4E85F8D40400213046B2
:101A60002C2215F026FC8E2373704FF07C0AE023A5
:101A70004FF07D09F37086F800A086F82B90214E78
:101A80002C220021304615F014FC8A23737010209C
:101A9000A023F37086F800A086F82B9036E000BFF4
:101AA0007C980108CC2600201C0F0020001002406A
:101AB00014020020000C014000040140B029002065
:101AC00010020020001000200C2C00202413002005
:101AD000A9080020102700200008014000366E01F0
:101AE0005C0000200004004034040040B49C010865
:101AF000AA0800203009002098100020F0100020D3
:101B0000C0100020F5100020C90A0020C5F8D884B4
:101B100006F06EFD1021C5F8DC0406F045FD85F8E1
:101B2000E0042020C5F8E48406F062FD2021C5F819
:101B3000E80406F039FD85F8EC0407F0D9FD814B87
:101B4000814D1B78022B67D1804A002613883220F2
:101B500023F040031B041B0C138013884FF48058A0
:101B600023F038031B041B0C138013889BB243F033
:101B7000400313809F238DF83C308DF83D608DF835
:101B80003E608DF83F600CF01CFA8DF85D60704E81
:101B90000422C6F8148017A80FA910F087FEC6F813
:101BA00010809DF85E309DF85D201B0243EA0242E2
:101BB0009DF85F301343674A934219D00AD8A2F5C3
:101BC0001A42033A93420CD002F51A42023293426F
:101BD00009D01CE0604A934205D00132934207D0FD
:101BE00015E0202300E080232B804FF4807302E077
:101BF0004FF480732B806B80AB882A881B02AB600C
:101C00005343EB60554B012283F8ED2404E000239D
:101C10002B806B80AB60EB60ED680DB32D0CA8469C
:101C20004FF00009A94514DA09EB050676100DF10D
:101C30005C0A3004514610220EF01EF800235AF8B8
:101C4000232001325AD10133042BF8D1B046354656
:101C5000E8E70BF00BFF414B4FEA0842C3F8F024D2
:101C60003B683F4A13F4002318BF012313700CF0A4
:101C700081F93C4B18606379052B02BF3A4B4FF456
:101C8000C8721A80394B4FF47A721A80384BC822C6
:101C90001A80384A137843F008031370364A1378D1
:101CA00023F00203137040F602033A6813406BB14D
:101CB0003249334B1960334B03211970324B0121E8
:101CC0001970324900230B8031490B80930341BFC7
:101CD000304B04221A71DA7844BF42F00102DA7004
:101CE0002D4B01229B683B602C4B1A702C4A1378B9
:101CF00063F07F03137023B0BDE8F08F06F1010994
:101D00002E46A4E7274B00221A7000B211F07EFD88
:101D1000254911F0CFFD1790B4F95E0111F076FD61
:101D2000214911F0C7FD1890B4F9600111F06EFD62
:101D30001D4911F0BFFD1D49199017A808F0E6FCD8
:101D4000FFF7C9B9E33300200C0000200038004041
:101D5000000C014018BA20001740EF0030090020A5
:101D6000C0310020BC020020D20E0020DA33002057
:101D7000D8330020A8100020E1330020662B00207B
:101D800090100020F410002050000020400E002091
:101D9000420E0020D0260020EC290020A8080020B8
:101DA000B83300202800002035FA8E3C181500209A
:101DB000B54B2DE9F04FB3F90610B44B85B01F6851
:101DC00001937A8991420EDBB1F5FA6FFC79BFBFBE
:101DD0008B1A6343A2F5FA6493FBF4F4ACBFC4F12D
:101DE0006404643400E06424A94BAA4AB3F896B1B1
:101DF00093F9623112689BB2029215460393002256
:101E000040F2E630A04B4FEA420C33F912E0CBEB44
:101E10000E0303F2F316864203D8002BB8BF5B42D1
:101E200001E04FF4FA73022A2ED0029E96F8116157
:101E30001EB1B342CCBF9B1B0023642093FBF0F880
:101E4000954E6FF0630A36F818900AFB083A08F1CD
:101E5000010836F918600FFA89F8C8EB060606FB88
:101E60000AF696FBF0F68D484E4420F80C60BE183A
:101E70003679642073438A4E93FBF6F364339BB246
:101E8000634393FBF0F02CE0029890F812611EB1CE
:101E9000B342CCBF9B1B0023642093FBF0F0DFF820
:101EA0002C926FF0630808FB003A39F9106001309A
:101EB00039F91000002BA0EB060000FB0AFA9AFB90
:101EC000F8FA0398C6EB0A0A0AFB00FA7348B8BF8F
:101ED0005B42A0F804A0B8794343714893FBF0F04B
:101EE00064306B784FF06408434393FBF8F36D4E16
:101EF000022AB354EB7A6C4E00FB03F393FBF8F326
:101F0000B3546B7D654E00FB03F090FBF8F0674B1C
:101F10009854674B0ED1DE4583F802800DDB5C4C94
:101F2000B4F89821914214DBB1F5FA6FA8BF4FF4D1
:101F3000FA610FE0DE459C5404DA36F80C305B425F
:101F400026F80C300132032A05F101057FF458AF61
:101F5000E5E71146891A4FF47A735943C2F5FA62DC
:101F6000B1FBF2F1642391FBF3F2DFF874E16FF05F
:101F700063073EF8120007FB021101323EF91220FE
:101F800007B2D21B514391FBF3F30344F380494B57
:101F9000424D1B885F063BD5474A484B10881B883B
:101FA000181A00B211F032FC454911F083FC0746C3
:101FB00008F0A2FB8046384608F02BFB0746B5F92F
:101FC000020011F023FC8146B5F9000011F01EFC5F
:101FD0004146824611F06EFC39468346484611F070
:101FE00069FC0146584611F05BFB11F029FE4146A1
:101FF0002880484611F05EFC39468046504611F074
:1020000059FC0146404611F04DFB11F019FE688065
:102010002C4D2B68980740F19E8045F207212A4BF2
:102020002A4F1A687B69D31A8B4240F394807A61F5
:1020300007F0FCF8264BDFF8AC901A789846032A94
:10204000B9F8003050D10A2B58D90023282088F83D
:1020500000300BF0B6FF07F0E9F81E4B188807F0C8
:10206000CFF81D4B1A68D37890FBF3F001300828A5
:102070001A4BA8BF08201870537980B243433B83A2
:1020800013795843788339E0C829002008100020CC
:10209000EC290020E00F00204213002088100020CF
:1020A0000CFEFFFF48270020360E00205C27002092
:1020B000A824002068110020160F002080100020A6
:1020C00035FA8E3C8C290020C0330020280E0020D9
:1020D000F410002054150020901000205000002023
:1020E0002A130020941000200A2B07D803239B4AB0
:1020F00088F80030002313703B837B8398F800300E
:10210000974A012B0CD002D3022B1BD023E03A8B31
:10211000B9F800309A421EDD012388F800300FE044
:10212000B9F800107B8B8B4202DD022313700FE0A5
:102130008C4B1B8B0133994202DD002313700AE0A4
:10214000082006E07B8BB9F8002001339A42E3DCDB
:1021500007200BF073FF2D68290575D5824B814F41
:102160001A68FB69C3EB020845F2072398456BDD4B
:10217000B6F906304FF47A71A3F57A7B7B4BFA619E
:10218000D3F8009098FBF1F899F80A30B4F85201AE
:10219000012B774E03D040D3022B1FD03FE0754B6D
:1021A000386A5A7B744B4FF0080E33F8122090FBBC
:1021B000FEF392B2C01A83183B6293FBFEF3BA841B
:1021C00040F6E4429BB25343B9F80820C2EB133304
:1021D0004B43B9F9062093FBF2F31FE0674BB9F8C4
:1021E00008A01B78C6F800A05A0718D510F0FBFD10
:1021F00020B915F0100F18BF4FF0000B0BFB0BF1BF
:10220000322391FBF3F3B9F906205B445A434FF4B0
:102210007A7392FBF3F3534400E000233360336896
:10222000D7E90A0103FB08F84FF47A7398FBF3F837
:1022300010EB080041EBE8710023C7E90A01504A9E
:1022400011F044FD4F4B18604F4E3368DB0427D527
:102250002F0622D54D4B1B789D071ED54C4B187869
:1022600004281AD900224B4B0521D718951C4FF092
:102270000A0E122AD154E9B287F801E004D0B0EB7B
:10228000510F2A46EFD800E014215A18322002F8E4
:10229000010CFF225A540F2000E00A200BF0CEFE62
:1022A0003D4D2A68002A51D03C4B3D4F1868396893
:1022B000984681424AD83B4BDFF8F490197852682F
:1022C000E1B94FF0010A83F800A0B9F80030D35CFF
:1022D00023B350460BF094FE334B83F800A011F06B
:1022E0009FF9B9F80030CBB92B681B78053B5345F3
:1022F00014D80BF03FFE2D4B18600FE04FF0000A92
:1023000083F800A0B9F80030D35C3BB150460BF025
:1023100077FE254B83F800A011F082F92B68B9F8FD
:1023200000205B6822499B5CFE2B02D100230B80BE
:102330000CE0FF2B02D10BF069FE07E0D8F800009B
:102340000A2505FB030301323B600A800B4D2B7805
:10235000580731D5174B08225A616BE05000002016
:10236000F4100020280E0020C03300209010002020
:102370009C1000203C1500204C150020E13300206B
:10238000407E0500A0100020A80F0020A81000200B
:10239000AE100020142800204C250020B029002079
:1023A0004425002040250020B03300207433002055
:1023B00048250020000C01403268D1075CBF43F083
:1023C00001032B70984B1B781F075EBF2B7823F0FF
:1023D00001032B70D60248BF2B78944A44BF23F0E8
:1023E00001032B70924B1B6813F0040F02D091492C
:1023F000098851B99049098809B1980705D48F4BCC
:102400001B88003318BF012333B1022313702B78CC
:1024100023F001032B7004E02978C90758BF022379
:1024200013700BF0A7FD864B1B68C01A002801DB58
:1024300011F0F6F807F05CF9824B1E789846002EF2
:1024400000F0AB80804E3368002B00F0E7863068E8
:102450000BF086FE002800F0E1867B4B7B4C186871
:102460000BF07BFE092801D03F2850D14FF0000A25
:102470005746D4F80090764DB9F1000F05D0754855
:1024800029684A4614F062FF10B9AA4607B92F46D8
:10249000714B10359D42EFD3C7B1D7F800E0DAF8A1
:1024A00000C023681EF803501CF80300A8420DD199
:1024B0005A1C684938B92D2B05D8644D2A6020254F
:1024C000CD54885402E0CD542260EAE723680BB172
:1024D000574511D061480EF055FF574507D857F8BA
:1024E000100B0EF04FFF09200EF044FFF5E75C489B
:1024F0000EF048FF4FF0000923689945A7D2554BCD
:1025000013F809000EF036FF09F10109F4E723681A
:10251000002B40F06886042840F0A6864D480CF059
:102520000FFC00F07BBED9F80000DFF844A10BF0EF
:1025300017FE40B3DAF800000BF00FFEDBF80030B6
:10254000024693F84810002935D1242840F09280A3
:10255000012283F84820DBF80030DFF810A193F85F
:102560004820062ADFD193F8490002F0C7FF8146D0
:10257000002800F0A3803B6898790EF050FE3B687D
:10258000002283F84820374B93F83530002B40F079
:1025900018864C36982E00F04186334BF21892F88C
:1025A0004A100129F5D1314FF3583A60304ABB4601
:1025B00013609146B7E7012904D14D2814BF0022CA
:1025C0000222C6E7022904D13C2814BF00220322BC
:1025D000BFE703290CD140284FF0000102D983F84E
:1025E0004810B8E758711971D97198710422B0E791
:1025F000042906D1997983F849004A409A71052245
:10260000A7E70529A7D1587919798842987906D979
:1026100050409871481C18710B441A729BE7904205
:102620000CBF0622002294E7A8100020B03300203F
:10263000A4100020D8330020D20E0020DA3300206E
:10264000B4330020E5330020CC2700200C270020E5
:1026500004A50108DC260020E4A601084CBF0108FF
:1026600051BF0108280E00206C11002048110020E5
:102670004C1100202B7858073FF56DAF232ADAF86C
:1026800000300ED1012188F80010AE49AE480B6031
:10269000AE4902920B630EF075FEAD480EF072FE6D
:1026A000029AAC4B1B681B78934201BFAA4AAB4B02
:1026B0001A60AB4A04BFAB4BDA604CE7DAF8002093
:1026C00092F849304A2B00F038815CD8332B00F067
:1026D0009E8421D8292B00F0388409D8252B00F0BE
:1026E0000F84272B00F01384232B40F0B9853CE2A4
:1026F0002D2B00F03B8407D82B2B40F0B1850EF03A
:1027000071FD607100F058BD2F2B00F00885312B52
:1027100000F01A8500F0A4BD3E2B00F004811DD806
:10272000372B00F0C48404D8352B00F0578200F01A
:1027300097BD392B00F0F8833C2B40F09185DFF8F2
:102740002892D9F800A00EF04DFD8AF80000D9F8C3
:10275000003018780CF030F900F02EBD432B00F05B
:10276000838406D8412B40F07B854FF0000900F0B0
:1027700053BC442B00F01C85482B40F071850BF0B6
:10278000B3F900F019BDD02B00F0338368D8CA2B01
:1027900000F0F2801CD84E2B00F00B8410D84C2B8C
:1027A00040F05E850EF01EFD84F8CE010EF01AFD9D
:1027B00084F8CF010EF020FDA4F8D00100F0FCBC9D
:1027C000C82B00F08380C92B00F0348300F048BD93
:1027D000CD2B00F0198304D8CC2B00F0278200F019
:1027E0003FBDCE2B00F01983CF2B40F039850EF082
:1027F00003FD6FF4AF6283189BB2C62B98BFA4F899
:1028000096010EF0F9FCA4F844010EF0F5FCA4F8D2
:1028100046010EF0F1FCA4F848010EF0EDFCA4F81E
:10282000D0010EF0DFFC84F8E1010EF0DBFC0EF0CD
:10283000D9FC84F8E2010EF0D5FC84F885010EF095
:10284000D1FC84F892010EF0CDFC474BD3F80090F8
:102850000EF0D2FC00EB80004000A9F8560063E3C4
:10286000D62B00F04B820AD8D22B19D0C0F00983A6
:10287000D32B25D0D42B00F04C8200F0F1BCEF2BF1
:1028800041D005D8D82B40F0EB844FF00009FFE091
:10289000F22B00F08682FA2B00F0C88200F0E0BC38
:1028A0002B78590700F188840EF09CFC022884F8EC
:1028B000A80740F2A4822D4B002283F8A8279EE2AD
:1028C0000EF09AFC2A4B188000F076BC92F8059026
:1028D0004FEA5909B9F1120F03D905F001F800F0D8
:1028E0006BBC4FF0000ACA4507D20EF085FC214BA5
:1028F00023F81A000AF1010AF5E7144B012283F8C4
:10290000342000F059BCDFF86090D9F800A00EF038
:1029100073FCAAF85A00D9F800900EF06DFCA9F8E3
:10292000580000F049BC0EF05DFC84F8D4010EF0B4
:1029300059FC84F8D30100F03FBC0EF05DFCA0818F
:1029400000F03ABCCC27002081BF0108280E0020EF
:1029500051BF0108E4120020EFBEADDEF04F0020B1
:102960000400FA0500ED00E0E00F0020EC29002053
:10297000140F0020C8290020D64B1A689A461278F6
:10298000022A6AD1DAF8003009F1080B02930EF03E
:1029900029FC10F037FFD04911F040F8029B43F8B2
:1029A0002B00DAF800B00EF01DFC09F10A030BEB66
:1029B000830B10F027FFC94911F030F8DAF8003026
:1029C000CBF8040002930EF00DFC10F01BFFC4497D
:1029D00011F024F809F10E0B029B09F10109B9F17C
:1029E000030F43F82B00CDD1B9F1070FDAF800B08F
:1029F0001AD10EF0F7FB10F005FFB74911F00EF8F1
:102A0000CBF84400DAF800B00EF0ECFB10F0FAFE60
:102A1000B14911F003F8CBF84800DAF800B00EF035
:102A2000E1FB8BF84C0012E00EF0DCFBCB448BF8A2
:102A30000100DAF800B00EF0D5FBCB448BF80B00A8
:102A4000DAF800B00EF0CEFBCB448BF8150009F19C
:102A50000109B9F10A0FC7D1AEE3DAF800B00EF000
:102A6000C1FBCB448BF80100DAF800B00EF0BAFBE2
:102A7000CB448BF80B00DAF800B00EF0B3FBCB447C
:102A800009F10109B9F10A0F8BF81500E5D193E3BB
:102A9000DFF840A209F1080BDAF8003002930EF0DB
:102AA000ABFB10F0AFFE8E4910F0B8FF029B43F86D
:102AB0002B00DAF800B00EF09FFB09F10A030BEBD4
:102AC000830B10F09FFE864910F0A8FFDAF8003063
:102AD000CBF8040002930EF08FFB10F093FE8049B8
:102AE00010F09CFF09F10E0B029B09F10109B9F1ED
:102AF000030F43F82B00CBD1B9F1070FDAF800B080
:102B00001AD10EF079FB10F07DFE754910F086FFAA
:102B1000CBF84400DAF800B00EF06EFB10F072FE55
:102B20006F4910F07BFFCBF84800DAF800B00EF0E8
:102B300063FB8BF84C0012E00EF05EFBCB448BF88D
:102B40000100DAF800B00EF057FBCB448BF80B0015
:102B5000DAF800B00EF050FBCB448BF8150009F109
:102B60000109B9F10A0FC7D126E30EF03BFB132888
:102B700083463FF6B2AEDFF85CA1DAF800900EF0C3
:102B800031FB002357490C2202FB0312117A8142C8
:102B900020D1137809EB8B0989F879300EF022FBEC
:102BA00089F87A000EF01EFB89F87B000EF01AFB04
:102BB0004D4A4E4B89F87C001A60DAF800004C4B05
:102BC00000211860793005F09FFD4A4B80F001002C
:102BD0001870F1E201331B2BD4D17EE60EF002FB1C
:102BE0000B2882463FF679AE3A4BD3F800900EF0B0
:102BF000F9FA03283FF671AE062303FB0A9989F818
:102C0000CE000EF0EFFA89F8C9000EF0EBFA89F861
:102C1000CA000EF0E7FA89F8CB000EF0E3FA89F863
:102C2000CC000EF0DFFA89F8CD00C5E25379092B0C
:102C30007FF653AE019BD3F800900EF0D3FA019BC0
:102C400089F80000D3F800900EF0CCFA89F8010062
:102C50000EF0C8FA019B64281B68A8BF6420187195
:102C60000EF0C0FA019B64281B68A8BF642058714D
:102C70000EF0B8FA019BFF281B68A8BFFF209871CF
:102C80000EF0B0FA019B6428D3F8009028BF6420AE
:102C900089F807000EF0A6FA019B89F80200D3F824
:102CA00000900EF09FFA019B89F80300D3F8009082
:102CB0000EF0A2FA3B68A9F80A005B790A2B40F2F1
:102CC0007B820D4BD3F800900EF08CFA89F8080047
:102CD00072E200BFE00F0020000020410000C84267
:102CE00000007A44949D0108302B00200C0F002036
:102CF000100F002008000020081000200EF07CFAC1
:102D0000CB4B23F8190009F10109B9F1080FF5D1EE
:102D100052E253790F2B7FF4E0AD0EF063FA0728EF
:102D200081463FF6DAADDFF834A3DAF800B00EF0F2
:102D300063FA0E2303FB09F9CB44ABF81901DAF867
:102D400000B00EF059FACB44ABF81B01DAF800B032
:102D50000EF052FACB44ABF81D01DAF800B00EF0D9
:102D600041FACB448BF81F01DAF800B00EF03AFAC2
:102D7000CB448BF82001DAF800B00EF033FACB44E4
:102D80008BF82101DAF800B00EF02CFACB448BF866
:102D90002201DAF800A00EF039FAD144C9F8230173
:102DA0000AE20EF01FFA0F2881463FF696AD0EF0AC
:102DB00019FAC9EBC909A14489F8D4000EF012FA36
:102DC00089F8D5000EF00EFA89F8D6000EF00AFA4E
:102DD00089F8D7000EF006FA89F8D8000EF002FA4A
:102DE00089F8D9000EF0FEF989F8DA000BF07CFBC7
:102DF000E2E12B785B0700F1DF810FF0F1F907F0DA
:102E00009FFD07F03FFED7E12B78580700F1D481F2
:102E1000884B4FF4C8721A80CEE12B78590700F125
:102E2000CB81854A137843F0040328E02B785A07B6
:102E3000E5D515E20EF0D6F97F4B1A7810B142F0C5
:102E4000020201E022F002021A700EF0CBF97B4B75
:102E5000DFF80C9218700EF0D9F9C9F800000EF0E6
:102E6000D5F9C9F804000EF0C7F9754B18800EF0BB
:102E7000C3F9744B744A1880137843F0020313703B
:102E80009AE10EF0AFF902900EF0C0F983460EF011
:102E9000BDF982460EF0BAF981460EF0ADF90EF09A
:102EA000ABF90EF09FF9029BA3B9684B1020C3F851
:102EB00000B0C3F804A007F0F0FC5F4A137843F0B9
:102EC00001031370B9F1000F00F07681604BC3F875
:102ED000009071E1102B40F06F815E4BC3F800B0A1
:102EE000C3F804A0B9F1000F02D0594BC3F8009009
:102EF0005848594B0222011D1A700AF0ADFB5BE1E4
:102F0000A0600EF083F9A3681843A06054E10EF0AE
:102F100073F9A4F85C010EF06FF9A4F85E010EF0ED
:102F20006BF9A4F8600147E10EF05CF984F87A01CE
:102F30000EF058F984F87E010EF054F984F87D0102
:102F40000EF050F984F87F0136E10EF055F9A4F83F
:102F500080010EF051F9A4F882010EF043F984F8D3
:102F600084010EF049F9A4F8860125E10EF03AF942
:102F700084F890010EF040F9A4F89A010EF03CF9A3
:102F8000A4F896010EF038F9A4F898010EF02AF989
:102F9000DAF8003084F891015B79082B40F20C815B
:102FA0000EF02AF9A4F89C010EF026F9A4F89E016F
:102FB00002E192F805900323B9FBF3F9B9F10E0F82
:102FC0003FF68BACDFF89CA04FF0040BCB4580F0B4
:102FD000F3800EF007F98AF8A0010EF00DF940F227
:102FE000ED23984205DD40F6CA039842A8BF184673
:102FF00001E040F2EE20A0F2EE20192390FBF3F066
:103000000BF1010B8AF8A1010AF1020ADEE70EF0CA
:10301000E9F884F89201CFE00EF0E4F804EB09033C
:1030200009F10109B9F1080F83F88801F4D1C3E06F
:10303000B2270020D20E0020A8100020AE100020E1
:10304000AC100020AA1000200E100020101000204C
:103050002010002018100020180F0020E00F002082
:10306000B0100020EC2900200EF0BCF8C4F8089045
:1030700060710EF0CBF8A3681843A0600EF0B2F8B0
:1030800084F890010EF0B8F8A4F85C010EF0B4F8E2
:10309000A4F85E010EF0B0F8A4F860010EF0ACF8F0
:1030A000A4F880010EF0A8F8A4F8820184E0537916
:1030B0004FF0070AB3FBFAF2C2EBC2029A1A12F0FF
:1030C000FF0F7FF40AACB3FBFAFA0AF1FF3A5FFA9A
:1030D0008AFABAF1FF0F6FD00EF084F85FFA80FB26
:1030E0004FFA8BF005F0AAF9814600283FF4F5ABC2
:1030F00080F800B00EF080F8A9F802000EF072F827
:1031000089F804000EF06EF889F805000EF06AF8F0
:1031100089F807000EF066F889F80600D5E7DFF8B1
:103120005C9209F1400A0EF067F8A9F8A0020EF0CF
:1031300059F889F8A2020EF055F809F1040989F846
:103140009F02D145EFD137E00EF04CF81F288146A1
:103150003FF6C3AB3B685B79082B7FF4BEAB0EF048
:103160004BF809F1880904EB890A00F03F00AAF83E
:1031700002000EF041F8BAF80230800100F4FE506F
:103180001843AAF802000EF02DF8000104F82900F7
:103190000EF028F814F8293000F00F00184304F856
:1031A00029000EF01FF88AF801000EF0FFFB03E083
:1031B0005F4B012283F8352000200EF05FF8FFF707
:1031C000DAB95C4B98590AF0C2FF18B932200AF0FC
:1031D000F8FEF6E70BF046F907F088FB564A574B26
:1031E000DA60FFF7D6B90C2840D00A2847D1544DF1
:1031F00054480EF0C7F82846232114F090F808B17F
:10320000401B20602368002B5CD14D4800213022F8
:10321000236014F04EF898F8003053BB4A4B1B68FB
:103220009B0614D5494B42491B688A6B9A1A002A9F
:103230000DDB474A1278042A09D903F5123303F546
:10324000F873444A8B63D36883F01003D360424B16
:103250009B68002B69D0414805B0BDE8F04F184786
:1032600004F03EFBFFF787B90C2804D13C480EF070
:1032700089F83C480DE07F2812D1FFF7E8B80D2807
:10328000B5D07F2809D12E4A013B00213648236062
:10329000D1540EF077F8FFF7DAB82F2B3FF6D7A806
:1032A000A0F12002D2B25E2A3FF6D1A813B920289D
:1032B0003FF4CDA85A1C2260214AD0540EF05AF88F
:1032C000FFF7C5B85A1EA95C202901D113469AE719
:1032D0001B4A00212360D154244B254DD3F800A074
:1032E000D5F800B0DFF85890584614F026F8074695
:1032F00059463A46484614F029F81E4A28B919F8A2
:10330000073053445B785B0703D010359542E7D311
:1033100006E0954204D2781CEB684844984702E0E6
:1033200015480EF02FF800236FE705B0BDE8F08FC9
:10333000280E00206C1100200400FA0500ED00E0CA
:10334000DC26002091CE0108A4100020C03300200C
:10335000AE100020000C014010120020640E00206E
:1033600056BF010851BF01087DBF0108640000205D
:1033700004A50108E4A6010861BF0108EC290020AA
:103380009148F0B50368914A9C8AA4B2E1B211F069
:10339000010F2ED0198821F400610904090C19804D
:1033A000198889B241F48061198000211170517827
:1033B00099B1917811B9D178FF290ED1012191707D
:1033C0001179022901BF198889B241F4006119807D
:1033D000517941F001011982E1E0517901F0FE01DA
:1033E0001982D378FF2B00F0DA80784BFF21197017
:1033F000D5E08E073AD5BFF35F8F1479E4B2012C84
:1034000013D1517889B1917879B1198821F480610B
:103410000904090C1980BFF35F8F198B1988947107
:1034200089B241F4007119801BE0198BBFF35F8FE3
:1034300014796649022C0AD14C7844B1897831B1AB
:10344000198821F480610904090C1980A1E014791C
:103450005E49032C05D14C781CB18978002940F0D5
:103460009880998889B241F4806197E04D0756D5DC
:10347000012191715178002937D09178002934D0F9
:1034800011791C88022911781DD924F48064240440
:10349000240C1C801E8A9568CCB2F6B249B26E54D8
:1034A000198889B241F4007119800168A31C137056
:1034B0000B8A0134DBB264B22B558B889BB243F488
:1034C00080638B8026E0A4B244F400741C801D8AC3
:1034D0009668CCB2EDB249B275541B8A611C49B2F0
:1034E000DBB203347354147014E09178374C09B98B
:1034F000217B41B1198889B241F400711980137898
:103500000133137006E0198889B241F48071198083
:103510000123A37001680B88DB05FCD43FE001F0B8
:10352000400101F0FF05E1B114781F8A9668E5B209
:10353000691C64B2FFB23755C9B21679117049B22D
:10354000CC1CA64201BF9C8824F480642404240C73
:1035500008BF9C8013798B4221D11C4B02351D7012
:103560001DE027061BD511784CB2661C0AD01569E0
:1035700001312C5DC9B21C821479117049B28C42A0
:103580000DD106E0D17815701982517809B91179F9
:1035900029B9998821F480610904090C998013796B
:1035A00092F9004001339C4208490CD100238B70F2
:1035B0008B7933B101688B8823F440731B041B0C97
:1035C0008B8000231375F0BD2C270020680E00208F
:1035D0006B4B6C4A2DE9F04F5E8994694FEA062ADD
:1035E000B4EB0A0A9C884FF000054FEA04481C8996
:1035F0004FF0000BA4FB0A6765EB0B0B04FB0B778A
:10360000F40944EA476418EB04065C884FF00009AB
:103610004FEAE7154FEAC438DC8849EB050787B065
:10362000CDE90467A4FB0A6704FB0B77340A44EA7C
:10363000076418EB04064FEA27259C894FF0000920
:1036400049EB0507CDE90067AAFB046704FB0B778C
:10365000F40D44EA472414F5FA664FEAE75545F1BC
:103660000007B6F5FA6F77F10003CDE902679646D9
:1036700066DADDE90489A4FB046704FB05F34FF077
:10368000050C07EB4307A6FB0C230CFB07335F106D
:103690004FEA3206B8EB06084FEA920646EA83760E
:1036A00069EB07099F10DDE90023921B63EB070319
:1036B000CDE90023DDE90267334A4FF0FF3396423C
:1036C00077EB0303CDE9048927DA40F6AC520023F7
:1036D000A4185D4104FB05F3A4FB04456FF006024A
:1036E00005EB4305664202FB0566A4FB0223334457
:1036F00018EB020649EB0307CDE904670B26A4FB90
:10370000062306FB0533DDE900455B104FEA320274
:10371000A41A65EB0305CDE90045DDE902450AFB86
:103720000BF3AAFB0AAB0BEB430B4FEADA7242EA4C
:103730004B02A41A4FEAEB7365EB0305CDE9024592
:10374000DEF81C40009B019DA4FB032304FB053312
:103750004FEA525848EAC3284FEA6359DDE9042387
:10376000B8EB020269EB03039946D30B43EA4943E2
:1037700000B1036009B1029B0B6007B0BDE8F08F98
:1037800030120020680E002024FAFFFF2DE9F04FD0
:10379000DFF8589285B00746D9F820000E4610F0A1
:1037A00035F88E4C8046208810F02CF84FF05C5194
:1037B0000546404610F07EF84FF064518246284698
:1037C00010F078F8014650460FF06AFF4FF0625152
:1037D0008246404610F06EF84FF06A518046284607
:1037E00010F068F8014640460FF05AFF0546B4F95C
:1037F000020010F00BF80146284610F05BF8514625
:103800000546504610F056F88046B4F904000FF013
:10381000FDFF0146404610F04DF8014628460FF0E6
:1038200041FF804610F00CFA6D490546A061404604
:1038300010F0F4F8D9F824308046284601930FF0B0
:10384000E5FF4FF07C5110F035F866490FF028FF86
:103850000546E389B4F90A0002930FF0D7FF294621
:1038600010F028F8294610F025F84FF0585110F0C4
:1038700021F88146B4F90800B4F810B0B4F80CA0EF
:103880000FF0C4FF294610F015F8014648460FF026
:1038900009FF4FF0585110F00DF84FF0605110F043
:1038A00009F84FF07E510FF0FDFE8146E0880FF0E1
:1038B000A9FF014648460FF0FDFF0021814610F0A8
:1038C0008DF900287BD1294628460FF0F3FF03909D
:1038D0000FFA8BF00FF09AFF039B014618460FF08A
:1038E000E9FF4FF060510FF0E5FF8346BDF9080096
:1038F0000FF08CFF014628460FF0DCFF01460FF069
:10390000D1FE014658460FF0CDFE4FF07A510FF030
:10391000D1FF834601980FF079FF01464FF09340A5
:103920000FF0BEFE05460FFA8AF00FF06FFF4FF062
:103930008F410FF0BFFF014658460FF0B3FE4FF026
:1039400066510FF0B7FF014628460FF0A9FE264941
:103950000FF0B0FF494610F061F80546B4F91600C3
:103960000FF054FF29460FF0A5FF29460FF0A2FFE4
:103970004FF040510FF09EFF8146B4F914000FF054
:1039800045FF014628460FF095FF4FF060510FF0BC
:1039900091FF014648460FF085FE8146B4F91200BA
:1039A0000FF034FF014648460FF07CFE4FF0765191
:1039B0000FF080FF014628460FF074FE00E0002063
:1039C00017B110F03DF938602EB1404610F038F9CB
:1039D00064235843306005B0BDE8F08F901200209A
:1039E0000000A04500007A470050C345680E002043
:1039F000704770472DE9F041324C334D62892B8D71
:103A0000B4F904809A1A2389B4F902E05A43B4F94C
:103A10001230D613B4F91420DB02324493FBF2F2D5
:103A200032440A26E2615643A2F57A6202FB02F3AF
:103A3000B4F90EC002FB0EFE02FB08F2B4F90C80D2
:103A40001B130CFB03FC03FB08F31B1403EB623298
:103A50000232E388921002F5004253434CF2503296
:103A6000B4F920704FEAEE2EB4F900400EEBEC2CC6
:103A70000CEB8404BC40ED6A0234A5EBA4043A418B
:103A800062434FEAD3384EBFB2FBF8F35400B4FBA5
:103A9000F8F340F6DE3448BF5B001A12524362432B
:103AA0000A4C08365C43241404EB224202F6CF622F
:103AB000361103EB221300B1036001B10E60BDE8C3
:103AC000F08100BF44120020680E002043E3FFFF96
:103AD000024B4FF480521A80704700BF1C00002038
:103AE00010B5224C2368998A89B211F4706F1EBFF9
:103AF0001F4A012082F8300011F4E06F2BD01A8B9E
:103B00009A88890522F480624FEA02424FEA124203
:103B10009A8020D41A8892051DD41A88D0050FD512
:103B20001A88D105FCD41A8892B242F400721A8025
:103B30001A889205FCD40F4B18780CF081F90AE032
:103B40001A8892B242F400721A809A8822F4407263
:103B50001204120C9A802268938A23F470631B0467
:103B60001B0C9382024B00221A7510BD2C270020DB
:103B7000680E002030270020054A08B5138801335D
:103B80009BB21380034B18780CF05AF9002008BD43
:103B9000A60F00203027002008B54FF4804005F024
:103BA000C9F9012801BF044B4FF480425A61034B0D
:103BB00008BF83F8310008BD00040140680E0020F2
:103BC00010B5054C2368186905F0B4F918B12368DD
:103BD0001A69024B5A6110BD2812002000040140EE
:103BE00070B50E46054C4FF4805565610EF094FE9D
:103BF00030460EF091FE256170BD00BF000C014003
:103C00001D4B07B51A681D4B9A420ED14FF4005355
:103C1000ADF8043002238DF80730042318480DEB6B
:103C200003018DF806300BF0BAFE80216B20FFF700
:103C3000D7FF64200AF0C5F900216B20FFF7D0FF01
:103C400064200AF0BEF96B200121FFF7C9FF1B2099
:103C50001821FFF7C5FF1C201021FFF7C1FF094BFA
:103C60001A201978FFF7BCFF19200021FFF7B8FFD1
:103C700003B05DF804FB00BF24000020001BB70068
:103C80000010014022000020F0B5264D85B095F8C7
:103C90003230002B44D1244C2368002B40D01A68CA
:103CA000224E12B1B1690A43B2619A889868ADF8A0
:103CB000002002228DF80320694604228DF802209C
:103CC0000BF06DFEB369002743F00103B361236875
:103CD0000126197D187B0BF04DFE15480AF022FADB
:103CE0002368144A1B695361029308230DEB0300F8
:103CF0008DF80D308DF80C708DF80E6005F0EAF837
:103D0000236801A85B7D8DF806708DF804300323CD
:103D10008DF805308DF807600EF0AAFD85F8326049
:103D200005B0F0BD680E00202812002000100240EF
:103D3000C13B00080004014008B5FFF7A5FF074B91
:103D40001B7813B1012B03D008BD4FF4006201E0D2
:103D50004FF48052024B1A8008BD00BF2D12002084
:103D60001C00002010B51E4C4000C0B2A3602361AF
:103D70001C4B6071E1700120002121736070227181
:103D80002075186884F8301040B383889B0515D4DB
:103D90000388D9050DD447F230530288920502D525
:103DA000013BFAD112E08BB103889BB243F48073DC
:103DB000038083889BB243F44073838047F230537F
:103DC000227D12B1013BFBD100E013B9BDE81040E8
:103DD000D2E6034B93F8300080F0010010BD00BF25
:103DE000680E00202C27002007B5002101AB03221C
:103DF0007720FFF7B7FF9DF805309DF804001B0200
:103E000043EA00439DF80600184303B05DF804FB45
:103E100008B5FFF7E9FF014BD86108BD680E002027
:103E200008B5FFF7E1FF014B986108BD680E00205F
:103E300007B5F7216B4606227620FFF793FF9DF822
:103E400000309DF801101B0343EA01139DF8021096
:103E5000094A43EA111353629DF803309DF8041098
:103E60001B0343EA01139DF8051043EA1113136283
:103E700003B05DF804FB00BF680E002013B5104CC2
:103E800094F831301BB9A38E0133A38616E00322C8
:103E900001AB7720F621FFF765FF9DF805309DF80F
:103EA00004201B0243EA02439DF806201343054AFF
:103EB000B2F92020C2F10802D340E36202B010BD83
:103EC000680E00204412002013B50B4C94F83130DA
:103ED0001BB9A38E0133A3860CE0022201AB77202D
:103EE000F621FFF73FFF9DF804209DF8053043EAD7
:103EF0000223238502B010BD680E002013B50122F5
:103F00000DF1070304463A216820FFF72BFF9DF8C7
:103F1000073003B10123237002B010BD13B5062290
:103F20000446432168206B46FFF71CFFA0B19DF8B3
:103F300000209DF8013043EA022323809DF80220EF
:103F40009DF8033043EA022363809DF804209DF826
:103F5000053043EA0223A38002B010BD13B5062248
:103F600004463B2168206B46FFF7FCFEA0B19DF89C
:103F700000209DF8013043EA022323809DF80220AF
:103F80009DF8033043EA022363809DF804209DF8E6
:103F9000053043EA0223A38002B010BD13B501220D
:103FA0000DF1070304461A216820FFF7DBFE9DF898
:103FB000073003B10123237002B010BD13B50222F4
:103FC000044601AB1B216820FFF7CCFE9DF80420BE
:103FD0009DF8053043EA022303F54E534FF48C72EB
:103FE000103393FBF2F32333238002B010BD13B5DB
:103FF00004466B461D2106226820FFF7B3FE9DF89C
:1040000000209DF8013043EA022323809DF802201E
:104010009DF8033043EA022363809DF804209DF855
:10402000053043EA0223A38002B010BD13B5062277
:1040300004466B4601211C20FFF794FE9DF80130D9
:104040009DF80020042143EA022242F38D0292FBF4
:10405000F1F29DF8023022809DF8032042EA03220B
:1040600042F38D0292FBF1F29DF8043062809DF8DC
:10407000052042EA032343F38D0393FBF1F3A3806E
:1040800002B010BD13B504466B460221062218206B
:10409000FFF768FE9DF800309DF801209B0803EBB8
:1040A000022323809DF802309DF803209B0803EB38
:1040B000022363809DF804309DF805209B0803EBE4
:1040C0000223A38002B010BD2F4B2DE9F3411B78D2
:1040D0000546002B39D0002426462746A046082254
:1040E0006B4653203221FFF73DFE9DF801209DF8DD
:1040F0000030013403EB02231BB29DF803209844E7
:104100009DF80230E4B203EB02231BB21F449DF87A
:1041100005209DF80430202C03EB02231BB21E4423
:104120009DF8073003F07F0301D0002BD7D198FB17
:10413000F4F897FBF4F796FBF4F6144BA5F800801F
:104140006F80AE8083F836401AE006226B4653201B
:104150003221FFF707FE9DF801209DF8003003EBA8
:1041600002232B809DF803209DF8023003EB0223ED
:104170006B809DF805209DF8043003EB0223AB8093
:1041800002B0BDE8F08100BF2C120020680E0020B4
:1041900013B5204B400002ACC0B2587104F8012D99
:1041A000D970012200211A7359701A711A751A4AAE
:1041B0001C6110689C6083F8301040B382889205BF
:1041C00015D40288D4050DD447F2305201888905F0
:1041D00002D5013AFAD112E08AB1028892B242F4D1
:1041E00080720280828892B242F44072828047F2EA
:1041F0003052197D11B1013AFBD100E012B9FFF73D
:10420000BBFC04E0034B93F8300080F0010002B0E7
:1042100010BD00BF680E00202C2700207720482109
:104220000122B5E7772058210122B1E77620F42159
:104230003122ADE7064B002193F82020054B920177
:10424000343283F831107720F42102F0FC029FE72A
:1042500044120020680E0020034B002283F8312016
:104260007720F4212E2293E7680E002008B5FFF78F
:104270000BFD6B2180226820FFF78AFF642009F084
:10428000A0FE6B2103226820FFF782FF0F2009F0B8
:1042900098FE124B19211A786820FFF779FF0F203A
:1042A00009F08FFE0E4B1A211A786820FFF770FF75
:1042B0001B2118226820FFF76BFF1C2110226820A9
:1042C000FFF766FF372102226820FFF761FFBDE894
:1042D00008406820382101225AE700BFAC120020B4
:1042E0002000002008B5192009F06BFE6820152178
:1042F0000022FFF74DFF10B9032009F0DDFE0C4B43
:1043000016211A78682042F01802FFF741FF1721A2
:1043100000226820FFF73CFF3D2101226820FFF7C3
:1043200037FFBDE8084068203E21012230E700BF8A
:104330002100002013B500222A211C20FFF728FFAE
:104340000E2102221C20FFF723FF0F2103221C2035
:10435000FFF71EFF2B2112221C20FFF719FF164A20
:1043600002249369154843F0040393612023ADF8B8
:10437000043004230DEB03018DF806308DF807405F
:104380000BF00DFB22462C211C20FFF701FF2D21F5
:1043900001221C20FFF7FCFE2E2100221C20FFF72B
:1043A000F7FE2A2105221C20FFF7F2FE044B4FF4F2
:1043B00080721A8002B010BD001002400008014057
:1043C0001C00002008B50F2108221820FFF7E0FE8E
:1043D0000E2218201021FFF7DBFE024B4FF4805213
:1043E0001A8008BD1C00002008B5134B53201B7811
:1043F0002D2108227BB1FFF7CBFE31210A22532069
:10440000FFF7C6FE2C210C225320FFF7C1FE5320DC
:104410003821902209E0FFF7BBFE31210A22532008
:10442000FFF7B6FE53202C210A22FFF7B1FE40F21F
:104430000912024B1A8008BD2C1200201C0000201B
:10444000FEF79EBFFFF74CBBFEF79ABFFFF748BBD6
:10445000F8B50F461646074C4FF48055656140F09D
:1044600080000EF059FA3846002132460EF01EFA4E
:104470002561F8BD000C014013B5012204460DF181
:1044800007013820FFF7E4FF9DF8073003B101234F
:10449000237002B010BD13B50446694643200622BE
:1044A000FFF7D6FF9DF800209DF8013043EA022374
:1044B00023809DF802209DF8033043EA02236380A5
:1044C0009DF804209DF8053043EA0223A38002B042
:1044D00010BD13B5044669463B200622FFF7B8FF1E
:1044E0009DF800209DF8013043EA022323809DF8C7
:1044F00002209DF8033043EA022363809DF80420E4
:104500009DF8053043EA0223A38002B010BD07B531
:10451000232009F056FD6820752101220DF10703C3
:10452000FFF720FC28B19DF80700A0F1680358426E
:10453000584103B05DF804FB2DE9F04FA04EA14DAA
:104540003368A14C03F59C43203323602B889F4A9A
:1045500001332B8042F20103116889B00B4092466F
:104560001BB19B4A13780133137004F079FEDAF81B
:104570000030DF0405D5974B1B68D80701D40EF037
:10458000F7FD954B37681A68907AB8B19349137B59
:10459000013831F810001BB1C0F53B60083080B223
:1045A00000B2A0F57A70B0F57A7FA8BF4FF47A70A8
:1045B00020EAE0700FF02AF9894930E0DAF800309B
:1045C000190435D56368804EFB1A002B30DB07F5E4
:1045D0009C4320337360834BD27A5979824B33F8F2
:1045E0001130317A9BB293FBF2F3013101F00F02EB
:1045F00032723244537203467C4A825C0130134467
:1046000010289BB2F8D11BB293FBF0F000B26428E3
:10461000A8BF642020EAE0700FF0F8F874490FF0AA
:10462000FDF974490FF046F90FF030FB724B18801A
:10463000DAF80030694E13F4807F00F081806F4B10
:104640009F4204D92B7913B95E4B01221A71B5F937
:1046500000E06B4ABEF1140F1778CCBF4FF0000E8C
:104660004FF0010E574BC7F38007BEF1000F06D085
:104670004FF0000883F8068083F8058001E04FF0D2
:104680000308E369A8790193D4F820C0B5F9009034
:1046900069796B883288032848D8DFE800F0020E79
:1046A0001B36BEF1000F02D0328000222BE0002F1B
:1046B00040F086863280AF713AE09CF8000000EB53
:1046C0008000814502DC328001221CE001206FB3B2
:1046D00000F0E6BE47B1019A4FF00208D28972801D
:1046E000B280BCF80200F0809CF800B09CF8010099
:1046F000584400EB8000814500F36586002F00F0F0
:10470000628632800222AA7112E032800322AA71EC
:1047100069716B8077B13A4A137843F002031370E2
:10472000284B00225A710EF023FD03E03280A8715D
:1047300069716B80B8F1000F02D0404609F07EFC31
:10474000304FB7F852010EF04EFB0197834668B91F
:104750000EF022FF2C4B0022C3F800B0C3F804B0C7
:10476000C3F808B0294B1A605A609A60244F3B780E
:104770005B0763D5DAF80030D8065FD5244B1B7889
:10478000D9065BD4234B1B7893B1019B93F8D431AA
:10479000BBF1000F42D173B11F4B1A68636A9B1AB9
:1047A000002B08DA0EF0E4FC074B83F828B045E054
:1047B000BBF1000F3AD1102009F040FC01233BE08F
:1047C000C0330020A8330020A40E00208C29002034
:1047D000EF150020A80F0020E8150020C8290020B0
:1047E00000007A443C1500204C150020AD0E00203E
:1047F0000000C84200C07F4404100020404B4C0021
:10480000E1330020EC290020C82400203C270020B0
:10481000A810002008000020B029002033B1904AE1
:104820004FF47A71126801FB0323636294F8283015
:1048300023B109F0EBFB002384F82830019B93F8A7
:10484000D2310293019B93F8D311B3F898E1B3F8F6
:104850009AC10023184636F9132080087245C4BF58
:1048600060F07F00C0B201336245B8BF40F0400045
:10487000042BF0D194F829307A4A834205D192F87A
:104880002A30F92B04D8013300E0002382F82A30C3
:10489000754B84F829001A78DFF8E4819946DAB973
:1048A000D8F80030DA0708D5BBF1000F14D13B78F7
:1048B000DB0711D50EF0B0FA0EE03B7858070BD5A8
:1048C0006A4B1B7843B16B7933B911B10EF050FCD0
:1048D00002E0BBF1000FF9D094F82A30614A142BA2
:1048E000DFF8A0B140F08F80029B003318BF012396
:1048F000029399F8003063B392F829305F2B11D1FD
:104900003B7803F0040303F0FF0113B10EF030FC19
:1049100008E00B200491039209F090FB039A04999C
:1049200082F82A10029BA3B194F829307D2B10D174
:104930003B7803F0040303F0FF0213B10EF018FC00
:1049400007E00B20039209F079FB464B039A83F8AA
:104950002A203B7803F0040303F0FF01002B52D11F
:1049600094F829303F4A572B16D1414B4FF47A72B5
:104970001A80DAF80030190601D508F003FF3D4B24
:104980001B685A0742BF3C4A0A21118013F00803F2
:1049900039D13A4A138036E0DAF80000400717D5DB
:1049A0005A2B15D192F82B302BB1012382F82B1002
:1049B00082F82C3027E092F82D3083F0010382F842
:1049C0002D300BB10C2000E00D2009F037FB1AE070
:1049D0005D2B00F0FB845B2B00F0FA845E2B02D190
:1049E000032000F0F6BC562B01D106F00DFA99F821
:1049F0000030002B00F0028594F829306F2B40F036
:104A0000F8840EF009FADAF800305A074BD594F81A
:104A10002D30144A93B13B785B070FD5019BB6F953
:104A20000610B3F89831994208DDD8F8003013F039
:104A3000010302BF3221118682F82D30D8F80030F0
:104A4000D80321D594F83220064B22B993F82B20B5
:104A50000AB932221A86012384F8323023E000BFDB
:104A6000B0290020A40E002008000020EE15002030
:104A7000DA330020A4100020D8330020801000205A
:104A8000A80F0020E00F002094F82B30AC4A53B15F
:104A90003B7803F0040303F0FF0123B9012382F8FC
:104AA0002B1082F82C30DBF800700023C8F800309F
:104AB00007F17B0607F1CB093278737816F8010C01
:104AC0009A420DD2314603F0FBFD48B116F8022C94
:104AD000012303FA02F2D8F800301343C8F800307B
:104AE00004364E45E8D1974B1B784BB1964EDFF814
:104AF00080823368954F13F0020F40F025831DE349
:104B000007F1CA0607F589773278737816F8010C31
:104B10009A4222D2314603F0D3FDF0B196F804E078
:104B20000C21B37801FB0E41894A013B03EB43039F
:104B300013448A6B96F803809A4281480DD08B63A8
:104B4000002390F86420CB63012303FA0EF322EADA
:104B5000030381F8348080F864300636BE42D3D136
:104B60007C4BDFF810921F687B4B4FF0000B1B68EB
:104B700002937A4B1B780393D9F80030002B00F096
:104B8000D48293F80080B8F1000F00F0CE82D9F8FB
:104B9000042002998A1A002A0CDB01F5FA72C9F87E
:104BA000042094F86410012202FA0BF221EA0202B6
:104BB00084F86420039A002A00F0B78219F8042CC4
:104BC00059780432D2B2002940F07082644931F938
:104BD0001210644AB2F8962102F1C800814201DD48
:104BE0009E7814E0C83A914202DA99784E420EE07B
:104BF00094F86420012303FA0BF322EA030384F8F8
:104C00006430029B03F5FA73C9F804308DE294F81E
:104C1000643043FA0BF3D90700F18782002ECCBF32
:104C20000220012009F030FA08F1FF32444B132A28
:104C300000F27382DFE812F0140021002E003D0024
:104C400056005D00DD004101A501D2010A0271029A
:104C50003D004C005D00DD004101AF001301770114
:104C6000397838460E44FA2EA8BFFA2626EAE676A8
:104C70003E7003F00BFD012019E0797838460E44B0
:104C8000642EA8BF642626EAE6767E7003F0FEFC5A
:104C900002200CE0F97838460E44642EA8BF642642
:104CA00026EAE676FE70996E03F0A8FC03203146F2
:104CB000C0E179790D2031446429A8BF642121EA3B
:104CC000E171797109F042F9B8F10D0F00F0258218
:104CD00039790E2031446429A8BF642121EAE171A9
:104CE0003971A7E1B9790520314481F30801B9711F
:104CF000A0E1DB6E1A78022A3ED1304604930EF012
:104D000085FD19490EF08AFE049B596A05930EF041
:104D1000C9FC002104900EF06BFF059B48B9049A72
:104D2000124910460EF082FF049A059B10B10F4AFB
:104D300000E000225A620F20114609F0F3F826E045
:104D4000A40E0020E5330020A80F002068110020E9
:104D5000289D010808100020B0290020EE15002031
:104D6000C8290020EC290020000020410000C84292
:104D7000A4100020DC0E002099780F203144C829AF
:104D8000A8BFC82121EAE171997009F0DFF8B8F1F4
:104D90000F0F00F0C281A94BD3F86C8098F8003057
:104DA000022B1AD130460EF031FDA5490EF036FE29
:104DB000D8F820100EF076FC002106460EF018FF01
:104DC00030B930469F490EF031FF10B19D4E00E0E2
:104DD0000026C8F82060122058E198F8011012202F
:104DE0003144C829A8BFC82121EAE17188F801101F
:104DF00020E1DB6E1A78022A22D1304604930EF0AD
:104E000005FD90490EF00AFE049B196B05930EF008
:104E100049FC002104900EF0EBFE059B48B9049A72
:104E2000884910460EF002FF049A059B10B1854A8E
:104E300000E000221A631020114609F073F80AE01E
:104E4000197B10203144C829A8BFC82121EAE1718B
:104E5000197309F07BF8B8F1100F00F05E81774B01
:104E6000D3F86C8098F80030022B1AD130460EF03F
:104E7000CDFC74490EF0D2FDD8F82C100EF012FCC7
:104E8000002106460EF0B4FE30B930466D490EF0F2
:104E9000CDFE10B16B4E00E00026C8F82C60132048
:104EA000F4E098F80B1013203144C829A8BFC8219A
:104EB00021EAE17188F80B10BCE0DB6E1A78022A57
:104EC00022D1304604930EF0A1FC5F490EF0A6FDFE
:104ED000049BD96B05930EF0E5FB002104900EF0C6
:104EE00087FE059B48B9049A564910460EF09EFE6F
:104EF000049A059B10B1534A00E00022DA631120A6
:104F0000114609F00FF80AE0997D11203144C829B3
:104F1000A8BFC82121EAE171997509F017F8B8F125
:104F2000110F00F0FA80454BD3F86C8098F80030F0
:104F3000022B1AD130460EF069FC43490EF06EFD8B
:104F4000D8F838100EF0AEFB002106460EF050FEE9
:104F500030B930463B490EF069FE10B1394E00E0E1
:104F60000026C8F83860142090E098F81510142036
:104F70003144C829A8BFC82121EAE17188F8151079
:104F800058E0D3F86C8098F80030022B1AD13046E4
:104F90000EF03CFC2A490EF041FDD8F828100EF026
:104FA00081FB002106460EF023FE30B9304625492C
:104FB0000EF03CFE10B1234E00E00026C8F8286039
:104FC000092063E098F8031009203144C829A8BFDC
:104FD000C82121EAE17188F803102BE0D3F86C8036
:104FE00098F80030022B1AD130460EF00FFC15490C
:104FF0000EF014FDD8F834100EF054FB00210646D4
:105000000EF0F6FD30B930460E490EF00FFE10B12D
:105010000C4E00E00026C8F834600A2036E098F80C
:105020000D100A203144C829A8BFC82121EAE17126
:1050300088F80D1008F08AFF6FE000BFA40E002072
:10504000000020410000C84200007A44D3F86C8080
:1050500098F80030022B1DD130460EF0D7FBB14935
:105060000EF0DCFCD8F840100EF01CFB00210646C8
:105070000EF0BEFD30B93046AB490EF0D7FD10B191
:10508000A94E00E00026C8F840600B20314608F029
:1050900049FF42E098F817100B203144C829A8BFF7
:1050A000C82121EAE17188F81710C3E7012934D13A
:1050B00098789E4B33F91230B3F5617F05DB40F6EB
:1050C00033029342A8BF134601E04FF46173B8F175
:1050D0000C0F22D14FF4966292FBF0F0A3F56173AE
:1050E00093FBF0F3924ADEB21378B34215D0042E4C
:1050F00034BF334602231370019A08FB03238D4A01
:1051000003F2AA7313600DF025F84046314608F00B
:105110001DFF701CC0B208F0B7FF94F86420012393
:1051200003FA0BF3134384F864300BF1010BBBF16A
:10513000040F09F10C097FF41FADD7E4DAF8003051
:10514000DA050FD56B796BB1D8F800309B0709D51C
:105150003B8813F001050AD10EF01EFA012005F07C
:10516000ADFB04E0012005F098FB012300E00023E3
:10517000326855070CD55BB1012005F08EFB3B88EA
:10518000980708D40EF008FA022005F097FB02E019
:10519000022005F082FB3B88674A13F0030F4FF0B3
:1051A000100114BF51611161D8F8002012F00A0FEC
:1051B00023D03268D10609D55A070AD4042005F055
:1051C0007DFB5E4B1B88A4F8703002E0042005F0E4
:1051D00064FB33689B0606D53B885D0606D44020F9
:1051E00005F06CFB02E0402005F057FB33685806E1
:1051F00042BF524B1B88A4F87230D8F80030990691
:1052000008D433681A0540F1A9804FF4807005F086
:1052100055FBA7E04A4B1B789B074DD5494B1B78A4
:10522000042B49D9336813F400780ED03B88DD068F
:1052300036D4102005F042FB202005F02EFB42481A
:10524000011D08F009FA022326E03D8805F010054B
:10525000ADB22DB1102005F020FB012584F874803B
:105260003368580511D5A36F38495A89B1F9003010
:10527000002BB8BF5B42934207DAB1F90230002B32
:10528000B8BF5B429342C0F211813B88990608D5B2
:10529000202005F002FB002384F87430012500E093
:1052A000002594F87C30B3B90E2008F0C7FE284BD7
:1052B000012283F87C200EE03B8803F03003002BB2
:1052C0009FD0102005F0E9FA202005F0E6FA00232F
:1052D00084F8743001E0002D93D0002005461D4B6A
:1052E000002423F815401C4B1A1D03F10A0122F873
:1052F00015400022425001444C608A6023F815405A
:1053000003F132015A334250C250014403444C600D
:105310008A605C609A601430002D7FF472AF0125C2
:10532000DDE700BF00007A440000C842C829002021
:10533000B027002008100020000C01408010002041
:10534000A8100020AE1000201010002088100020AF
:10535000A40E0020DC330020220F00204FF48070C8
:1053600005F09BFA5D4B5A791C46082A01D00E2A9B
:1053700002D1402005F091FADAF800305A0540F1E8
:10538000AA8094F8103223B9554B1B7813F0040F00
:1053900002E0336813F4002F0BD0524B00221A7036
:1053A0003C2002F049FB002800F095800BF0FAFE4B
:1053B000F6E704F09DF909B0BDE8F04F01F06BBDD0
:1053C0000120FFF768B90320FFF765B9012000E06D
:1053D00002205FFA80F9019A09F1FF3382F8A837B9
:1053E00005F0AEFA05F04EFB484608F04DFEFFF71B
:1053F0000ABB029A12B17E2B3FF403AB94F829301A
:10540000972B05D1384B4FF4C872DA85FFF7FBBAFA
:10541000A72B06D1354A137843F004031370FFF726
:10542000F2BA0022BB2B079201D1022303E0B72B73
:1054300004D14FF6FE73ADF81E3009E0BE2B01D14A
:10544000022303E0BD2B1AD14FF6FE73ADF81C30DA
:10545000DBF80020BDF81C10B2F858300B44A2F85D
:105460005830BDF81E10B2F85A300B44A2F85A302A
:1054700005F0CAFC002384F82A30FFF7C4BA792B60
:1054800004D11B4AD37823F0010306E07A2B7FF482
:10549000BAAA174AD37843F00103D370FFF7B3BA1F
:1054A000013301469BB20220FFF7F5B83B889B060B
:1054B0003FF5F7AE202005F001FA0E4B0E481A68B2
:1054C0005B68011D4360026008F0C6F8064B0125C9
:1054D00083F87450E5E609B0BDE8F08FEC290020B0
:1054E000E1330020E1120020A40E0020A8100020CB
:1054F000D0260020B0100020181000202DE9F04721
:105500004B28A0B0044600F04C8600F2B48030284E
:1055100000F0D88651D8222800F0998423D8032897
:1055200000F0608114D8012800F05081022840F07A
:10553000348704200BF0A2FE43200BF070FE4C20B9
:105540000BF06DFE46200BF06AFE4C2000F05EBEB4
:10555000042800F05181052840F01F871A200BF025
:105560008DFE00245BE1282800F0E98515D8242869
:1055700000F0D085262840F01087B54C06200BF0AF
:105580007DFEB4F85C010BF07CFEB4F85E010BF01C
:1055900078FEB4F8600100F0BABD2C2800F0E28576
:1055A0002E2800F05E862A2840F0F78601200BF0B6
:1055B00065FEA74B587900F029BE3D2800F0F48223
:1055C0001ED8362800F033860BD8322800F0188613
:1055D000342840F0E28648200BF050FE002500F011
:1055E00058BC3A2800F0B4823B2800F029843828BF
:1055F00040F0D38604200BF041FE954C00F090BDA6
:10560000452800F0B78627D8402800F002864228B7
:1056100040F0C3868E4C10200BF030FE60790BF00A
:10562000FEFDA0680BF036FE94F890010BF0F7FD3C
:10563000B4F85C010BF025FEB4F85E010BF021FE1E
:10564000B4F860010BF01DFEB4F880010BF019FEF8
:10565000B4F8820100F05BBD472800F06986C0F015
:105660005686492840F0998602200BF007FE784BB9
:10567000988900F04CBD702800F0EC8258D8692859
:1056800000F046822AD8652800F0FE8015D84D2803
:1056900000F09685642840F0808607200BF0EEFD30
:1056A000E7200BF0BCFD6A4B58790BF0B8FD0020E9
:1056B0000BF0B5FD042000F06CBE672800F0AB8154
:1056C00000F2198212200BF0D9FD624B00241B88D6
:1056D000B3F5806F8CBF082501257EE16C2800F0B2
:1056E0002A8217D86A2800F099846B2840F05586E2
:1056F00005200BF0C3FD584B18880BF0C2FD574B2B
:1057000018880BF0BEFD564B93F86A0000F00100BC
:1057100000F07CBD6E28524D00F0218200F27282B2
:1057200006200BF0ABFDA86D0BF0B4FD4D4B0DE268
:10573000782800F07D8119D8742800F0CB830BD82D
:10574000722800F02B84732840F0278608200BF085
:1057500095FD012400F05BBC762800F07F8400F208
:10576000FD832F200BF08AFD3F4C61E3A42800F05D
:105770009A8414D87B2800F00183A02840F00D867D
:105780000C200BF07BFD394B18680BF083FD384B78
:1057900018680BF07FFD374B186800F0FABDF12850
:1057A00000F08281FE2800F0A584F02840F0F58505
:1057B0002B4C04200BF062FDE36BB3F85A000BF0A6
:1057C00060FDE36BB3F8580000F0A1BC03200BF0C0
:1057D00055FD00200BF023FD20460BF020FD0A2094
:1057E00000F014BD0BF04AFD01200BF018FD09205C
:1057F0000BF015FD00F055BC06200BF03FFD4120DD
:105800000BF00DFD46200BF00AFD4E200BF007FDBE
:1058100041200BF004FD184B187800F078BC174BB2
:10582000185D01340BF0FBFC0B2CF8D10024144B59
:10583000185D01340BF0F3FC082CF8D10024114B57
:10584000185D01340BF0EBFC072CF8D100F0A3BD80
:10585000EC2900201C00002022110020241100202F
:10586000A40F002078100020639D0108E8F7FF1FB7
:10587000ECF7FF1FF0F7FF1FE3330020C4BB010864
:10588000D0BB0108A5BB0108CD4C0B200BF0F6FCEA
:1058900020880BF0F6FC608880B20BF0F2FCC94B5C
:1058A0001B68C3F3C000C3F38002800040EA4200DB
:1058B000C3F340021043C3F3401240EAC20003F0B6
:1058C000100318430BF0DDFCBF4B1A88636812F01D
:1058D000010F14BF4FF0020C4FF0000C12F0020F3A
:1058E00002F0080814BF4FF0040E4FF0000E03F44E
:1058F000475912F0040F14BF1027002749EA08097E
:1059000012F0400F03F4804814BF2026002649EA15
:10591000080912F0100F03F4004814BF4FF400758B
:10592000002549EA080912F0200F03F4803814BF5B
:105930004FF48060002049EA080912F4807F03F4E4
:10594000003814BF4FF40061002149EA080912F43D
:10595000007F03F480289D4A49EA080903F40028DF
:1059600049EA0809127803F4801849EA080903F0A3
:10597000007349EA0303C2F3800243EA020343EAE5
:105980000C0343EA0E0E4EEA070746EA070645EA0D
:10599000060540EA050041EA00014FF00000034619
:1059A00014BF4FF400184FF0000841EA0808217AAC
:1059B0008B420BD2864A9C5C012202FA04F414EA60
:1059C000080F1CBF9A4010430133F1E70BF062FC53
:1059D000804B93F8A80700F019BC7F4B33F91400F3
:1059E000013490FBF5F080B20BF04BFC032CF4D1AA
:1059F000734CA08C0BF045FCE08C0BF042FC208D2E
:105A0000764C0BF03EFC20880BF03BFC60880BF0E2
:105A100038FCA0887BE310200BF030FC0024704B96
:105A2000185D01340BF0FBFB102CF8D100F0B3BC77
:105A300070200BF023FC00260E247443604D0136C9
:105A4000EB6B2344B3F819010BF01BFCEB6B234405
:105A5000B3F81B010BF015FCEB6B2344B3F81D01ED
:105A60000BF00FFCEB6B234493F81F010BF0D7FBFB
:105A7000EB6B234493F820010BF0D1FBEB6B234439
:105A800093F821010BF0CBFBEB6B234493F822013D
:105A90000BF0C5FBEB6B1C44D4F823010BF0FAFBB5
:105AA000082EC9D100F077BC70200BF0E7FB494C01
:105AB00004F1700594F8D4000BF0B1FB94F8D50014
:105AC0000BF0ADFB94F8D6000BF0A9FB94F8D700CF
:105AD0000BF0A5FB94F8D8000BF0A1FB94F8D900CB
:105AE0000BF09DFB073494F8D3000BF098FBAC420D
:105AF000E0D100F050BC10200BF0C0FB0024394B6B
:105B0000185D01340BF08BFB102CF8D100F043BC76
:105B1000354D00242878400000F0FE000BF0AEFB6D
:105B20002B789C4280F03784304B33F814000BF014
:105B3000A8FB0134F4E72E4C06200BF09FFB2088D5
:105B40000BF09FFB60880BF09CFB2A4B1888DEE271
:105B500004200BF093FB1A4BD86D00F01ABC072001
:105B60000BF08CFB244B1888FF28A8BFFF20C0B285
:105B70000BF055FB214B186880F3100080B20BF03E
:105B800080FBB5F860000BF07CFB124B93F885218D
:105B90001B4B186822B10A23584380F3100001E020
:105BA00000F30F0080B2B2E20A4C02200BF066FB59
:105BB00094F8D4010BF033FB94F8D30126E300BF33
:105BC000A40F0020A410002068110020E133002061
:105BD000AD0F0020EC29002072100020C812002018
:105BE000CE0F0020E40F0020EC150020C829002073
:105BF000842900208010002094100020A010002094
:105C00009C1000200B200BF039FB6B6E00261878DF
:105C10000BF005FB6B6E58780BF001FB6B6EBE4C06
:105C20003344187901360BF0FAFA032EF6D1636E7D
:105C3000D8790BF0F4FA636E98780BF0F0FA636E93
:105C4000D8780BF0ECFA636E58890BF01AFB636E90
:105C5000187ADBE2B04C1E200BF010FBE36B002542
:105C60001B78022B77D1E36B05F1080253F8220071
:105C7000AA490DF01FFE11F029FDFA28A8BFFA204D
:105C800020EAE070C0B20BF0CAFAE36BA44903EB60
:105C90008503D86A0DF00EFE11F018FDFA28A8BF92
:105CA000FA2020EAE070C0B20BF0B9FAE36B05F11C
:105CB0000E0253F822009B490DF0FCFD11F006FD89
:105CC0006428A8BF642020EAE070C0B201350BF060
:105CD000A6FA032DC7D1072DE36B2AD1586C8F4943
:105CE0000DF0E8FD11F0F2FCFA28A8BFFA2020EA36
:105CF000E070C0B20BF093FAE36B8849986C0DF03A
:105D0000D9FD11F0E3FCFA28A8BFFA2020EAE070E0
:105D1000C0B20BF084FAE36B93F84C000DF072FD07
:105D200011F0D4FCFA28A8BFFA2020EAE070C0B233
:105D30000BE02B4458780BF072FAE36B2B44D87AC3
:105D40000BF06DFAE36B2B44587D01350BF067FACD
:105D50000A2DC0D11FE3E36B2B4458780BF05FFA98
:105D6000E36B2B44D87A0BF05AFAE36B2B44587D43
:105D700001350BF054FA0A2DEDD10CE33C200BF069
:105D80007DFA0024644D04F10802EB6B654953F879
:105D900022000DF08FFD11F099FC80B20BF071FA2A
:105DA000EB6B604903EB8403D86A0DF083FD11F0BF
:105DB0008DFC80B20BF065FAEB6B04F10E0253F828
:105DC000220058490DF076FD11F080FC013480B2BC
:105DD0000BF057FA032CD5D1072CEB6B16D1586C6E
:105DE00050490DF067FD11F071FC80B20BF049FADB
:105DF000EB6B4C49986C0DF05DFD11F067FC80B2C7
:105E00000BF03FFAEB6B93F84C000BE0234458780F
:105E10000BF037FAEB6B2344D87A0BF032FAEB6BCA
:105E20002344587D01340BF02CFA0A2CD4D1B2E271
:105E300014F8010F002800F0AE820BF0F0F9F7E73C
:105E400001200BF01BFA344BDB6B1878DEE150209D
:105E50000BF014FA0025304B0C21DC6B324B04EBB9
:105E6000850494F87920013501FB023393F838005A
:105E70000BF0D5F994F87A000BF0D1F994F87B0087
:105E80000BF0CDF994F87C000BF0C9F9142DE2D198
:105E900081E2214BDC6B062303FB054494F8CE0022
:105EA0000BF0BDF994F8C9000BF0B9F994F8CA00E9
:105EB0000BF0B5F994F8CB000BF0B1F994F8CC00E5
:105EC0000BF0ADF9013594F8CD000BF0A8F90C2DCD
:105ED000DFD160E24FF00008012600270E4B1A7A4E
:105EE000974232DA0933FA5C00240C2363430E4DE7
:105EF00005F13001595C914207D12B44586B11F0E8
:105F00001CFA82462EB9B14610E001341B2CECD1AC
:105F100019E0804417E000BFA40F002000002041DA
:105F20000000C84200007A44649D0108D1450ADAA5
:105F30000C2303FB04535B6B13F809000BF06FF9A0
:105F400009F10109F2E70137C8E7002E00F02382CA
:105F50005FFA88F00BF092F90026BEE7CC4D0024E2
:105F6000287A0BF08BF92B7A9C4280F01482C94B73
:105F70000021E65C0C2202FB01F3C74800F1300768
:105F8000DA5DB24205D1034493F838000BF047F9CB
:105F900002E001311B29EDD10134E4E7BF4C1620AA
:105FA0000BF06CF9B4F896010BF06BF9B4F84401FE
:105FB0000BF067F9B4F846010BF063F9B4F8480147
:105FC0000BF05FF9B4F8D0010BF05BF994F8E10144
:105FD0000BF025F900200BF022F994F8E2010BF008
:105FE0001EF994F885010BF01AF994F892010BF060
:105FF00016F900200BF013F9A54B0A20DB6BB3F95F
:10600000563093FBF0F080B20BF03BF988E0E0B241
:1060100001340BF004F9092CF9D1BCE110200BF08C
:106020002DF99F4B9F4C187800F002000BF0F7F809
:106030009D4B18780BF0F3F820680BF02BF9606893
:106040000BF028F9994B18880BF01BF9984B18881E
:106050000BF017F98E4BB3F8680058E00BF0C2F85C
:10606000074612200BF00AF9894C17B9E66E256F26
:1060700005E0102F19BF00252E46666FA56F384624
:106080000BF0CDF830460BF005F928460BF002F97D
:10609000E06F0BF0FFF800200BF0F3F800200BF09E
:1060A000F0F80020B2E07A4D002495F880002E46EA
:1060B00080000130C0B20BF0E1F895F880000BF0E1
:1060C000AEF896F880309C4280F06581794D285D6D
:1060D0000BF0A5F805F11003185D0BF0A0F805F121
:1060E0002003185D30350BF09AF8285D0BF097F817
:1060F0000134E6E708200BF0C1F800200BF0C1F8EE
:1061000000200BF0BEF800200BF0BBF800200BF0D5
:10611000B8F840E104200BF0B1F8604B986838E122
:1061200094F87A010BF07BF894F87E010BF077F885
:1061300094F87D010BF073F894F87F0166E0574CFA
:1061400007200BF09BF8B4F880010BF09AF8B4F834
:1061500082010BF096F894F884010BF060F8B4F823
:106160008601D4E74D4C0C200BF088F894F8900190
:106170000BF055F8B4F89A010BF083F8B4F89601D7
:106180000BF07FF8B4F898010BF07BF894F89101CC
:106190000BF045F8B4F89C010BF073F8B4F89E01CD
:1061A000B5E73E4C04200BF069F894F8CE010BF0F3
:1061B00036F894F8CF010BF032F8B4F8D001A6E726
:1061C0003D4C3E4D20780426043800EB4000C0B220
:1061D0000BF054F8237802359E4280F0DC8015F8ED
:1061E000020C0BF01CF815F8010C013600EB8000D6
:1061F00000EB800000F2EE2080B20BF042F8E9E7FD
:1062000001200BF03BF8254B93F892010BF007F8B7
:10621000C1E008200BF032F80024204B234493F80F
:10622000880101340AF0FBFF082CF6D1B3E0184BCB
:106230001A4C93F8C10004F12805C0EBC000C0B2AD
:106240000BF01CF894F8E80100231D4AD25C904240
:1062500000F0A5800C333C2BF7D10834AC42F1D1CF
:1062600099E040200BF00AF80C4C04F14005B4F81A
:10627000A0020BF006F894F8A2020AF0D0FF043452
:1062800094F89F020AF0CBFFAC42F0D183E000BF4C
:10629000A40F0020AD0F0020649D0108EC29002010
:1062A000A8100020B0100020AE100020AC1000207C
:1062B000AA10002025100020EC1500208C2B0020B7
:1062C000E8120020E0200AF0D9FF424C04F18005DA
:1062D000B4F82202043400F03F000AF0D2FFB4F810
:1062E0001E02C0F386100AF0CCFF94F81C020009CD
:1062F0000AF095FF94F81C0200F00F000AF08FFFDF
:1063000094F81D020AF08BFFAC42E1D143E0324C1D
:106310000D200AF0B3FF09F07BFC0AF080FF208813
:106320000AF0B8FFE0680AF0B5FF07F0E5FA30E0E0
:106330000AF06CFF054684200AF0A0FF28460AF008
:10634000A9FF254BDC6805F18003A3428CBF641BC9
:10635000802407F08BFB28462246694609F08CFC16
:1063600005460024AC4216DA1DF804000AF057FF77
:106370000134F7E713200AF081FF0024174B185D62
:1063800001340AF04CFF0B2CF8D100200AF082FFF8
:1063900000200AF07FFF012018E0002016E00AF03C
:1063A0003EFFB4F8EA010AF06CFF94F8EC010AF041
:1063B00036FF94F8ED010AF032FF94F8EF010AF08D
:1063C0002EFF94F8EE010AF02AFF46E720B0BDE860
:1063D000F08700BFEC2900200C000020C4BB01089E
:1063E0002DE9F347C54C06462378C54F002B00F036
:1063F000D9813A686368D31A7C2B40F2D381237A1F
:106400006260013323724FF0000808F12400BB4D95
:10641000C0B203F021F905F10A0333F918000DF0B9
:10642000F5F9B84B814618880DF0F0F90146484659
:106430000DF0F4FAB4490DF03DFA0DF001FC08F14D
:10644000010800B203F0F6F8B8F1030FDDD13020F7
:1064500003F002F9B5F9100003F0ECF803F0F4F8DA
:106460002B7A9A072CD141F288336A689A4218D95C
:10647000102003F0F1F868694FF0640890FBF8F021
:1064800000B203F0D7F8212003F0E6F8686990FB2A
:10649000F8F308FB13000028B8BF404200B203F035
:1064A000C9F8142003F0D8F8B4F9180003F0C2F8C2
:1064B0001C2003F0D1F8002003F0BCF803F0C4F86E
:1064C000237ADFF838825B0740F04981022003F02D
:1064D000C3F8D8F81C006423323090FBF3F000B20C
:1064E00003F0A8F8B8F926504FF0050A95FBFAF525
:1064F000032003F0B1F8854BADB21B78DFF8209292
:1065000013F0040F0BD030460CF06DFC28B9D9F80D
:10651000003013F0100F18BF002528B205E0D8F89E
:1065200028309889B0FBFAF000B203F083F8D9F86C
:1065300000309E0765D5DFF8EC91A28D99F8003008
:106540004FF0640808FB02325B00B2FBF3F3E68D08
:1065500006203601B6B246EA0326B6B2C3F30323D9
:106560001E4303F079F830B203F064F8E38D99F834
:10657000001001339BB293FBF1F201FB1233E38570
:10658000236B5E4D9B7B012B05D1392003F064F812
:10659000B5F92C0019E0AD8D6E235D43152695FBF2
:1065A000F6F53A20AEB203F057F8B6FBF8F528B28C
:1065B00008FB156503F03EF83B2003F04DF8A8B248
:1065C000451D0A2095FBF0F000B203F033F82820B7
:1065D00003F042F8636B0A2093FBF0F000B203F083
:1065E00029F8042003F038F8A36A9B8913B102F05C
:1065F000E1FD03E0414B986B80F3100000B203F023
:1066000019F8E36B3D4E9D0640F19F8096F84030AF
:1066100098071DD5112003F01FF8B6F842004FF47B
:10662000F36568433A4B90FBF3F000B203F002F8D5
:10663000192003F011F8B6F842004543642095FB99
:10664000F0F595FBF0F300FB135000B202F0F2FFFF
:1066500094F84030B4F8445013F0020F08BF0025FE
:10666000012002F0F9FF28B202F0E4FF092002F055
:10667000F3FF002002F0DEFF264B94F846501A8804
:10668000B2F5967F0AD91D4B1B7A03F00F03072B37
:1066900004D842F20F75954228BF1546052002F036
:1066A000DBFF236B5B7B0BB928B216E0A5F1200062
:1066B0000DF0ACF818490DF0B1F9002105460DF0C8
:1066C00097FA10B94FF07C5101E04FF03F41284656
:1066D0000CF0E8FF0DF0B4FA00B202F0ABFF94F852
:1066E0004020064B910703D493F84720012A1BD181
:1066F000012384F8473009482DE000BF68100020CE
:10670000B02900201C00002000007A44E133002062
:10671000A0860100520000206666E63FB01000200F
:106720008C290020500000201D6BAF4968680DF0D7
:10673000C1F80DF085FAAC490090A8680DF0BAF8E0
:106740000DF07EFA0190684605E0A84A92E8030041
:106750008DE80300684602F08FFF02F075FF237A90
:10676000282B1FD1A24B00221A723B684FF47A707B
:10677000B3FBF0F83C26172002F06EFFB8FBF6F5ED
:10678000B5FBF6F006FB1050000200B202F052FF1B
:10679000182002F061FF06FB158000B202F04AFFEC
:1067A00002F052FF94F85030914D002B00F04081E0
:1067B00007F0E0FB6B6D8F4AC31A9342064640F226
:1067C000C280002385F85A3085F85C30AB8DDAB290
:1067D0001B0A85F8762085F8773085F86C2085F8D7
:1067E0006D30D5F884203B689A1AD5F88830D97B6B
:1067F0004FF47A734B439A420ED37F4B1B68C5F814
:10680000843095F88C30013B012B9FBF102385F815
:106810005A30022385F85C30626B0A20A36B92FB2E
:10682000F0F293FBF0F384F87420121284F87520D0
:1068300084F8783094F840201B1284F8793094F86A
:10684000463092076A4984F8A73003D42D2381F893
:10685000A83077E0D4F848906848DFF8ACC199FBDD
:10686000F0FA0CFB0A924FF0060E042B0EFB02F21C
:106870008CBF3323322381F8A830614BE76C92FB45
:10688000F3F197FBF0F003FB1122642592FBF5F284
:106890000CFB007C0EFB0CFE84F89920121284F88D
:1068A0009A209EFBF3F203FB12E393FBF5F30AEB52
:1068B0008A0A4FFA81F80AEB8A0A08EB8A0189B240
:1068C00084F8971000EB8000090A84F8981000EB18
:1068D000800051B201EB800292B284F89C20120A2F
:1068E00084F89D2084F89E30B4F842201B1284F86E
:1068F0009F302423534393FBF5F5B4F8BA300A22B2
:1069000084F8A0301B0A84F8A130B4F844304FEA70
:10691000D979B3FBF2F303F5FA739BB284F8A23092
:106920001B0A84F8A330B4F8BC30FF0F84F89450ED
:10693000C5F3072584F8969084F89B7084F89550E9
:1069400084F8A930666594F8BE80294DB8F1000F2F
:106950000DD1D5F8C40007F003FC012807D902289F
:10696000284F00F0388202F057FE0123BB70D4F8A4
:10697000C8001F4D00285BD095F8BE703FB140F6AF
:10698000B732D5F8D030F31A93420BD850E0012338
:10699000D5F8C400022185F8BE3007F0D5FB85F894
:1069A000D47043E095F8CC305BB9D5F8C400012130
:1069B000C5F8C83085F8BE3007F0C6FB02F02CFEE3
:1069C00034E0013BDBB285F8CC3095F8D41095F873
:1069D000D520DBB94B1C013285F8D43085F8D520A1
:1069E000D5F8C40020E000BF8096184BE49E010853
:1069F000681000203F0D0300B02900208096980009
:106A000040420F001C000020806967FF034613F816
:106A1000017B01327818394685F8D400D5F8C400D6
:106A2000C5F8C83085F8D52007F09DFBC4F8D060C4
:106A300094F8D6309C4DF3B1D5F8D830DBB1D5F809
:106A4000DC30C3B1C5F8E0301B68984AC5F8E430C3
:106A5000D5F8E8301344187AFEF750FDD5F8E03049
:106A600098790AF0DCFBD5F8E8300133092B88BFB0
:106A70000023C5F8E8308E4D94F8EC202E688A4B40
:106A8000002A00F0E281D3F8F020002A00F0DD8136
:106A900093F8F430013B012B00F2D781D4F8F000D9
:106AA000814F07F05DFBE0B1D7F8F00007F055FB30
:106AB00097F8F53080467E2BD5F800900ED1022352
:106AC0001B2887F8F43009D1D7F8F00007F048FB0D
:106AD00020B90123C7F8F89087F8FC3084F8F580D6
:106AE000DCE7D7F8F8202B689B1A41F6583293421E
:106AF0001DD9032387F8F430A7E16E4A32F813005A
:106B000010B903464FF403600133B0F5C06FDBB238
:106B100075D01DD9B0F5006F7AD031D9B0F5036FBB
:106B20003ED184F8FD30E36B5F4F99063FD494F873
:106B3000FC1094F8FD30002900F04A812A68921B6D
:106B4000012ADAD984F8FD30002384F8FC307CE196
:106B5000B0F5007F42D007D8B0F5807F47D0B0F5C0
:106B6000887F00F08380E6E7B0F5806F00F0A680B4
:106B7000B0F5826F00F0EB80B0F5047FDBD123E04D
:106B8000B0F5E26F00F08280B0F5E46F00F0838032
:106B9000B0F5E06FCFD184F8FD30B4F90A107EE093
:106BA000B0F5046F6BD0B0F5026FC4D1FAE097F87E
:106BB00040309A07BBD5B7F8421024234B436421D9
:106BC000123393FBF1F1FDE084F8FD303A4B364F80
:106BD0001B689B07ABD5BB8D0A21F2E084F8FD3022
:106BE000354B314F1B681905A1D5796BEAE084F864
:106BF000FD30E36B2C4F5A0799D57969E2E084F8B0
:106C0000FD302D4B284F1B681B0590D5B96BD9E083
:106C1000E16B254A8F0684F8FD3088D592F8401044
:106C2000880784D5D90710D5D36C192283EAE3717C
:106C3000A1EBE37101EB5101B1FBF2F1002BACBF11
:106C400041F0004141F040410DE0936C192283EA8C
:106C5000E371A1EBE37101EB5101B1FBF2F1002B08
:106C6000B8BF41F080414FF400608AE084F8FD3005
:106C7000E36B0D4F5B077FF55AAF3969A2E084F8EB
:106C8000FD30B4F91830642159437AE084F8FD30BE
:106C9000B4F90C1003E0B4F90E1084F8FD302C2385
:106CA00091FBF3F16DE000BF68100020E49E010845
:106CB000B029002094C001088C29002084F8FD3000
:106CC00094F8FE30624A0133DBB2032B88BF012304
:106CD00082F8FE3042F2107394F8FE1059435D4B77
:106CE0001B78D80748BF01319A0748BF02315F07B8
:106CF000B4F8003148BF0431D80748BF0A319A07B9
:106D000048BF14311F0648BF2831D80548BF283175
:106D10005A0748BF64311F0748BFC831980548BFAC
:106D200001F5C8719A0648BF01F57A71DF0648BFC0
:106D300001F5FA61580648BF01F57A614FF48060A9
:106D400002F036FC424B002283F8FC20EFE6E16BB8
:106D5000DFF8FC8011F0200784F8FD3017D098F898
:106D6000402012F0020F14BF4FF47A71002112F08C
:106D7000010F14BF4FF4FA6300230B4494F846103C
:106D8000194402F015FC002384F8FC30CFE6324BA6
:106D90001B6819067FF5CBAE394602F009FC88F86E
:106DA000FC70C4E684F8FD30E36B294F9A067FF54A
:106DB000BEAE97F840309B077FF5B9AEB7F84430C8
:106DC0006421594302F0F4FB002387F8FC30AEE65F
:106DD00084F8FD3039E0BB7823B1C5F8C06087F88E
:106DE0000280C4E5D5F8C030F31AB3F57A6FFFF42A
:106DF000BEAD0123D5F8C400BB7007F0AEF907465D
:106E0000D5F8C40007F0A9F97F067FF4B0AD8A2851
:106E100002D08E280CD0AAE5EB6B98067FF5A7ADC3
:106E200095F8BE30002B7FF4A2AD05F18D0306E08E
:106E300095F8BE30002B7FF49AAD05F15803C5F8E4
:106E4000C8302D2385F8CC3091E502B0BDE8F0873D
:106E500068100020E13300208C29002010B5044682
:106E6000B0F900000BF0FDFCB4F902000BF0F9FCE6
:106E7000B4F90400BDE810400BF0F3BC10B50446B3
:106E800000680BF0EEFC60680BF0EBFCA068BDE85E
:106E900010400BF0E6BC2DE9F74F012001F0A8FBF4
:106EA000002480B3012C2ED84FF04C0A0AFB04F7C3
:106EB000DFF85C8008EB070B0BF14806B57815B1DD
:106EC0000134E4B2EDE790F9003090F804E01846A0
:106ED0000E4B03228DE8240001212A4653F82E3060
:106EE00001F05CFA814650B158462946524610F0EE
:106EF000E0F901231C4448F80790B370E4B2012084
:106F000001F05CFBCDE703B0BDE8F08FF89E01080F
:106F10006C11002000212A2210B5114810F0C9F987
:106F2000104B0022194610480424105C013283F8EB
:106F3000E801052083F8ED4182424FF0000483F818
:106F4000EC0183F8EF4183F8EE0103F10803EAD185
:106F50000123A1F8EA31522381F8E63110BD00BFC8
:106F6000D22B0020EC290020B4C0010870B50646E1
:106F7000441E14F8011F89B1094D284610F0CFF9BD
:106F80000028F6D005F1080398423FBF054B401B8F
:106F9000C018A31B38BF80F88831EAE770BD00BF76
:106FA000C6D80108EC2900202DE9F04FB34C8BB076
:106FB0009A469DF85430019205460C220E4604F183
:106FC00098000021009310F074F90021142204F1BC
:106FD000A40010F06EF9002384F8B830A84B1F7895
:106FE0009846A84B03F11802012F88BF1346C4F836
:106FF000BC30FDF78CFA8146834670B3A24BB5F5E1
:10700000807FC4F8A430A14BC4F8A830A04BC4F8CA
:10701000B030A04BC4F8B4309F4B01D1002216E031
:10702000BB2D01D9012212E0612D01D902220EE00F
:10703000292D01D903220AE0132D01D9042206E0EB
:10704000092D01D9052202E0002DE7D006221A7091
:10705000012384F8B83002236DE0192006F0B1FF57
:10706000682015214A46FDF793F878B38B4B622DC3
:10707000C4F8A4308A4BC4F8A8308A4BC4F8AC30AA
:10708000894BC4F8B030834BC4F8B430824B0FD076
:1070900004D80A2D13D0142D0FD00CE0BC2D05D030
:1070A000B5F5807F07D183F801900AE0012200E066
:1070B00002225A7005E00322FBE70422F9E70522C9
:1070C000F7E7012384F8B830042334E0032F40F0BD
:1070D000E0830122752004A9FDF7BAF99DF810207C
:1070E000702A40F0D683714BBB2DC4F8A430704B8E
:1070F000C4F8A8306F4BC4F8B030664BC4F8B43055
:10710000654B01D901220EE0612D01D902220AE06E
:10711000292D01D99F700AE0132D01D9042202E024
:10712000092D02D905229A7001E00622FBE701230E
:1071300084F8B8300723604A604913700B68604FC9
:1071400043F001030B6000233B709146082E33D8B7
:10715000DFE806F0373237101D22102D2D004FF0DA
:10716000000B0AAB03F818BD532059460122FCF767
:10717000F9FD58BB434B98F8001003F118020129A0
:1071800088BF1346C4F8BC30FDF7C1F970BB98F84E
:107190000030012B40F29E8000210AAB03F8181D3D
:1071A00018200122FCF7DEFD002840F0B28098F89C
:1071B0000030032B00F0BC80012E40F2D38000266B
:1071C0003E7098F80030012BD4D8C8E79DF81030F5
:1071D000E52BCFD13B4B84F8C0B0C4F898303A4B84
:1071E000C4F89C3004233B700223B4E006210A4615
:1071F00004AB6820FCF7B6FD9DF8151001F0010204
:107200009DF8131001F001014B0043EA82019DF843
:10721000112002F001030B430AD05BB2012B01D114
:10722000002302E0022B0FD1012384F8C13012E0C9
:107230000C210DEB010368200122FCF793FD9DF862
:107240000C3013F00F0303D1052006F035FF02E0E8
:10725000042BE9D1E4E71D4BC4F898301C4BC4F86B
:107260009C3094F8C130002B0CBF6F236E2384F840
:10727000A03001233B7003236DE000BF6C110020A0
:10728000E3330020189F01086D4200081D3F0008ED
:10729000FD3E000890C1793D20000020E542000835
:1072A000EF3F0008BD3F00089D3F0008013C00087B
:1072B000974400087944000854000020A4100020DE
:1072C000E2330020E9430008C9400008393D0008C6
:1072D0005D3F000800220AAB03F8182D1C200D2189
:1072E0000122FCF73FFD00283FF456AF9DF8103017
:1072F0002A2B02D01A2B7FF44FAFD24A84F8C23027
:10730000C4F89820D04A02233B70C4F89C20042380
:1073100021E09DF81030FB2B7FF449AFCB4BC4F834
:107320009830CB4BC4F89C3001233B70052312E00E
:10733000752004A90122FDF78BF89DF81030702B01
:107340007FF43AAFC34BC4F89830C34BC4F89C30B9
:1073500001233B700823C14A89F80130136843F0C8
:107360000203136098F80030012B05D10BF0FAFAF4
:10737000BB4B4FF400525A610A2006F022FE7720E0
:10738000A021012203ABFCF7EDFC30B994F8D480C6
:10739000B44EB8F1000F6FD073E21E2101227720A6
:1073A000FCF7F6FE4FF42F6006F000FE0027A7F171
:1073B00060010026C9B2022204AB77208DF810606C
:1073C0008DF81160FCF7CEFC9DF811309DF810206F
:1073D00043EA0222A34B03F1C4017A520237102F71
:1073E000E5D1B3F8D210324601F00F0701F47F4126
:1073F000A3F8D21033464FF0010E22F001002044D2
:10740000B0F8C400002818BF4FF0000ED60703D50F
:10741000C0B24340082002E083EA1023FAE71E04CA
:1074200048BF83F4C05301384FEA4303F7D1013218
:10743000102AE2D139438B4AA4F8D210BEF1000FD2
:10744000A4D1C3F303339F42A0D142F21073A2F838
:10745000FC30A2F8FE30844BC2F80031834BC2F8F6
:107460000431834BC2F80831824BC2F80C31824B95
:10747000C2F8103103234FE1794C0BF073FA4FF44B
:107480008047042303A92046ADF80C708DF80E3018
:1074900008F085FA4FF400532361784806F042FE65
:1074A0000E21022008F066FA0823049704A8012799
:1074B0008DF815308DF814808DF816704FF0030993
:1074C00001F008FD282302A88DF808308DF80990F6
:1074D0008DF80A808DF80B700BF0CAF9142006F0B5
:1074E00070FD7720D0213A4603ABFCF73BFC002827
:1074F00000F090809DF80C30A6F8F890552B86F897
:10750000EF3040F08780D1213A4603AB7720FCF77B
:1075100029FC9DF80C30772003F00F021B0986F838
:10752000F02086F8F130162204ABAA21FCF71AFCF1
:107530009DF810209DF8113043EA0223A6F8D830B8
:107540009DF812209DF8133043EA0223A6F8DA30A2
:107550009DF814209DF8153043EA0223A6F8DC308C
:107560009DF816209DF8173043EA0223A6F8DE3076
:107570009DF818209DF8193043EA0223A6F8E03060
:107580009DF81A209DF81B3043EA0223A6F8E2304A
:107590009DF81C209DF81D3043EA0223A6F8E43034
:1075A0009DF81E209DF81F3043EA0223A6F8E6301E
:1075B0009DF820209DF8213043EA0223A6F8E83008
:1075C0009DF822209DF8233043EA0223A6F8EA30F2
:1075D0009DF824209DF8253043EA0223A6F8EC30DC
:1075E00041F2707386F8D470A6F8FC3046F6781332
:1075F000A6F8FE30224BC6F80031224BC6F8043103
:10760000214BC6F80831214BC6F80C31204BC6F887
:10761000103136E11F4A136823F480431360114B85
:10762000164AD3F81411914209D0D3F81811914297
:1076300032D0D3F81C11914234D102222DE0002225
:107640002BE000BF354300082D400008C54300086B
:1076500085400008D13A0008D3440008A410002057
:10766000001001406C11002025420008213E000856
:107670001D420008113E0008D1350008993B000862
:1076800059420008C93E0008354200087D3E000806
:10769000F539000800040140012203EB82020021B9
:1076A000C2F8141193F820314FF4005262617B4C00
:1076B0008BBB142006F085FC04F221137620D02128
:1076C0000122FCF74FFB94F82131582B2BD104F504
:1076D0009273882118227620FCF744FB7620F4214F
:1076E0003122FCF755FD012384F820316C4BA4F8BE
:1076F000FC80C4F804316B4BC4F8003145F6D81354
:10770000A4F8FE30684BC4F80831684BC4F80C315B
:10771000674BC4F810310423664A9370664A1368B5
:1077200043F004031360644E5C4C336813F0020FA3
:1077300002D0D4F898309847009B63B315F0FF0F40
:10774000336809D140F2596213F0020F40F27123FD
:1077500018BF13467D2208E09A0759BF4FF47A7389
:107760001A464FF4FA634FF47A721499994205DB82
:10777000B1F57A6F0B46A8BF4FF47A63511E0B44E4
:10778000B3FBF2F3013BDBB203FB022284F840318E
:10779000C4F8442106E09DF8003084F84031149B81
:1077A000C4F84431D4F8A4309847444B019F93F86F
:1077B0000090434B03F11802B9F1010F94BF9946B1
:1077C0009146404D00232B700FB1022F55D14FF041
:1077D00000080AAB03F8188D1E200A210122DFF8E9
:1077E000BCB0C4F84891FCF7BDFA98B19DF81030D0
:1077F000482B48D1344B0222CBF84C31334BCBF8D9
:10780000503103232B702B4BDA70336843F008039D
:10781000336001E0804636E02D4B93F858210AB1E1
:1078200084F8B82093F859210AB12A490A7093F8CC
:107830005A3103B12B7033681B0718D564269AFBA5
:10784000F6F528460BF0E2FF074606FB15A000B24E
:107850000BF0DCFF20490CF02DF8014638460BF008
:1078600021FF1E490CF026F8C4F8540102E0002361
:10787000C4F854314FF0010B0BE0012FCCD91F4657
:107880009FE7022348E7012FC6D9002785F800802B
:107890009DE758460BB0BDE8F08F00BF6C1100208B
:1078A000F1390008F33900082D420008313E000884
:1078B0008D37000854000020A4100020E33300207E
:1078C000489F0108E433002003FA0008A9F60008E5
:1078D000EC290020E23300208988883C0000204108
:1078E0000120002109F0ACBCF8B5494B494C1B689C
:1078F000D4F858219A1A002AC0F2888003F5C333BD
:10790000A033C4F8583104F5AE70D4F8503198471C
:10791000414B04F5AE701A78014601F08DFB3F4BE8
:1079200004F5AE7519781A4611F0040F14D0D4F886
:107930005831C4F864310023394800261844A0F8AF
:107940007461EE5A37481E5206301E520233062B1F
:10795000F2D121F00401117094F874212D4BAAB1D9
:107960002F49B3F85C21B1F87401121AA3F85C2115
:10797000B1F87601B3F85E21B1F87811121AA3F8C4
:107980005E21B3F86021521AA3F86021D4F8641183
:10799000204A00293AD0D2F8583102F5B4745B1A63
:1079A000214902F5B7708B421BD8204AD36883F077
:1079B0000803D360002335F8132034F9137016B28E
:1079C000B742C8BF174F4FEA4301C8BF27F813207B
:1079D000475E0133B742BCBF154E8A53032BEAD131
:1079E000F8BD00231349C2F8643134F9135030F95B
:1079F000132001332A44022592FBF5F2032B21F8D0
:107A0000022FF2D1BDE8F84003F0FEB9F8BD00BF87
:107A1000C03300206C110020E4330020A8100020A7
:107A2000EC290020D41200207FC3C901000C0140C2
:107A3000DA1200205E2B0020174AF0B5164692F8A5
:107A40007531D2F878E1042B10D85C1C0EEBC3031F
:107A50009D1CE4B208D09A88D10705D5104203D006
:107A600008E00131052907D12346ECE786F8753196
:107A70000020F0BD9F7800210C2202FB01F3064D8F
:107A800005F5BE7C1CF803209742EAD12B4485F80B
:107A90007541D3F88001F0BD6C110020F8B50446A3
:107AA0000E4617460025204620210FF038FC0446DC
:107AB000D0B1013420460FF095FCB0F5617F05DBB5
:107AC00040F634039842A8BF184601E04FF46170B5
:107AD000A0F56170192390FBF3F00DB9307000E050
:107AE00070703B7801333B700DB90125DBE7204610
:107AF000F8BD7FB504780646E4B9364B19211868FD
:107B000000EB840090F87B5090F879204D4305F508
:107B1000617590F87A30009590F87C00414301F54A
:107B2000617101912C482146013402F043FD142C6F
:107B3000E3D14CE00FF056FC1328054641DC254B01
:107B4000701C1C68202100238DF80F300FF0E7FB1C
:107B50001E35064670B1013630460FF043FC192839
:107B60009FBF04EB850358709DF80F30013398BF19
:107B70008DF80F30304620210FF0D1FB064670B152
:107B8000013630460FF02EFC0D289FBF04EB850315
:107B900098709DF80F30013398BF8DF80F3004EBCB
:107BA00085043046E11C0DF10F02FFF777FF9DF8C9
:107BB0000F30042B0BD0601C002104220FF079FB46
:107BC00005E0064806490022132302F0F3FC04B046
:107BD00070BD00BFE00F00208CC10108A1C10108E9
:107BE000C0C10108014809F0CDBB00BFC6C10108F2
:107BF0002DE9F04304788FB00546002C59D17B4B1A
:107C00000021142209A807AED3F800800FF051FB21
:107C10000722304600210FF04CFB00231A46A70034
:107C200005A8059308EB070583807149B5F802E0C4
:107C300031F813C01CEA0E0F0AD00E310DF1380CCA
:107C4000595C02F1010E624402F81C1C5FFA8EF2CC
:107C50000133072BE9D100210B46664AB5F802E053
:107C600011F802C01CEA0E0F0AD006320DF1380CD2
:107C70008A5C03F1010E634403F8242C5FFA8EF34F
:107C800001310629E9D118F807308DE841006A78FA
:107C90005949029209A81A0903F00F0302F075FC72
:107CA0002146564809AA013402F084FC202CA6D1B2
:107CB00099E00FF097FB1F28044600F386802846C2
:107CC0002021E4B20FF02BFB1F2C02D9FFF78AFF13
:107CD00089E0464B451C1B68002103EB84042046C9
:107CE00004220FF0E6FA0027454B09AE304600218A
:107CF0000A2217F803905FFA87F80FF0DAFA0023E8
:107D000015F8012B32B10A2B04D04A4502D0F254A7
:107D10000133F5E74A455FD108F1FF33032B09D85A
:107D2000DFE803F01005023F0DF1230134E00DF10F
:107D300023011EE030460FF055FB2378C0B243EA22
:107D4000001006E030460FF04DFB237800F00F00E6
:107D50001843207031E00133062B0AD0244800F18B
:107D60001B069E5D9642F6D103445A7D63881343F9
:107D7000638011F8012F02B30023EFE70133072BD3
:107D80000AD01B4800F10E069E5D9642F6D130F8EF
:107D9000132063881343638011F8012F6AB1002315
:107DA000EFE730460FF01EFB0F2804DC30460FF0E3
:107DB00019FB607001E0002363700137052F93D138
:107DC000012409F0F3FD74B980E70E4900221F2356
:107DD0000D4802F0EFFB06E02046002104220FF0E0
:107DE00068FA0024EDE70FB0BDE8F083241300200B
:107DF000789F01088D9F0108D4C10108E3C10108E3
:107E0000999F0108C0C10108A1C101082DE9F041F5
:107E1000047807467CB9344D2146B5F8BC21B5F845
:107E2000BE313248013402F0C5FB042C05F10405D3
:107E3000F2D1BDE8F0812E490FF044FAB0B92A4BD7
:107E40004FF47A714FF4FA62A3F8BC11A3F8BE2183
:107E5000A3F8C011A3F8C221A3F8C411A3F8C62146
:107E6000A3F8C811A3F8CA21BDE8F08138460FF085
:107E7000B9FA032805462ED8384620210FF04FFACC
:107E8000044630B1013420460FF0ACFA0127064613
:107E900000E00746204620210FF041FA10B9BDE866
:107EA000F0419FE601300FF09DFA012FF7D140F22B
:107EB000DC53A6F2EE229A42F1D8A0F2EE229A42C8
:107EC000EDD88642EBDA084B6E3503EB85039E80D6
:107ED000D880BDE8F0810748074900220323BDE8A8
:107EE000F04102F067BB00BFEC290020EFC10108A0
:107EF00002C20108A1C10108D9CF01082DE9FF4143
:107F000004780546002C34D16E4809F03BFA6E4DDA
:107F1000686900210BF062FE002840F0CF80214606
:107F20006A4802F047FB6869694602F0C9F90146F0
:107F3000674802F03FFBA869694602F0C1F90146B3
:107F4000634802F037FBE869694602F0B9F9014677
:107F50005F4802F02FFB286A694602F0B1F901344C
:107F600001465C4802F026FB0C2C05F11005CFD130
:107F7000A4E0594905220FF0E9F938B9524B002223
:107F800003441030C0285A61F8D197E0284653497D
:107F900004220FF0DBF904462846002C3FD12021B3
:107FA0000FF0BDF9002800F08980451C28460FF02D
:107FB000C4F907464A4B53F824601EB9494809F0F2
:107FC000E1F97BE028463146FAB20FF0BFF90134FF
:107FD0000028EFD13C4B0021C2181030C02851615D
:107FE0009E46F7D1404B03EBC402D2F804C098463A
:107FF000BCF1000F04D131463C4802F0DBFA53E0FB
:10800000002718F834309F42F5DA3B010EEB0305E8
:10801000143563440FCB013785E80F00F1E70FF00B
:10802000E1F90B28064643DC284620210FF077F9BA
:10803000054648B10135284602F0ACF8224B012430
:1080400003EB0613586100E00446284620210FF098
:1080500066F9054640B10135284602F09BF81A4BF7
:10806000013403EB06139861284620210FF057F9DD
:10807000054640B10135284602F08CF8124B013418
:1080800003EB0613D861284620210FF048F910B9F8
:10809000FFF7A8FD12E0013002F07CF80A4B032C38
:1080A00003EB06163062F3D11148FFF727FF05E016
:1080B0001048114901220C2302F07CFA04B0BDE8FB
:1080C000F08100BF08C20108EC29002023C201088A
:1080D00029C2010835CD010802C201082DC20108DC
:1080E000E4A6010832C20108BCC0010841C201086F
:1080F00080BF0108A1C10108C0C10108F0B5047822
:1081000087B0064614BB514B19201968062303FBA0
:10811000041191F8CA5091F8CE20454305F56175D8
:1081200091F8C930009591F8CB50C831684300F5FB
:108130006170019008790290497945480391214680
:10814000013402F037FA0C2CDDD17DE00FF04AF952
:108150000B28044672DC3D4B701C1D682021002357
:108160008DF817300FF0DBF8064680B10136304647
:108170000FF038F903289FBF062303FB045383F84D
:10818000CE009DF817309CBF01338DF81730304674
:1081900020210FF0C4F8074680B1013738460FF0B0
:1081A00021F90D289FBF062303FB045383F8C90060
:1081B0009DF817309CBF01338DF8173006266643B3
:1081C000A9193846CA310DF11702FFF767FC2021C3
:1081D0000FF0A5F8074670B1013738460FF002F9E5
:1081E00014289FBF9DF817307619013386F8CC000C
:1081F00098BF8DF81730384620210FF090F878B1ED
:1082000001300FF0EFF80D289FBF062303FB045346
:1082100083F8CD009DF817309CBF01338DF81730DF
:108220009DF81730062B0FD0062202FB04500021C8
:10823000C9300FF03EF8FFF7D5FC05E005480649C8
:1082400000220B2302F0B6F907B0F0BDE00F0020CA
:108250004DC20108A1C10108C0C10108F7B50478E9
:1082600005464CB9204601A90AF0ACFD0134FFF7E0
:10827000F5FF0E2CF6D150E00FF0B4F8C6B20D2E7B
:1082800047D8681C20210FF04AF8034650B15B78AC
:108290000130682B07D0732B01D1012704E0FFF7D1
:1082A000A1FC3AE000E0002720210FF038F81C4C38
:1082B00006F1D005C8B101300FF094F840F2ED237B
:1082C00080B2984205DD40F6CA039842A8BF18461E
:1082D00001E040F2EE20A0F2EE20192290FBF2F035
:1082E00004EB450304F81570587014F8153004EBCE
:1082F00045046278012B4FF0190303FB02F331466A
:108300000CBF7322682203F2EE23064802F052F9F2
:1083100003E005480E2102F04DF903B0F0BD00BFA7
:10832000EC2900206DC201087FC2010810B5044687
:10833000204605F00CFF18B90A2005F042FEF7E7C9
:1083400010BD30B5094900220B78094C15578542FC
:1083500002BFFF25155503F1FF3302F10C0208BFE0
:10836000DBB23C2AF1D10B7030BD00BF651000209C
:10837000E8120020002208490C2303FB021359686D
:10838000814204D10022C2621A725A6070470132DF
:10839000052AF0D1704700BFE81200202DE9F7430D
:1083A000064689469DF8288011461A469DF82C30CD
:1083B00000250C2068431D4FC419C057B04202D19C
:1083C000207A20B12BE00135052DF2D127E0022ED5
:1083D0000FD005DC56B1012E21D1009314480AE0DC
:1083E0001E2E0DD01F2E1AD1012009E00093114836
:1083F00001E011480093434604F028FC044605E0E0
:1084000002F090FF4146044605F09EFE4CB10C235D
:1084100003FB0575267185F808906C6001E000206B
:1084200000E0204603B0BDE8F08300BFE812002062
:1084300000440040003801400048004010B5084B9F
:108440000022196801EBC20393F90240844201D172
:10845000981C10BD0132052AF4D1002010BD00BFC8
:10846000E4120020F0B5027887B08AB94A4C04F1D2
:10847000280694F8E8210023484950B25956814211
:108480006ED00C333C2BF7D10834B442F1D181E0EB
:10849000002204920592451C0EF0A4FFC4B260B203
:1084A000FFF7CCFF074618B18DF81040012400E01B
:1084B0000446284620210EF032FF054638B101352A
:1084C00028460EF08FFF0134ADF81200E4B200260A
:1084D000284620210EF023FFB0B3451C28460EF09D
:1084E00081FF00222E495FFA82FE51F8223083423A
:1084F00004D00132082AF5D1002300E0734651F878
:108500002320824220D1022E0FD0032E12D05A1ED9
:10851000012ED2B204D0042A13D88DF814300EE004
:10852000042A0ED88DF8153009E0052B09D88DF8EE
:10853000173004E09A1E052A03D88DF8163001344E
:10854000E4B20136042EC3D1052C04D807B0BDE82F
:10855000F040FFF747BB04AB03CB3860796019E00C
:1085600094F8ED010E4B94F8EC5153F82000B4F858
:10857000EA21009094F8EF0153F82000019094F85C
:10858000EE0153F8200053F825300290054802F020
:1085900011F879E707B0F0BDEC290020E8120020BF
:1085A000F89E010896C2010838B1438811EA030019
:1085B00003D08B420CBF01200220704730B50A4B1C
:1085C0000A491C680A79042A0AD81346551C04EB88
:1085D000C303EAB29D882842F5D00A71981C30BDC9
:1085E0000A71002030BD00BFE412002024130020D7
:1085F000014B00221A71E1E7241300202DE9F04716
:10860000877890F803C0BBB2C7F1640E03EB830612
:108610005C42C3F178001C4D5FFA8EFE7600CCF10F
:108620006408A4B280B2A3B20FFA83F9B9F1000FC3
:1086300004DC002B14BF3B46012300E0734609FB1A
:1086400009F25B4302FB0CF292FBF3F3434403FB9E
:1086500009F30A2293FBF2F333449BB225F8023F5D
:10866000B1F800904A880A34C9EB020A1AB202FB38
:108670000AF24FF47A7392FBF3F3A4B24B448442B0
:108680002B80D0D1BDE8F0872813002010B54478A6
:108690000078002240F6C41102FB02F3193B634349
:1086A00003F6C4135343434393FBF1F3034921F807
:1086B00012300132072AEDD110BD00BF4213002055
:1086C000104B043033F91000B0F5617F05DB40F644
:1086D00033039842A8BF184601E04FF461700A784E
:1086E00019235A4302F28332824208DA4A7853430A
:1086F00003F283338342B4BF00200120704700207F
:10870000704700BFC829002010B500F1500302785F
:108710008A4203D18478C278944204D304309842C8
:10872000F5D1002010BD012010BD00BF084BDA6854
:10873000D10709D4DA68520708D4DB6813F0100FA8
:1087400014BF0320042070470120704702207047A7
:108750000020024003788B4286BF024B33F81100A1
:1087600000207047501300200022134670B52349A3
:1087700014180C44247E83EA0423082413F4004FC5
:108780004FEA430318BF83F4815304F1FF3418BF49
:1087900083F0010314F0FF049BB2EFD10132192AD8
:1087A000E5D100F1190200F11A050A440D44167EC4
:1087B0002A7E02EB062292B29A421ED10F4B93F808
:1087C0003950E2B2AA4215D2431C03EB4203DBB29A
:1087D000CA1801330B44127E1B7E03EB02239BB2AB
:1087E0004FF4AF6253431B1303F5487321F8143061
:1087F0000134E6E7012381F83A3070BD50130020C0
:1088000003788B420BD9074B890093F83B2019441E
:10881000C86B02B1400800F5777080B27047002045
:10882000704700BF5013002007299DBF034B03EB87
:108830008101B1F86C000020704700BF5013002088
:10884000034B03EB8101D1F88C00C0F3CF007047DC
:108850005013002008B5084B03EB8101D1F8CC0080
:108860000AF0D0FF05490BF025F805490AF01AFF78
:108870000BF00CFA80B208BD501300200000203F1E
:1088800000005C44014B33F811007047C8290020F8
:10889000024B03EB4101B1F8140170475013002063
:1088A00070B5054605F066FB314CD4F82C31C4F8A0
:1088B0002C01C31AB3F5FA5FC4F8303182BF00232C
:1088C00084F8343184F8353194F834312BB9A12D42
:1088D00002BF274A012182F8351194F83511244A44
:1088E00029B1D118EDB201330D7682F8343194F804
:1088F000345194F83631AB4239D11D4B93F83731AE
:10890000052B02D0062B03D02CE00020FFF72CFF14
:10891000637E1E2B26D100200246C1B26B1E9942F7
:1089200019DA21440B7E0821DBB283EA0206F6073E
:1089300044BF83F01803C3F3460301F1FF3154BF72
:108940005B0843F0800311F0FF01C2F34702ECD152
:1089500001301A46E1E723441B7E9A4202D10320EC
:10896000FFF702FF002384F8353184F8343170BDFD
:108970005013002010B5044605F0FCFA41F288318E
:108980000E4BE4B2D3F83821C3F83801821A8A4278
:10899000C3F83C2184BF002283F8402193F8402192
:1089A00006490F2A134418BF013283F8414112BF10
:1089B00081F84021012381F8513110BD501300206E
:1089C00010B5044605F0D6FA41F288310E4BD3F8C3
:1089D0005421C3F85401821A8A42C3F8582184BF33
:1089E000002283F85C2193F85C210749142A134480
:1089F00018BF013283F85D4112BF81F85C21012369
:108A000081F8723110BD00BF5013002010B504462C
:108A100005F0B0FA184A1849D2F87431C2F8740156
:108A2000C31AB3F57A6F84BF002382F8783192F8C5
:108A3000783123B9A82C1DD181F8793106E0022BB9
:108A400002D181F87A4101E0242B02D8D11881F8B3
:108A50007B410133DBB282F8783192F87A21064902
:108A600052000532934201BF002381F8783101237F
:108A700081F8793110BD00BF5013002010B50446B5
:108A800005F078FA40F6AC510F4AD2F8A031C31A7B
:108A90008B42C4BF002382F8A43192F8A431D118CC
:108AA00081F8A54123B90F2C0DD10749C1F8A001C8
:108AB0000133DBB2192B044982F8A4310CBF012326
:108AC000002381F8BE3110BD501300208A6810B514
:108AD0000C6A036814430A6923F4FF4314434A6988
:108AE00023F0700314438A691443CA6914434A6A21
:108AF00014438A6A224313430360CB6843600B68C4
:108B000083604B68C36010BD4FF6FE73026813406C
:108B100003600023036043608360C360284B984276
:108B200001D1284A27E0284B984201D1254A2AE062
:108B3000264B984201D1234A2DE0254B984201D182
:108B4000204A30E0234B984201D11E4A33E0224BA9
:108B5000984204D11B4A536843F470032EE01F4B24
:108B6000984204D1174A536843F0706326E01C4BC7
:108B7000984204D11B4A536843F00F031EE01A4B7E
:108B8000984204D1174A536843F0F00316E0174B9C
:108B9000984204D1134A536843F470630EE0144BB7
:108BA000984204D10F4A536843F4704306E0114BD6
:108BB000984204D10B4A536843F4702353607047C2
:108BC00008000240000002401C0002403000024049
:108BD00044000240580002406C0002408000024005
:108BE00008040240000402401C0402403004024019
:108BF00044040240580402401F4A10B5536803F071
:108C00000C03042B03D0082B04D01C4B14E01C4B8A
:108C10001B6811E053685168C3F38343C90303F130
:108C2000020301D4174906E0516811F4003F1449CA
:108C3000096818BF49084B43036053681249C3F3DE
:108C40000313CC5C0368E34043605468C4F302241C
:108C50000C5D23FA04F484605468C4F3C2240C5DF0
:108C6000E340C3605268C2F381320A44127CB3FB12
:108C7000F2F3036110BD00BF0010024000127A0041
:108C80002400002000093D0060A4010810B504463E
:108C9000FFF74CFD012806D11CB1FFF747FD013C51
:108CA000F8E7052010BD002C08BF052010BD0A887C
:108CB000F0B54B888E88B1F808E0CC88002A3AD10C
:108CC000028C43F0010322F001021204120C028410
:108CD000058B078CADB225F0F30545EA0E1189B27C
:108CE00041EA06027A49BFB2884212D001F500611A
:108CF00088420ED0B0F1804F0BD0A1F59831884258
:108D000007D001F58061884203D001F58061884277
:108D100002D127F0020701E027F00A071F43028370
:108D20000784038B23F00C031B041B0C0383038BAE
:108D30009BB21C4344E0042A44D1028C22F010026E
:108D40001204120C0284018B058C21F4407212056E
:108D5000120D42EA0E325E4992B242EA062288427F
:108D6000ADB292B212D001F5006188420ED0B0F1DE
:108D7000804F0BD0A1F59831884207D001F5806172
:108D8000884203D001F58061884207D125F0200197
:108D900041EA03139BB243F0100304E025F0A00165
:108DA00043F010030B4302830384038B23F44063DB
:108DB0001B041B0C0383038B9BB243EA0424A4B261
:108DC0000483F0BD082A028C3ED122F48072120482
:108DD000120C0284828B3E4D92B222F0F307018C7A
:108DE00047EA0E1292B2A84289B242EA060212D0B3
:108DF00005F50065A8420ED0B0F1804F0BD0A5F567
:108E00009835A84207D005F58065A84203D005F53E
:108E10008065A84207D121F4007141EA03239BB287
:108E200043F4807304E021F4206143F480730B4326
:108E300082830384838B23F00C031B041B0C83832A
:108E4000838B9BB21C4341E022F480521204120C2B
:108E50000284858B018C25F440752D052D0D45EA86
:108E6000062545EA0E321A4D89B2A84292B212D0B6
:108E700005F50065A8420ED0B0F1804F0BD0A5F5E6
:108E80009835A84207D005F58065A84203D005F5BE
:108E90008065A84207D121F4005141EA03339BB217
:108EA00043F4805305E047F6FF5543F480530D40EB
:108EB0002B4382830384838B23F440631B041B0CAA
:108EC0008383838B9BB243EA0424A4B28483F0BDE2
:108ED000002C0140016830B5CD43154B1C682C4077
:108EE0001C605A682A405A60027902F1804202F5F9
:108EF000823214682143116002689C68D5432C407B
:108F00009C60D9682940D9604179102909BF9968C6
:108F100001F180431143996015BF03F58233D9688D
:108F200019680A4316BF0A43DA601A6030BD00BFF1
:108F300000040140054B1A685B69034004D01042ED
:108F400014BF0120002070471846704700040140FC
:108F5000CA78F0B5D40648BF8C780D8802F00F03AC
:108F600048BF234315F0FF0F1DD0016800240126E0
:108F7000A64006EA0507B74211D14FEA840E0F2634
:108F800006FA0EF621EA0601282A03FA0EF641EA4D
:108F9000060101D1476102E0482A08BF0761013498
:108FA000082CE4D10160FF2D1FD94168002404F191
:108FB00008070126BE4006EA0507B74211D14FEA6D
:108FC000840E0F2606FA0EF621EA0601282A03FA75
:108FD0000EF641EA060101D1476102E0482A08BFC6
:108FE00007610134082CE2D14160F0BD0F4B1A68D3
:108FF00042F001021A6059680D4A0A405A601A6824
:1090000022F0847222F480321A601A6822F48022DC
:109010001A605A6822F4FE025A604FF41F029A60E6
:10902000044B4FF000629A60704700BF001002408E
:109030000000FFF800ED00E02DE9F8435B4C036809
:10904000013AC4F8C03183880D46A4F8C431072A18
:1090500042D8DFE802F0040A101822292F35B4F8AC
:10906000C0310B80B4F8C23113E0B4F8C2310B80C8
:10907000B4F8C03105E0B4F8C0315B420B80B4F8FD
:10908000C2315B4205E0B4F8C2315B420B80B4F8F8
:10909000C0316B80B4F8C4311DE0B4F8C0315B421C
:1090A0000B80B4F8C23112E0B4F8C2310B80B4F8CE
:1090B000C0310CE0B4F8C0310B80B4F8C23105E027
:1090C000B4F8C2315B420B80B4F8C0315B426B80B4
:1090D000B4F8C4315B42AB80354B1B79002B62D1B5
:1090E000B5F900000AF092FB8046B5F902000AF0DB
:1090F0008DFB0746B5F904000AF088FBD4F8C811C7
:10910000064640460AF0D6FBD4F8D41181463846CC
:109110000AF0D0FB014648460AF0C4FAD4F8E01140
:10912000814630460AF0C6FB014648460AF0BAFAC4
:109130000EF0CCFAD4F8CC11288040460AF0BAFBE5
:10914000D4F8D811814638460AF0B4FB01464846A7
:109150000AF0A8FAD4F8E411814630460AF0AAFBD6
:10916000014648460AF09EFA0EF0B0FAD4F8D01143
:10917000688040460AF09EFBD4F8DC1180463846F1
:109180000AF098FB014640460AF08CFAD4F8E81140
:10919000074630460AF08EFB014638460AF082FA4E
:1091A0000EF094FAA880BDE8F88300BF50130020A9
:1091B0002400002038B50F4B1B689C890E4B1868A3
:1091C00080F31000201A0AF021FB0C490AF072FB10
:1091D000054620460AF01AFB014628460AF01EFC06
:1091E0000AF02EFD6428A8BF642020EAE070C0B217
:1091F00038BD00BF90100020A01000200000C84221
:1092000044F6FB71084B1A68137803EB431300FB19
:1092100003135078C0EB0030B3FBF0F39078B3FB4E
:10922000F0F080B2704700BF9010002008B50A48E7
:109230000A2290F8ED3100EB4303B3F8FC1100F57E
:10924000027089B220F8041C04F090FF80B2FFF78E
:10925000D7FF024B188008BD501300209410002047
:109260002DE9F047604E356815F4804540F0B9802F
:109270005E4B2F46994683F8905299F89C82FCB237
:109280004445DFF868A180F08C80DAF89432DFF88A
:1092900064811BB920460AF099F97EE0DAF8982239
:1092A000DFF848A1072C94BF115D21460AF527700D
:1092B0009847032C2FD8DAF8982204F10C0302EB1C
:1092C0008303B3F804E0D988B8B1CEEB00004FF4C3
:1092D0007A734343CEEB010093FBF0F040F6C903F1
:1092E00000F57A70984205DC40F2EE239842B8BF50
:1092F000184601E040F6CA0080B2938A83420AD839
:10930000D38A834221BF012399F89022A3401343BB
:1093100028BF89F89032D9F898329A8A824206D8C2
:10932000DB8A834203D3314B93F89E3213B9204634
:109330000AF04CF942F2010233681A406AB399F814
:109340009F220323B2FBF3F303EB4303D31A610021
:10935000DBB201EB040E734409EB4303A3F8A00254
:1093600099F8E8322BB9022A17D9204B012283F849
:10937000E822062303FB0493B3F8A002B3F8A22269
:10938000B3F8A4321044184480B24944A1F8EA0268
:10939000032300B290FBF3F080B228F814000137E9
:1093A0006BE79AF890320F2B09D1114B5B79C3B15F
:1093B0000AF000F901238AF89E32BDE8F08733688D
:1093C0009B0402D500238AF89E32E8B2404506D2BB
:1093D0000AF0FCF8074B23F815000135F5E7BDE866
:1093E000F087BDE8F08700BF8C29002050130020D3
:1093F00024000020C82900200028114AB8BF40429C
:1094000090FBF2F330B50F4C3C2504FB030068439E
:109410000D4D90FBF2F22D682D7B25B903EB8303F4
:1094200003EB830301E0C3EB031302EB830304FBB1
:1094300002020B804FF47A7392FBF3F24A8030BD44
:1094400080969800806967FF98100020022803D05A
:10945000431E584258417047064B1B681B7823B186
:10946000054B1868C0F3C0407047044B1878C0F330
:1094700080007047F40D0020A80F0020E133002089
:10948000A0F17D03012B70B504460D460A4E05D8A8
:1094900030687D2104F067FE84F0200430682146A6
:1094A00004F061FE35B12B881C4404EB142404F055
:1094B000FF042C8070BD00BF5811002010B50A4C6D
:1094C0005E280146206805D15D2104F04CFE20682D
:1094D0003E2105E05D2903D104F045FE20683D21D1
:1094E000BDE8104004F03FBE5816002037B51A4BB7
:1094F0001A4C1B491B4A20B11B480088B0F5805FFD
:1095000021D209881278154D9B79ADF804108DF899
:10951000062001A8291D04228DF807300DF0AEFEAB
:10952000C0B101986860532009F05AF9A08809F089
:1095300089F9A07909F086F9E07909F083F90A4BF5
:1095400000221A8006E0098812789B79A180A27116
:10955000E371E8E703B030BDA833002058160020BF
:1095600068110020A8100020803300202DE9F84366
:1095700005460E460D4B002493E88003B44213DAEF
:109580007B1933F9140008EB050333F9142009EBB8
:10959000050333F9143001341344022293FBF2F330
:1095A000C01A09F05EF9E9E7BDE8F883DC31002074
:1095B00030B585B004AC002524F8025D0091ADF80B
:1095C000060021461020FFF75BFF9DF806002146AC
:1095D000FFF756FF9DF807002146FFF751FF9DF862
:1095E00000002146FFF74CFF9DF801002146FFF7E0
:1095F00047FF9DF802002146FFF742FF9DF8030058
:109600002146FFF73DFF9DF80E002946C043C0B23A
:10961000FFF736FF05B030BD10B5054C206804F0EB
:109620009FFD18B1206804F098FDF6E710BD00BF5B
:109630002C11002010B50446C0B2FFF73FFFC4F361
:109640000720BDE8104039E7024B5E21186804F09E
:109650008ABD00BF5816002038B50546054C5E216E
:10966000206804F080FD20682946BDE8384004F0F9
:109670007ABD00BF5816002013B5044601A9006842
:10968000FFF7BAFE1320FFF7E7FFBDF90400FFF76D
:10969000D1FF1B20FFF7E0FFBDF90600FFF7CAFF6F
:1096A0002320FFF7D9FF2368002BB4BF53204E209F
:1096B000FFF7C0FF01A96068FFF79EFE1220FFF7C9
:1096C000CBFFBDF90400FFF7B5FF1A20FFF7C4FF79
:1096D000BDF90600FFF7AEFF2220FFF7BDFF63686C
:1096E000002BB4BF57204520FFF7A4FF02B010BDE8
:1096F000674B73B51878FFF7A9FE664D04462B78C3
:10970000834220D0C8B1644B1B68E3B193F90000D9
:1097100002230093614B04211B6800225B78003315
:1097200018BF012301934FF41653FEF737FE5C4B2D
:10973000186040B101232B7005E0594E3068FEF7E8
:1097400019FE34602C70574B574D1878FFF77EFE8A
:109750002B780446834218D088B1544B1B68A3B1C0
:109760000022012493F9000008214FF4964300944D
:109770000192FEF713FE4E4B186028B905E04C4EDF
:109780003068FEF7F7FD34602C704A4B4A4D18786C
:10979000FFF75CFE2B78044683422E4643D0002818
:1097A00038D0464B1A68002A3DD0D37992F9000090
:1097B000002B4FF00202424C08BF0223009200220D
:1097C00054F8233001921021FEF7E8FD3D4B054689
:1097D000186040B33C4C94F84A30022B0BD094F8FC
:1097E0009620022A01D14C3405E023B1002A04F16D
:1097F0004C0418BF0024354B1C6044B120460021A6
:109800004C220DF056FD0223256084F84A300123D6
:10981000337008E02B4E306807F0C4FC3068FEF768
:10982000A9FD34602C702A4B2A4D1878FFF70EFEE4
:109830002B780446834229D000B3274B1B682BB3F7
:10984000264A93F900001268032352782021002A47
:109850000CBF08220922009301924FF461430022B9
:10986000FEF79CFD1E4B186080B11E4A0123137049
:109870002B701D4B1A681D4B1A6007E0184E30689C
:10988000FEF778FD174B34601C702C7002B070BD71
:10989000FC0D002068100020F80D0020981000201A
:1098A00058160020040E0020B8100020000E0020E2
:1098B0002C110020100E00203E1100200C0E002064
:1098C000F89E0108401100206C1100204411002076
:1098D0001C0E002054110020180E0020140E002031
:1098E000581100205C110020B029002060110020D8
:1098F0002DE9F74304F03EFB924CA368C31A002BFA
:10990000C0F2618300F5433303F5A073A3608E4B6F
:109910001D78237BC5F38005EB1A18BF012325733F
:109920004DB1002B00F04F83884B5A789A7001227A
:109930005A701A702BE0854A2BB1D37843F002039A
:10994000D37093785370D67806F0020101F0FF03CC
:1099500039B97E498968411A002903DB06F0010301
:1099600000E0012303F00107784917707BB1F2078B
:109970000DD50A7905230132D2B2B2FBF3F303EB22
:109980008303D31A724ADBB20B71D35C4B706F4EF8
:10999000DFF8088233787BB3F37823F00203F370A7
:1099A0006C4B0344AE20B36006F0B5F908B106F085
:1099B000B7F988F80000002800F00583B02006F011
:1099C000AAF9402006F0A7F9002006F0A4F910201B
:1099D00006F0A1F94FF48067013F0020BFB206F006
:1099E00071F9002FF8D1384606F009FA72785A4B0F
:1099F00053F8220006F086F998F80030002B00F0AA
:109A0000E2827378062B00F2B382DFE813F00700DE
:109A1000B102180078006B018801ED014F49504AEE
:109A2000504B514800F0B1FD012006F0E8F94E48D6
:109A300006F068F9022006F0E2F94C48ADE14C4F1F
:109A40003B689B0735D5DFF858810A23B8F800102A
:109A5000DFF85091B1FBF3F203FB121399F80010F9
:109A600092B29BB200914048424900F08EFD01F055
:109A700005FF012006F0C3F93B4806F043F93E4BD1
:109A800099F800201868B8F80030067902FB163102
:109A900064234B43C17802208E1B5643B3FBF6F67A
:109AA000F6B206F0ACF93146152001F0ABFE032604
:109AB00000E001263B681F0540F15A822F4B3049D8
:109AC0001F68642397FBF3F2096803FB127300918C
:109AD00025482C4900F059FD01F0D0FE304606F033
:109AE0008EF9214806F00EF9FFF764FB0746701C5B
:109AF00006F085F91520394601F084FE38E2012090
:109B0000214F06F07CF9214806F0FCF83B689807E5
:109B10004AD51F4A1448B2F90210B2F90030009138
:109B2000B2F904201B4901921B4A00F02EFD01F0FE
:109B3000A5FE022006F063F90B4806F0E3F80326C1
:109B400033E000BF58160020E1330020D02600206B
:109B5000B5C20108404B4C0074A40108BAC2010808
:109B6000C3C20108A5BB010865160020C9C20108CF
:109B70008C290020D0C20108901000209C100020E9
:109B8000A0100020E8C20108A4100020FDC20108B6
:109B90007210002013C3010822C30108A50A002087
:109BA000941000205000002002263B68D9071AD5E7
:109BB0007B4A7C48B2F90210B2F900300091B2F948
:109BC000042079490192794A00F0DFFC06F101088E
:109BD00001F054FE304606F012F95FFA88F8714839
:109BE00006F090F846463B681A0718D5704A6D484B
:109BF000B2F90210B2F900300091B2F904206A49BA
:109C000001926C4A00F0C1FC771C01F037FE30462F
:109C100006F0F5F8FFB2634806F074F83E46664A6F
:109C20006149B2F90030B2F902205E480092634AFD
:109C3000DFF8B091B2F90020771C0192604A00F081
:109C4000A4FC01F01BFE304606F0D9F8554806F09A
:109C500059F85449D9F8000000F032FB51480DF092
:109C60006CFBFFB2C1B2092909D84B1CDBB22144FD
:109C700020224A730021E21891731946F3E7DFF8B6
:109C80002481D9F80400414400F01AFB01F0F6FDEC
:109C9000384606F0B4F8404606F034F84146D9F8A4
:109CA000080000F00DFB40460DF047FB0236F6B20F
:109CB000C7B2092F09D87B1CDBB2274420227A7354
:109CC0000021E21891731F46F3E73E4BB3F9000001
:109CD00009F09CFD08EB070100F0F2FA01F0CEFD5F
:109CE000304657E00026384F3B78B34240F240817F
:109CF0000E2E00F03D817008013006F080F83046ED
:109D000009F03AF83B78B34206D9202005F0DFFF8E
:109D1000701CC0B209F030F80236F6B2E3E72B4E01
:109D20002B4996F8A8271F4800F02FFC012006F0C9
:109D300066F81C4805F0E6FF264B27491F781948AE
:109D40003A4600F022FC022006F059F8154805F0CA
:109D5000D9FF0C2303FB0766204996F8AB2796F83A
:109D6000AA37104800F011FC01F088FD032006F02E
:109D700046F80C4805F0C6FF96F8B01796F8AE27DF
:109D800096F8AF3707480091154900F0FEFB01F047
:109D900075FD042006F033F8024805F0B3FFE7E054
:109DA000C80F00206516002013C3010826C3010850
:109DB000C8120020B9D80108842900208010002092
:109DC0002AC301089C260020EC150020EC29002065
:109DD0002EC30108B02700203AC301084BC3010875
:109DE0005CC3010890260020784B1B681B0640F1DD
:109DF000BB80636AA16A764A8B421CBF936292F869
:109E00002C304FF001011CBF013303F003034FF06E
:109E1000000018BF82F82C3005F0FDFF94F82C30BC
:109E20006C4A0026D05C05F052FF0220012105F0AB
:109E3000F2FF694B3620F35C0136C3EBC30393FB9F
:109E4000F0F0C0B2062828BF06206038C0B205F086
:109E50003EFF102EEDD1614B61491B78614813F034
:109E6000020F614B1A7814BF59234E2300F08DFB6B
:109E700001F004FD022005F0C2FF5A4805F042FF40
:109E80005A495B4B4E680A68564892FBF3F25949AF
:109E900096FBF3F300F079FB01F0F0FC032005F0F2
:109EA000AEFF504805F02EFF534B54491A884D48D9
:109EB00000F06BFB01F0CFFC042005F0A0FF494847
:109EC00005F020FF4E4B4F491A88464800F05DFBD5
:109ED00001F0C1FC04210A2005F09DFF414805F076
:109EE00011FF4949226B3F4800F04FFB474E01F0FC
:109EF000B2FC052005F083FF3A4805F003FF7268C5
:109F0000B3684349374800F040FB01F0A4FC052149
:109F10000A2005F080FF334805F0F4FE3369F2684B
:109F20003C49D21A2F4800F030FB01F094FC062087
:109F300005F065FF2B4805F0E5FEB2683649294873
:109F400000F023FB01F087FC06210A2005F063FFE7
:109F5000244805F0D7FE3149152222480DF018FAA1
:109F600001F079FC072015E7F37843F00203F37062
:109F70004DBB2B4B00219B791220032B97BF294A05
:109F80003F259B181D7F05F046FF284605F09FFEE4
:109F90001320002105F03FFF234B1B78002B14BF3B
:109FA0005220212005F093FE1420002105F033FFFC
:109FB00094F83450074B585D013505F0030505F062
:109FC00086FE84F8345003B0BDE8F0838C2900206D
:109FD000581600206EC3010855100020A81000205C
:109FE00073C3010865160020AE100020B0100020D9
:109FF0008096980084C30108AA10002091C301082C
:10A000000C10002099C30108A0C301081802002009
:10A01000A7C30108B0C30108B7C30108B40A0020F0
:10A02000A833002074A40108EE150020F0B5012427
:10A03000B0FBF4F58D4201D34C43F9E70026D4B1CF
:10A04000B0FBF4F504FB1500B4FBF1F41EB9002DD0
:10A0500001DC002CF3D1092D03F1010EEFB204DD78
:10A06000002A14BF3725572500E030253D441D70D8
:10A0700001367346E3E71C70F0BDF0B50124B0FB78
:10A08000F4F58D4201D34C43F9E70026D4B1B0FB7F
:10A09000F4F504FB1500B4FBF1F41EB9002D01DC4E
:10A0A000002CF3D1092D03F1010EEFB204DD002ADB
:10A0B00014BF3725572500E030253D441D7001367B
:10A0C0007346E3E71C70F0BD03685A1C0260197008
:10A0D00070472DE9F843089E002B07468846144632
:10A0E000334614BF4FF030094FF0200913F8012B0D
:10A0F0000AB9254603E0002CFBDD013CF6E7002D04
:10A1000004DD38464946C047013DF8E7354624EAB4
:10A11000E474A01B284415F8011B11B13846C04750
:10A12000F7E7BDE8F883024B186804F01CB800BFDD
:10A13000580E0020F8B507460C4648680021154621
:10A140001E4609F04BFD58B1284609F05FFB104947
:10A1500009F0B0FB01464FF07E5009F05FFC6060F3
:10A160006168304609F09EFA0146304609F056FC17
:10A17000256806462946384609F092FA01463046D7
:10A1800009F098FB0146284609F08CFA2060F8BDDA
:10A19000DB0FC9402DE9F04102780346202A00F187
:10A1A0000100F9D0092AF7D02D2A02D10346414DEA
:10A1B00004E02B2A08BF03464FF07E551C460026BC
:10A1C000234614F8012BA2F13007F9B209290DD862
:10A1D0003949304609F06EFB0646384609F016FB51
:10A1E0000146304609F05EFA0646E9E72E2A17D105
:10A1F000314F234614F8010B3038C2B2092A0FD868
:10A2000009F004FB394609F009FC0146304609F023
:10A2100049FA29490646384609F04CFB0746E8E763
:10A220001A7802F0DF02452A39D15A782D2A02D154
:10A230000233012704E02B2A14BF01330233002725
:10A24000013B002413F8012F303AD1B2092903D879
:10A250000A2101FB0424F5E7B4F59A7F28BF4FF4E7
:10A260009A74A0464FF07E53B8F1070F07D91846ED
:10A27000124909F01FFBA8F108080346F4E704F0AF
:10A28000070434B118460C4909F014FB013C03469D
:10A29000F7E719462FB1304609F0C0FB04E04FF054
:10A2A0007E51304609F006FB0146284609F002FBC4
:10A2B000BDE8F081000080BF0000204120BCBE4C02
:10A2C00030B5054687B00C4603A800210C220CF0DF
:10A2D000F0FF2846002109F0A9FC20B128462849B2
:10A2E00009F0E0F903E02846254909F0D9F92549A4
:10A2F00009F0E0FA09F0A4FC054680EAE07069463E
:10A30000A0EBE57008F05EFD002DACBF20232D23EF
:10A3100068468DF80C300DF010F8012807D1302375
:10A320008DF80D308DF80E308DF80F300CE00228CE
:10A3300005D130238DF80D308DF80E3004E0032860
:10A3400004BF30238DF80D30694603A80CF0D8FF08
:10A3500003A80CF0F2FF0338C5B22A4603A9204631
:10A360000DF016F800236355204607490CF0C8FF8E
:10A3700003AB204659190CF0C3FF204607B030BD8F
:10A380006F12033A00007A44F0C3010870B5064624
:10A39000B6FBF2F40846154614B12046FFF7F6FF67
:10A3A00005FB1464024B1B5D00F8013B70BD00BF50
:10A3B000F2C301082DE9F04F81468A4616461C4635
:10A3C00089B000253178002900F0DB80252902D0F2
:10A3D0000136484674E072784FF00008302A0CBF0E
:10A3E000B278B71CA2F1300312BF4FF0000BF71C7C
:10A3F0004FF0010B092B19D8A2F13003D9B209296A
:10A4000005D80A2202FB083817F8012BF4E7A2F15D
:10A410006103052B02D8A2F1570305E0A2F1410325
:10A42000052B03D8A2F137030A2BEADD6C2A30D1C1
:10A430003A787E1C642A00F083800BD8252A3DD010
:10A4400003D8002A00F09D80BCE7582A0CD0632A6C
:10A4500019D0B7E7732A22D002D86E2A37D0B1E7D5
:10A46000752A5CD0782AADD1271D2068A2F1580446
:10A4700062424FF01001624155E02CD9582A32D087
:10A48000632A2AD13E4648462178271DD047013508
:10A490000FE0642A63D00ED9732A14D13E46236894
:10A4A00048460093514642460023FFF712FE271DFF
:10A4B00005443C4686E7252ADFD13E46484625210D
:10A4C000D04701357EE70AD86E2A06D13E4623687A
:10A4D00004341D6076E7002A53D03E4672E7752AA1
:10A4E00026D0782AF9D1A2F1580304F1040C5A427B
:10A4F0002068CDF80CC04FF010015A4105ABFFF7B2
:10A5000095FDDDF80CC03E46644605AB0093484619
:10A51000514642465B46FFF7DCFD054452E72068A2
:10A52000271D0A21002205ABFFF7A7FD3C46ECE7FB
:10A5300004F1040CCDF80CC020680A210022DDE7EC
:10A540002068271D002808DA2D238DF8143040429A
:10A550000DF115030A210022E6E705ABFAE72068B2
:10A5600004F1040C00280ADA2D238DF8143040423F
:10A570000DF11503CDF80CC00A210022BFE705AB91
:10A58000F8E7284609B0BDE8F08F0EB40FB505AB6B
:10A5900053F8042B0190064901A80393FFF70AFF23
:10A5A000019B00221A7004B05DF804EB03B0704701
:10A5B000C9A000080FB413B50B4904AB08680B49D8
:10A5C00053F8042B09680193FFF7F4FE0446084B87
:10A5D000186803F0BCFD0028F9D0204602B0BDE8A1
:10A5E000104004B0704700BF34090020300900203B
:10A5F000580E002080EAE073A3EBE0738B4206DB89
:10A60000002801DD401A704702D00844704700203E
:10A61000704770B5044609F013FB2030402857D826
:10A6200020462C4909F002FB28B120462A4909F0AE
:10A6300037F80446F4E72046284909F0D9FA28B14A
:10A640002046254909F02EF80446F4E7204624491F
:10A6500009F0ECFA30B12249204609F021F8014610
:10A660001F480AE020461F4909F0C2FA40B11C49C0
:10A67000204609F017F801461A4809F011F8044677
:10A680002146204609F016F905462046294609F0DC
:10A6900011F915490646284609F00CF9134908F046
:10A6A000FFFF0146284609F005F9114908F0FAFFB5
:10A6B0000146284609F0FEF80E4908F0F1FF014670
:10A6C000304609F0F7F80146204608F0EBFF70BD70
:10A6D000002070BDDB0F4940DB0FC940DB0F49C0D4
:10A6E000DB0FC93FDB0FC9BF9A7C2E36FAAF4F395B
:10A6F0003587083CA4AA2A3E08B5034908F0D2FFD2
:10A70000BDE8084085E700BFDB0FC93F2DE9F04FEA
:10A71000056885B0814628460C46FFF7EDFF804668
:10A720002846FFF776FFD9F8045006462846FFF77B
:10A73000E3FF07462846FFF76CFFD9F80890054667
:10A740004846FFF7D9FF82464846FFF762FF414679
:10A750008146504609F0AEF841468346484609F026
:10A76000A9F851460190304609F0A4F849460290F4
:10A77000304609F09FF839460390504609F09AF8A0
:10A780004946206007F1004009F094F829466060CE
:10A79000A560029809F08EF80146019808F082FF42
:10A7A0002946E060039809F085F80146584608F00C
:10A7B00077FF3946206106F1004009F07BF8294611
:10A7C0006061584609F076F80146039808F068FF82
:10A7D0002946A061019809F06DF80146029808F039
:10A7E00061FF4146E061384609F064F8206205B037
:10A7F000BDE8F08F2DE9F04107688AB046688568AA
:10A800000446084601A9FFF781FF0199384609F07F
:10A8100051F804998046304609F04CF8014640460C
:10A8200008F040FF07998046284609F043F80146A2
:10A83000404608F037FF02992060384609F03AF8A0
:10A8400005998046304609F035F80146404608F043
:10A8500029FF08998046284609F02CF80146404611
:10A8600008F020FF03996060384609F023F8069944
:10A870000746304609F01EF80146384608F012FF38
:10A8800009990646284609F015F80146304608F0B1
:10A8900009FFA0600AB0BDE8F081074B10B51A8827
:10A8A0001C4622EA00009042188002D0012003F0EA
:10A8B000EBFB208810BD00BF68110020064B10B5CF
:10A8C0001A881C4610439042188002D0012003F0E1
:10A8D000DBFB208810BD00BF68110020024A93688E
:10A8E00023EA000090607047EC29002008B5104B67
:10A8F0001A780023D9B2914207D20E49002051F8AC
:10A900002310013309680880F4E7322003F059FB73
:10A91000094B1B685A0309D5084B9B685B0305D498
:10A92000BDE8084040F2DC5003F04BBB08BD00BF5F
:10A93000D0270020D42700208C290020EC290020DB
:10A940004B4A68232DE9F341137040F2D4735380CE
:10A95000BE231371EF2382F8D13700231946164620
:10A9600082F8D237F25C0133514040F2D472934204
:10A97000F8D13F4B3F4A83F8D2173F4B04275A6028
:10A9800002F188325A600020013F17F0FF075ED0C5
:10A99000394B3422394CDA6004F17848A8F5FC3898
:10A9A000C8F3090353B100234FF4005056F8088050
:10A9B0000193FEF76BF90428E6D11CE04FF4302038
:10A9C000FEF764F90428DFD12B4D4FF430202B69BA
:10A9D00043F002032B616C612B6943F040032B6150
:10A9E000FEF754F941F6FD732A69042803EA0203CD
:10A9F0002B61D8D0C8E7204D4FF400502B6943F0AD
:10AA000001032B611FFA88F32380FEF73FF9042826
:10AA100013D1A31C0193019B4FEA1848A3F80080AF
:10AA20004FF40050FEF732F941F6FE732A6904280C
:10AA300003EA02032B6106D0A6E741F6FE732A69FA
:10AA400013402B61A0E70E4B04349C42A4D10A4A68
:10AA50000428136943F08003136102D107F09EFBC1
:10AA600010B90A2003F028FB02B0BDE8F08100BF56
:10AA7000EC290020230167450020024000F801086E
:10AA8000D4FF01082DE9F04107F088FB10B90A2036
:10AA900003F012FBB74CB84940F2D47220460CF0D8
:10AAA000FDFB94F8A8374FF4CC71022B84BF002330
:10AAB00084F8A83794F8A827B04D01FB02F303F5FA
:10AAC000387020442344286093F8340301FB024289
:10AAD000022803F54C7384BF0020187192F83433B8
:10AAE000A74A13700C2202FB0343A64A03F2AA737F
:10AAF000136046F20902A3681A401AB99D4A43F44A
:10AB000000539360A368DF0703D54FF40050FFF7AD
:10AB1000E5FEA3685E0409D50820FFF7DFFE4FF4C9
:10AB20000050FFF7DBFE0120FFF7D8FEA3681807EF
:10AB300006D54FF40050FFF7D1FE0120FFF7CEFEFF
:10AB4000A368990413D54FF40040FFF7C7FE894B63
:10AB500093F88431012B03D14FF40060FFF7BEFE60
:10AB60004FF48030FFF7BAFE4020FFF7B7FEA3682E
:10AB70005A0603D54FF48030FFF7B0FEA36803F404
:10AB80000852B2F5085F0AD11B0508D5794B93F836
:10AB90008431012B03D14FF40060FFF79FFE94F83E
:10ABA000D221744B2AB193F8D62112B1002283F836
:10ABB000D6214FF0000C6746734E744B1E6004EBB9
:10ABC0000C03B3F8EAE14FEA5E0101F077314FEA96
:10ABD0009E0303F03333C1EB0E00C11A4FEADE03CC
:10ABE00003F01133CB1A03EB231303F00F32FF23CF
:10ABF00092FBF3F31EF00108C3EB032318BF0137E8
:10AC0000A2EB030318BFFFB2012B0ADD022B40F0B9
:10AC1000AE80B8F1000F00F0AA801EF0BC0F00F06B
:10AC2000A6800CF1080CBCF1280FC8D1013F012F00
:10AC300000F29D8007F08EFA3022002154480CF07B
:10AC400038FB544F544BD5F800801F60534B002104
:10AC500008F17900C3F80080FDF756FD504B80F0F5
:10AC6000010018704F4B07F126021A604E4B07F196
:10AC7000CC021A6098F8000003F09EFE28684B4B47
:10AC800000F5C5721A6002F02DFD494B07F18A02EA
:10AC90001A60484B00221A809A71474B2D6807F1C1
:10ACA0002A021A60454B05F219121A60444B05F24C
:10ACB00089121A60434B07F108021A60424BDFF811
:10ACC00044811F60414B07F192021A6007F19C0317
:10ACD000C8F800303E4BB4F866011E6008F092FDE3
:10ACE000C8F80800B4F8680108F08CFD95F85C30ED
:10ACF00008F1040288F8043095F87830C8F80C00A0
:10AD000088F8053094F8D531286E88F81030314B2A
:10AD1000C8F814501A60304B05F164021A602F49CC
:10AD200008F0C8FD01464FF07C5008F077FEB5F8FA
:10AD300016412B4B1860204608F068FD0146294853
:10AD400008F06CFE284908F0B5FD284A284B15602C
:10AD5000284A186005F168031360274A05F21115A7
:10AD60001560264A1760264A1360BDE8F081FCF79B
:10AD7000D1F85FE7EC29002000F80108E00F00207F
:10AD8000B027002008100020742B0020E8150020B8
:10AD9000D80E0020302B00200C0F0020100F0020B8
:10ADA0000800002040020020F40D00201C0F0020AD
:10ADB000C40E0020A8330020940200201427002095
:10ADC00064040020F0250020F425002078030020F2
:10ADD0003C04002078260020B8260020DB0F4940E4
:10ADE000B4260020000061444C3D0F440C020020BA
:10ADF0007403002000020020640300206C03002084
:10AE0000080100209016002008B5FFF799FDFFF714
:10AE100039FEBDE80840012003F036B9426A806A75
:10AE2000131A5842584170474171704743799B0744
:10AE30000AD5436A8269D154436A01690133B3FB7D
:10AE4000F1F201FB123343627047437913F00103BF
:10AE50001FBFC36803F1FF32C369006A1DBF181A20
:10AE60001040C0B218467047437910B513F0010383
:10AE700004460DD0FFF7E9FF58B1236A6269E16823
:10AE8000D05C0133B3FBF1F201FB1233236210BD3E
:10AE9000184610BD90F83B3210B57BB990F83A32A5
:10AEA00090F83942A34209D2B0F8401201229A40E8
:10AEB0000A430133A0F84022DBB2F3E710BD8379E7
:10AEC000DB0748BFB1FA81F1D0F8343148BF4909F6
:10AED0005A681B8909B1136170475361704710F8B4
:10AEE0000A3C0133DBB20A2B84BF10F8131C054A5D
:10AEF00000F80A3C82BF002322F8113000F80A3C17
:10AF0000704700BF64140020334A70B5136C90681A
:10AF1000194440F68C23081A98429160D060516021
:10AF200013463BD9127893F9451010468A420BD14B
:10AF3000111F082908D893F84610182901D80131A3
:10AF400003E083F8442002E0002183F8461093F9DF
:10AF500044402149A24219D191F84740B4B10C3183
:10AF60000024944206DA51F8046F1C4D25F8146051
:10AF70000134F6E70C2805D01849002421F81040C8
:10AF80000130F7E7164801780131017083F8452058
:10AF9000002201211A7083F8471070BD92F8471003
:10AFA000C9B140F2DA51A0F2EF248C4208D81178EE
:10AFB0000B2905D80B1D0131117042F8230070BD1B
:10AFC000002283F84720074B03F13002002143F8A9
:10AFD000041F9342FAD170BD5C0900206414002064
:10AFE000E100002068090020024A136C0133194473
:10AFF000116470475C090020024B53F820301B6835
:10B0000019807047D4270020074BA1F57A7153F8B7
:10B0100020301A681B8959434FF47A7391FBF3F17E
:10B0200089B21180704700BFD42700201FB50123CB
:10B03000ADF80830ADF80410002301A9ADF80A30CE
:10B04000ADF80C30ADF80620FDF731FE05B05DF827
:10B0500004FB38B5A0F513746379A579DB0745D5F2
:10B0600094F8383205F00105F3B1226B1068838D36
:10B07000C3F34E03838494F83C3223B1B4F84232D4
:10B080000133A4F84232917A6A00FFF7CFFF01231F
:10B0900084F83B32002384F8393284F83A3284F859
:10B0A0003832A4F8403238BD94F83B322046012BA8
:10B0B00004BF94F8393284F83A32FFF7EBFE94F883
:10B0C0003B22236B3AB9012284F83B221868997A13
:10B0D00005FA02F207E0002284F83B229542186844
:10B0E000997A08BF0222BDE838409FE738BD10B505
:10B0F000A0F5127494F83C22BAB9A36A616A994225
:10B1000028D0591CA069A162C35C2069DBB25B0036
:10B1100043F400738142A4F83E324FF00A0384F8EE
:10B120003D3228BFA262012312E094F93D327BB187
:10B13000B4F83E1220464B08A4F83E3201F001015B
:10B14000FFF7BDFE94F83D32013B84F83D3201E04B
:10B1500084F83C3294F83832002B4ED194F83932CE
:10B160000133DBB2092B84F8393203D12046BDE824
:10B1700010408FE60A2B40D194F83B322BB9B4F83B
:10B18000403243F00103A4F840326379D9071CD55B
:10B19000B4F84002820501D4C30705D4B4F84432A0
:10B1A0000133A4F8443210E0E36AC0F347000BB166
:10B1B00098470AE0E3696269D054E369E1680133C2
:10B1C000B3FBF1F201FB1233E361012284F8382270
:10B1D00094F83B220023012A84F839320DD1A27958
:10B1E00084F83B32236B12F0010F1868997A0CBF78
:10B1F00002220022BDE8104018E710BDF0B5046D32
:10B200008279A389467923F4005312F0020F4FEAA2
:10B2100003434FEA13430CBF00214FF4005112F0D7
:10B22000040FA38114BF4FF4806E4FF0000E16F090
:10B23000010F8768054614BF04200020B307238A46
:10B2400048BF40F008029BB223F4405343EA010395
:10B250002382A18948BF90B289B221F4B05121F074
:10B260000C014EEA010140EA0102A281A38A87B0E3
:10B2700023F440731B041B0CA38201A8FDF7BCFC44
:10B28000039B049E254A944218BF1E46A389192297
:10B2900072431BB2002BB4BF7E00BE00B2FBF6F6B9
:10B2A0006427B6FBF7F00001010907FB1163A289CF
:10B2B00012B2002AB7BFD9001A013231B1FBF7F23E
:10B2C000A7BF3232B2FBF7F302F007021043A8BF68
:10B2D00003F00F03AA79A8BF184380B212F0010F40
:10B2E00020812B6D06D00E498B4202BF042001F550
:10B2F0004841086112F0080F9A8A0BBF22F0080239
:10B3000092B2120442F0080208BF120C9A829A8983
:10B3100092B242F400529A8107B0F0BD0038014069
:10B32000004400402DE9F04F504C4FF4147685B0A6
:10B33000804691461D4606FB0046274608B94C4B01
:10B3400002E0012804D14B4B33631033C6F834318B
:10B350004FF4147303FB08F3474AFC18FA50032216
:10B360006271224603F59C733B44E162A3610021B4
:10B370004FF48070D4F8343134324FF0010B6261F5
:10B380002162E161A162616284F83C1284F83912A1
:10B39000A4F84212A4F84412C4F80890A571E06021
:10B3A000206184F838B284F8468258681B890222EA
:10B3B000ADF80C3003A910238DF80E308DF80F2056
:10B3C000019204F0ECFA236B019A597B58681B89AF
:10B3D0008DF80E1003A9ADF80C308DF80F2004F095
:10B3E000DEFA30465946FFF76AFD322002F0E9FDE9
:10B3F000224BD4F834A11B681A46B2FBF9F1B1F51F
:10B40000803F03D3012AF8D95208F6E71C4A504678
:10B41000B3FBF2F289B2D2B201F04CFB4FF41470DC
:10B4200000FB08F0174B07EB000800F512703C1802
:10B430000022C8F848325046214601F083FBD8F874
:10B44000307015F0010F0CBF022200223868B97A63
:10B45000FFF7ECFD0C4B3846C8F84C32211D00229A
:10B4600001F070FB304605B0BDE8F08FA816002053
:10B47000ACBE0108CCBE010894A401085C00002009
:10B4800040420F00EFB0000853B0000803460A46E0
:10B4900090F84602D96A9B7944E71FB50123ADF8BD
:10B4A00008300023ADF80C30ADF80A30084BADF889
:10B4B00004101B7801A9012B08BF0323ADF8062057
:10B4C00008BFADF80C30FDF7F2FB05B05DF804FBEA
:10B4D0005809002038B510F80E2C044650F8043CEA
:10B4E00052B9012200F80E2C20F80C1C997A186829
:10B4F0000222BDE83840D0E730F80C2C20F80A1CB6
:10B50000891A89B220F8081C074A10F80F0C002588
:10B5100022F8101004F80E5C1868997A2A46FFF792
:10B52000BCFF04F8065C38BD64140020044B53F8DB
:10B5300020301BB107289CBF1B681980704700BFD3
:10B54000840A00202DE9F7438E460546DFF8A092D5
:10B55000114699F8A0440068164698467246631C46
:10B5600089F8A03401F052FA2B8901A9ADF8043012
:10B5700018238DF80630686802238DF8073004F030
:10B580000EFAAB7A09F2A447240127442A684946F7
:10B590000C2B00F2F680DFE813F00D00F400F4004D
:10B5A000F4005100F400F400F4008A00F400F40008
:10B5B000F400C200138CDFF83CC223F001031B042B
:10B5C0001B0C1384138CB2F804E0108B624520F03E
:10B5D00073004FEA00404FEA10409BB21FFA8EFE04
:10B5E00040F0700014D00CF5006C624510D00CF5E2
:10B5F000406C62450CD00CF5806C624508D00CF5AF
:10B60000806C624504D023F0020343F0030307E09B
:10B6100023F00E032EF4407E43F003034EF4807EAD
:10B62000A2F804E01083A2F834801384138B23F073
:10B6300008031B041B0C43F0080336E0138CDFF8EF
:10B64000B4C123F010031B041B0C1384138CB2F839
:10B6500004E0108B624520F4E6404FEA00404FEAD8
:10B6600010409BB21FFA8EFE40F4E04008D00CF56B
:10B67000006C624504D023F0200343F0300307E060
:10B6800023F0E0032EF4406E43F030034EF4806E5E
:10B69000A2F804E01083A2F838801384138B23F4FB
:10B6A00000631B041B0C43F40063138369E0138CD9
:10B6B000DFF840C123F480731B041B0C1384138C2C
:10B6C000B2F804E0908B624520F073004FEA00402E
:10B6D0004FEA10409BB21FFA8EFE40F0700008D077
:10B6E0000CF5006C624504D023F4007343F44073FE
:10B6F00007E023F460632EF4405E43F440734EF49D
:10B70000805EA2F804E09083A2F83C801384938BBF
:10B7100023F008031B041B0C43F0080330E0138CD8
:10B72000DFF8D0C023F480531B041B0C1384108C4F
:10B73000B2F804E0938B20F4005023F4E6431B049A
:10B7400000041B0C000C62451FFA8EFE43F4E0431C
:10B7500040F4405003D00CF5006C624503D12EF448
:10B76000804E4EF4804EA2F804E09383A2F840800D
:10B770001084938B23F400631B041B0C43F40063BD
:10B7800093832B7B43B1B2F844306FEA43436FEAB3
:10B7900053439BB2A2F8443013889BB243F0010399
:10B7A0001380AB7A0C2B19D8DFE803F007181818B0
:10B7B0000B1818180F18181813000B1902F1340081
:10B7C0000AE00B1902F1380006E00B1902F13C0007
:10B7D00002E00B1902F14000C3F8A40438460C44FF
:10B7E000A4F8AC64C4F8A82403B0BDE8F08300BF9B
:10B7F000A8160020002C014003F0A0BF03F09EBF5C
:10B8000003F09CBF642928BF6421F8B501FB00F553
:10B81000642495FBF4F40646E4B20027FBB2A3428D
:10B8200004D29F2004F053FA0137F7E7B4420BD259
:10B83000142195FBF1F5C4EB8410663DC4EB800048
:10B840002844C0B204F043FA0134E4B2B44201D255
:10B850009A20F7E7F8BD08B507480BF06EFDC0B2B7
:10B8600009280246044B04DC01302021C0B299545F
:10B87000F6E700221A5408BD6516002008B50748EF
:10B880000BF05BFDC0B21428044B04D8421C2021ED
:10B890001954D0B2F7E700221A5408BD65160020EB
:10B8A0002DE9F74F02F066FBA64C804626686568D6
:10B8B000A768861BF643451BC71BED43FF43F60FE6
:10B8C000ED0FFF0F2EB93FB9002D00F08782B9466A
:10B8D0002CE04FF0000929E0B14627E003EB8A0B8A
:10B8E000BBF802301A050ED413F4805F1DBF964AD0
:10B8F0009BF801101268954A954B14BF52F821200D
:10B90000126843F82A20BBF80230D80516D49905EE
:10B910000AD5904B1B7813F0040F0CBF8E4A8F4A48
:10B920008B4B126843F82A2009F10109207B5FFA4A
:10B9300089FA8B4982450B68D0D326E0894A504664
:10B94000594605F0C3FF884B1B885A0603D550465D
:10B950005946864A16E0580703D550465946844A48
:10B9600010E0190703D550465946824A0AE09A0763
:10B9700003D550465946804A04E0DB07D4D55046EB
:10B9800059467E4A05F0A2FFCEE7DFF808E20093B1
:10B99000BEF906307822A3F57A7353434FF47A72D6
:10B9A00093FBF2F3F34603F22B13019300225FFAA9
:10B9B00082FE864517D2009B03EB820EBEF802E0A2
:10B9C0001EF4806F0DD040F2671ADFF88491019B5E
:10B9D00039F822E09E449EFBFAFC0AFB1CEE29F893
:10B9E00022E00132E3E74DB308F5C333A0336360CF
:10B9F000637B544A13BB9373614B1B6813F0020FB4
:10BA00000AD0DFF894E19EF800E0BEF1000F03D009
:10BA10004FF0010E82F80EE0DA0506D5594B5B793E
:10BA20001BB1A37B43F00203A3734A4B1B7813F0B3
:10BA3000050F02BFA37B43F00403A37394F80EE049
:10BA4000BEF1000F03D13F4B5B7B002B4FD094F82E
:10BA50000DC01CF0010FACF10C031DD1BCF1030FA4
:10BA600007D8DFF8E8901EF0040F3B4A08BF4A46AB
:10BA700000E0364AACF1040CBCF1070F05D8DFF842
:10BA80001CC11EF0010F18BF6246DBB2032B0ED89B
:10BA90001EF0020F3C4B06E0DBB2032B06D82F4B07
:10BAA0002A4A1EF0020F18BF1A4600E0274A4FF03C
:10BAB000000C5FFA8CF383420DD20B6803EB8C030E
:10BAC0005B881B0642BFD2F80090214B43F82C90B4
:10BAD0000CF1010CEDE785B1BEF1000F08D0637BDE
:10BAE000184A0133DBB2142B06D1002304E025B140
:10BAF000637B002BF3D100E05373002E52D0234A16
:10BB00003223B2F90250B2F90020002DB8BF6D42C5
:10BB1000002AB8BF524295FBF3F592FBF3F2EDB267
:10BB2000D3B2AB4238BF2B46194A13B192FBF3F3A1
:10BB300000E0134643442360E37B024A83BB0123B6
:10BB40002FE000BF0C1C0020102700206CBB010858
:10BB5000AA080020E133002040BB010830BB0108E7
:10BB600024130020ACA4010868110020B2A401082D
:10BB7000B8A40108BEA40108C4A40108CAA401080D
:10BB80008C290020A833002048BB01088810002021
:10BB9000400D0300C8290020F410002050BB01080C
:10BBA0000023D3738F4D904B2D78E27BADB9002FDE
:10BBB00000F00F818D4B267B1A788D4B02F004022A
:10BBC00093F800C08B4BD2B2D3F800E00B68002191
:10BBD000894D03EB86060F46B5E01AB9874A1A610C
:10BBE000002508E0864AFAE70A68AB00D61876888E
:10BBF000760604D40135EBB28342F5D3D7E7814E04
:10BC0000B6F90060192E25DD12F803E094F814C08F
:10BC10000EF00F09E14526690CDCDFF8CCC19CF879
:10BC200015C0BCEB1E1FDEBFD6F800C0DFF8D8E1A0
:10BC300043F80EC012F803E094F816C00EF00F0996
:10BC4000E14533DBDFF8A0C19CF815C0BCEB1E1F3B
:10BC50002CDC26E0193629DA12F803E094F814C037
:10BC60000EF00F09E14526690CDCDFF87CC19CF879
:10BC700017C0BCEB1E1FA2BFD6F800C0DFF888E1DA
:10BC800043F80EC012F803E094F816C00EF00F0946
:10BC9000E1450BDBDFF850C19CF817C0BCEB1E1F61
:10BCA00004DBD6F800E0584E43F806E0554EB6F9EE
:10BCB0000260192E1BDD12F803C094F814E00CF09A
:10BCC0000F09F14526690CDCDFF81C9199F81590F5
:10BCD000B9EB1C1FDEBFD6F80090DFF82CC143F88B
:10BCE0000C90D25C02F00F0CF4451EDD82E7193691
:10BCF00080DA12F803C094F816E00CF00F09F14551
:10BD000026690CDBDFF8E09099F81590B9EB1C1F61
:10BD1000DEBFD6F80090DFF8F0C043F80C90D25C9C
:10BD200002F00F0CF445FFF665AF94F817E0BEEB98
:10BD3000121FA2BF3668344A9E505BE75888000540
:10BD400004D404330435B342F8D122E04AB101EB04
:10BD50000C0A06209AFBF0F900FB19A001280DDC63
:10BD600001E057B9012793F801900EEB89003EF8E6
:10BD700029A090F80290C07803E017460020814681
:10BD80008246013125F802AC85F800906870C9B28E
:10BD9000D7E7174A1378013B13F0FF0308BF0623C8
:10BDA0001370124B1B785B0741BFBBF906304FF491
:10BDB0007A72A3F57A7303EBC30348BF93FBF2F3E4
:10BDC000124A46BF0133DBB2012392FBF3F3434433
:10BDD000A36003B0BDE8F04F03F0EEBC03B0BDE8D4
:10BDE000F08F00BFEE1500200C1C0020E133002076
:10BDF0002C00002010270020AC0800204CBB0108BC
:10BE00006CBB010888100020AA080020400D030028
:10BE1000344B354A1B68126810B51A60334A1168F2
:10BE20005960516892689960DA60314A1168196105
:10BE30005168926859619A612E4A1168D9615168B6
:10BE4000926819625A622C4A11881985518859855D
:10BE50009188D2889985DA85284A1188198651886F
:10BE6000598692889A86264A1188D986518892885E
:10BE70001987194621F83A2F224A10780022824267
:10BE800006DA214C34F81240013221F8024FF6E76D
:10BE90001E4A1288A3F864201D4A1288A3F866205F
:10BEA0001C4A1188A3F86C1051889288A3F86E1070
:10BEB000A3F87020184A3B2112689A66174A126844
:10BEC00092FBF1F2B2F5967FC8BF4FF0FF325A678E
:10BED000134A1288A3F87820124A5289A3F85E20E8
:10BEE00010BD00BFDC310020C03300201825002029
:10BEF000242500203025002088100020C80F0020B5
:10BF000072100020D0270020E40F002054150020DC
:10BF10004C0E0020C81200207C10002000000020E1
:10BF200004100020CE0F002070B5472006F058FC0A
:10BF3000174B1B681B0307D5164B174A5B68106825
:10BF40001B68C01A06F07EFC144E154C154D307857
:10BF500006F078FC23682868C01A06F082FC636843
:10BF60006868C01A06F07DFC0F4B188806F06AFC62
:10BF70000E4B188806F066FC0D4B188806F062FC24
:10BF8000337823742B68A3606B68E36070BD00BFD7
:10BF900060330020DC310020C0330020AE100020D0
:10BFA000C8310020B0100020AC100020AA100020E2
:10BFB0000C1000200A4A138801331380094A1368C1
:10BFC00001331360084A138801339BB2202B01BF51
:10BFD00000231380054A138808BF0133138070477C
:10BFE00080330020683300206C3300206E33002043
:10BFF00038B53A4B05461B780C46083B012B6BD8ED
:10C00000452006F0EDFB284606F0EAFB0C2D23D078
:10C0100004D80A2D0AD014D835B138BD0E2D4BD016
:10C020002ED3FF2D50D038BD206849E0207806F08F
:10C03000D7FB62796378002A14BF80200020184360
:10C0400000E0207806F0CCFBA07806F0C9FBE07891
:10C0500006F0C6FB20793BE0B4F9000006F0E8FBEF
:10C06000A07806F0BDFBE07806F0BAFBB4F9040056
:10C0700006F0DEFBB4F90600BDE8384006F0D8BB98
:10C08000637820788BB180F0800006F0A9FBA4686B
:10C09000E0B206F0A5FBC4F3072006F0A1FBC4F351
:10C0A000074006F09DFB200E12E006F099FB606849
:10C0B000BDE8384006F0D5BB206806F0C3FB6068D9
:10C0C000BDE8384006F0BEBB054806F00DFB002079
:10C0D000BDE8384006F084BB38BD00BFC031002049
:10C0E00017C401082DE9F04FBF4B8BB0188801939E
:10C0F000002840F0A380BD4EFDF7F8F9FFF788FE59
:10C1000034684920254606F06BFBB94B04F11C0846
:10C11000186806F097FB55F8040B06F093FB2846C9
:10C12000FAF7ACFE04F11000FAF7A8FE1027B14DA3
:10C1300001232A68BB40134203D0D8F8000006F060
:10C1400090FB0137132F08F10408F0D1AA4F04F136
:10C150002800FAF783FEB7F84431B4F92E00B84648
:10C16000C01A06F06FFB2B6813F4805F08D0A34B56
:10C17000B4F864001B88181AC0F30D0006F062FBC7
:10C180002B68990403D5B4F8660006F05BFB2B68B6
:10C190005A0503D504F16C00FAF760FE2B681B0505
:10C1A00002D5A06E06F05DFB2B685F0402D5606FC0
:10C1B00006F057FB2B68180403D5B4F8780006F096
:10C1C00041FB274604F13000FAF748FE04F136003F
:10C1D000FAF744FEB8F8443137F93C0F4FF0010844
:10C1E000C01A06F02FFB864B1B78984509DA37F901
:10C1F000020FB4F93C3008F10108C01A06F031FB17
:10C20000F1E72B68990505D5B4F95E00A0F2DC5082
:10C2100006F027FB32687B487260B260121A9110F8
:10C22000794A4A43531C032293FBF2F202EB420287
:10C230009A1A7C2303FB0203336068E2734B744A4F
:10C240001B6811688B4206D00AA941F8203D0020E6
:10C250001360FFF7CDFE684A019B92F8CE171B884A
:10C2600092F8CF070B44013BB3FBF0F200FB123313
:10C270008B4280F017825D4F0120FDF737F9FFF701
:10C28000C7FD50203E687D6806F0AAFABA683B6890
:10C2900010681B687A6803441068A3EB400006F03E
:10C2A000E0FA6A68736802A89B1A0293AA68B368E6
:10C2B0009B1A0393EA68F3689B1A0493FAF7DEFD6E
:10C2C0002A6933699B1A02936A6973699B1A0393FB
:10C2D000B369AA699B1A04930023194602AA52F86B
:10C2E000212002F120003F2842D802F108000F2847
:10C2F00006D80232032A04D9002B08BF012300E02C
:10C30000022301310329E9D1012B02980ED0022B1F
:10C3100021D0039B00F0030003F003039B0043EADA
:10C320000010049B03F0030318430CE000F00F001F
:10C3300040F0400006F054FA0498039B00F00F0010
:10C3400040EA0310C0B206F04BFA06F11C0B05F1EF
:10C350001C0810246FE000F03F0040F0800006F061
:10C360003FFA9DF80C0006F03BFA9DF81000EAE752
:10C3700002224FF0000802AB53F822304FEA88083F
:10C3800003F18001FF2910D903F50041B1F5803F89
:10C3900002D248F0010808E003F50003B3F1807F02
:10C3A00034BF48F0020848F0030812F1FF32E2D22D
:10C3B00068F03F00C0B206F013FA02AC0DF1140AA7
:10C3C00008F00303022B207807D0032B22D0012B87
:10C3D00029D106F005FA607825E006F001FA6078C8
:10C3E00006F0FEF9A0781EE06C330020DC3100205E
:10C3F0006833002060330020EC2900205C330020EB
:10C40000D0270020E8310020DF7BEFBD743300200F
:10C410007033002006F0E4F9607806F0E1F9A078C6
:10C4200006F0DEF9E078043406F0DAF954454FEA14
:10C43000A808C5D189E7B84901220B68A2401A4271
:10C440008A4606D0DBF80000D8F80030C01A06F0A3
:10C4500008FA0134132C0BF1040B08F10408EAD19B
:10C4600006F1260005F12601002331F9024F30F9CB
:10C47000022F121B02AC44F823200133042BF4D109
:10C4800003214FF000094FEA89035FFA83F902ABF9
:10C4900053F821206AB102F108000F2802D849F0B0
:10C4A000010906E08032FF2A94BF49F0020949F0F1
:10C4B000030911F1FF31E6D24846002406F090F955
:10C4C000A0460DF1080B09F00302022A16D0032A38
:10C4D0001DD0012A38D1B8F1000F05D1DBF800409A
:10C4E00090462401E4B22FE0DBF800004FF0000892
:10C4F00000F00F00204306F073F925E0B8F1000FBB
:10C500000CD0DBF80000C0F30310204316E0B8F1B4
:10C51000000F08D19BF8010006F062F99BF80000BB
:10C5200006F05EF910E0DBF80000C0F303302043B2
:10C5300006F056F9DBF80000C0F3071006F050F9DA
:10C54000DBF800402401E4B20BF1040B06AB9B4581
:10C550004FEA9909B7D1B8F1010F02D1204606F090
:10C560003FF9DAF8003013F480541FBFB6F86420A6
:10C57000B5F864100124521A18BF02929A040AD521
:10C580000AAA02EB8401B5F86600B6F86620013409
:10C59000121A41F8202C580513D502AA02EB840C7C
:10C5A00006F16A0E05F16A0000223EF9021F30F919
:10C5B000028FC8EB01014CF822100132032AF4D19A
:10C5C0000334190508D50AAA02EB8400A96EB26EDD
:10C5D0000134521A40F8202C5A0408D50AAA02EB5A
:10C5E0008400696F726F0134521A40F8202C1804CD
:10C5F0000BD50AAB03EB8402B5F87810B6F87830A7
:10C6000001345B1A42F8203C00E0FCB1012C03D15C
:10C61000029806F026F919E0631E002002AA52F8DB
:10C6200023204000C0B20AB140F00100013BF5D523
:10C6300006F0D6F84FF0000802AB53F8280008B116
:10C6400006F00FF908F10108A045F5DB30200321C1
:10C65000FCF78CFF36200321FCF788FF2F4B3C2092
:10C660001978FCF783FFDAF80030990506D5B6F99A
:10C670005E00B5F95E30C01A06F0F3F83A68284853
:10C680007B687A60121A9110264ABB604A43531C99
:10C69000032293FBF2F202EB42029A1A7C2303FB81
:10C6A00002033B60204B1B681A0630D51F4C204DFF
:10C6B00022682B689A420BD162686B689A4207D154
:10C6C000019B1B88102B11D11A4B1B885B060DD1C7
:10C6D000482006F085F8206806F0C3F8606806F088
:10C6E000C0F823682B6063686B600EE0124A104B41
:10C6F00011782A7C914208D1104A996810688842C2
:10C7000003D15268DB689A4201D0FFF70DFC05F0B7
:10C71000D9FF0BB0BDE8F08F60330020D027002098
:10C72000E8310020DF7BEFBD8C29002010100020B5
:10C73000C83100206E330020AE100020B010002061
:10C740002DE9F84F0C9EC2EB030B394C0B9B0029D3
:10C7500014BF4FF0060A4FF0040AF61A6368054644
:10C760000133904613D1236853455ED2314A032BDF
:10C7700098BF294652F823202F4806F01FF8636817
:10C780000022013363602D4B05461A7013E000252B
:10C7900011E02B4A1278954240DA0B9BE3B109FB7A
:10C7A00006F2995C01228A40264909680A4213D19F
:10C7B000636801336360D4F804900A9B1C4F994569
:10C7C000E7DB2BD10A2006F00BF83B6801333B6016
:10C7D0004FF0FF337B6021E0184A117821B12C2003
:10C7E00005F0FEFF013501E00121117009FB0BF39B
:10C7F000226808EB030752B958F8030005F074FFEC
:10C8000097F9041005444B1CD2D00F4802E03A447B
:10C810000E48117905F0D2FF0544C9E7206850455C
:10C820002CBF00200120BDE8F88F0020BDE8F88F64
:10C8300078330020D0A4010822C40108241C002061
:10C84000600000206033002031C401089DC301084E
:10C85000026D70B515880446ADB2A90613D5036BF9
:10C860008BB9C36A1BB1908880B298470BE0E1692D
:10C87000928840694E1CD2B2E6614254E169E26896
:10C88000914228BFE3612B0613D5636AA26A9A42DC
:10C89000236D0AD0511CA069A162825C9A80236931
:10C8A000994206D30023A36270BDDA6822F08002A9
:10C8B000DA6070BD026B0346C16810B5406942B1D1
:10C8C0001A6C8C1A013A08BF0A46005D1A64C0B29D
:10C8D00010BD1A6A805C01328A4228BF0022C0B2B1
:10C8E0001A6210BD436B13B190F844007047836A1D
:10C8F000406A1B1A584258417047036B13B15B687A
:10C90000016C01E0C369016A8B423CBFC2689B189D
:10C91000581AC0B27047836A8169426B1944D1606A
:10C92000416A994297BF0169CB1ACB1A536096BFEF
:10C930000023536083624FF0000380F84430136893
:10C9400088BF816243F0010313607047436A8269C4
:10C95000D154436A02690133934228BF00234362E2
:10C96000436B1BB11B68DB0705D4D4E7026DD368AA
:10C9700043F08003D36070474171FEF73FBC816094
:10C98000FEF73CBC2DE9F04105460E46078A838937
:10C990009BB21F40002F37D0B7FA87F24FF0004309
:10C9A000D340DB4399B21F40A2F11B032982042B21
:10C9B000F0D8DFE803F0221F1C190300746A24B1C9
:10C9C000013C0023A4B2736201E0AC8DA4B2D6F89E
:10C9D0002080B8F1000FDDD0D8F800304046214665
:10C9E0009847D8F80480F4E73068A98E08E07068AA
:10C9F000298F05E0B068A98F02E0F068B5F8401013
:10CA0000036889B29847C5E7BDE8F081254B10B5AA
:10CA10005A43254B254C1B680139B3FBF2F20388BE
:10CA2000013AA04289B292B29BB212D004F50064DE
:10CA3000A0420ED0B0F1804F0BD0A4F59834A042A4
:10CA400007D004F58064A04203D004F58064A042BE
:10CA500002D123F070039BB2154CA04206D004F51E
:10CA60008064A0421CBF23F440739BB203800F4B31
:10CA70008185984202850FD003F5006398420BD060
:10CA800003F54063984207D003F58063984203D0D2
:10CA900003F58063984201D100230386012383823A
:10CAA00010BD00BF40420F005C000020002C014080
:10CAB0000010004073B505460068FFF7A7FF2A681D
:10CAC0000124138800269BB243F001031380EB7A04
:10CAD00001A88DF804308DF805408DF806608DF8BA
:10CAE000074005F0C5FEEB7A1B2B0BD1192301A8DB
:10CAF0008DF804308DF805408DF806608DF80740FC
:10CB000005F0B6FE02B070BD0C4B800A98420CD006
:10CB100004D8B0F5801F0CD101207047084B984213
:10CB200005D04933984206D003E002207047032025
:10CB30007047FE2070470020704700BF01001000C2
:10CB4000020010002DE9F843046807462046884695
:10CB50009146FFF7D9FF03284BD8BA7A9108B8F16C
:10CB6000000F06D1A589AEB202258D4026EA050543
:10CB7000A5810A2303FB00131F4A42F823800433D4
:10CB800042F82390B8F1000F07D0BD7AA189AD0813
:10CB90000223AB400B439BB2A3812823434303F101
:10CBA00020011144EFF31286502585F3128803F11A
:10CBB0000C051C331544134455F8047F17B10F605E
:10CBC000296804319D42F7D100230B60F3B283F34F
:10CBD0001188282303FB0020036A23B1A3899BB299
:10CBE00043F0010304E0A38923F001031B041B0CA1
:10CBF000A381BDE8F88300BF50250020004827E648
:10CC0000281C0020004823E67C1C002000481FE66A
:10CC1000D01C00200B4B4FF400525A604FF6FE73AD
:10CC20000948D0F8DC2011680B401360D0F8CC2004
:10CC3000D0F8D0309A4201D0A8306CE6012380F8B9
:10CC4000EC30704700000240281C00202DE9F04322
:10CC50001D46A64B8DB09842884617469DF85060F9
:10CC60005CD1A34BA34AA449C3F8A82003F1FC025A
:10CC7000C3F8BC2003F5FE72C3F8C0204FF48072E5
:10CC8000C3F8B420C3F8B8209C4AC3F8B070C3F806
:10CC9000D820A2F54842543AC3F8F420C3F8F02053
:10CCA000C3F8F800C3F8DC10954B9A6942F480424F
:10CCB0009A615A6942F001025A6102238DF80330E9
:10CCC0004FF40073ADF80030330701D51C230FE09B
:10CCD000AC0706D518238B4869468DF8023002F060
:10CCE0005EFEE8070AD54FF48063ADF800304823B4
:10CCF000844869468DF8023002F051FE0E238DF80B
:10CD000004300022012301A88DF805308DF806209B
:10CD10008DF807307C4C05F0ABFDA1E07B4B9842D1
:10CD20004ED1734B734ADF655A654FF480721A66B1
:10CD30005A6603F53F729A6603F57F72DA66744AA3
:10CD4000C3F8A400C3F89C20C3F8A0206C4B3107A3
:10CD5000DA6942F40032DA615A6942F001025A613A
:10CD60004FF002038DF803304FF00403ADF80030AC
:10CD700001D51C230EE0AA0706D518236148694691
:10CD80008DF8023002F00BFEEB0709D50823ADF851
:10CD9000003048235B4869468DF8023002F0FFFD01
:10CDA00026238DF804300022012301A88DF80530D8
:10CDB0008DF806208DF80730564C05F059FD4FE0F0
:10CDC000554B984240F0ED80494B4A4A9F601A60AB
:10CDD00003F2FC425A6103F2FC529A614FF48072F2
:10CDE000DA601A614D4A18659A64DA64444B340774
:10CDF000DA6942F48022DA619A6942F008029A61A3
:10CE00004FF002038DF803304FF48063ADF800302B
:10CE100001D51C230FE0A80706D518234048694612
:10CE20008DF8023002F0BBFDE9070AD54FF400632C
:10CE3000ADF8003048233A4869468DF8023002F0D8
:10CE4000AEFD27238DF804300022012301A88DF8C0
:10CE500005308DF806208DF8073005F009FD244CCB
:10CE60004FF00009012384F84430C4F82090C4F83E
:10CE70001C90C4F82890C4F82490C4F82C806571E4
:10CE8000A760A6712046FEF7B9F9EA0752D5206BD4
:10CE9000002847D0E36CCDF80C9001934FF48053F9
:10CEA0000A9380230693E368CDF81490049320231B
:10CEB00009936369CDF81C900293CDF82090CDF8CA
:10CEC0002C90FBF721FE01A9206BFBF7FFFD226BE5
:10CED000216D136843F0010313608B8A9BB243F00A
:10CEE00040038B8253689BB2236423E000380140E7
:10CEF000281C0020E8A40108440002405800024019
:10CF00000010024000080140D01C002000440040F6
:10CF1000044400407C1C00200048004004480040BD
:10CF2000000C01404FF6DF72236D1A80DA6842F080
:10CF30002002DA60AB072CD5606B28B3A36C002508
:10CF400001934FF480530A9380230693236902953B
:10CF500004931023039305950795089509950B9560
:10CF6000FBF7D2FD606B01A9FBF7B0FD636B1A689C
:10CF700042F002021A60226D5D605D60938A9BB28E
:10CF800043F08003938204E0226DD36843F0800372
:10CF9000D360226D204693899BB243F40053938162
:10CFA00000E000200DB0BDE8F08300BF10B506F032
:10CFB0002DFC0021044606F039FE08B1204601E0B0
:10CFC00004F10040054906F029FD054906F072FC10
:10CFD000FDF792FB034B186010BD00BF8096184B05
:10CFE00035FA8E3C4C000020F8B59C4B04461B687B
:10CFF000187818B1012800F06A819AE2242C984D23
:10D000000CD006D80A2C00F0D9800D2C00F0D68068
:10D0100048E12A2C06D02C2C04D043E128706870FB
:10D02000A87050E18F4B69782F7800208C4A5854B3
:10D030002FBB1978D770472921D1597850291ED193
:10D040009978472907D1D978472904D119794129F5
:10D0500001D10121D1709978824A522903D1D17826
:10D060004D2900F0688299787E4A472907D1D17806
:10D07000532904D11279562A04BF0322EA70EA78B0
:10D08000774E022A39D0032A4CD0012A40F08580FD
:10D09000BA1E072A00F28180DFE802F004080F13AD
:10D0A0001A257F2A05F0E2FD686076E01B78532B95
:10D0B00073D16B685B426B606FE005F0D7FDA860D1
:10D0C0006BE01B78572B68D1AB685B42AB6064E0C8
:10D0D0001B78302B644B1A788CBF42F0020222F08E
:10D0E00002021A7059E0002005F020FE287354E077
:10D0F000002005F01BFEE8814FE0072F06D0082F27
:10D100004BD1012005F012FE708246E0012005F0AF
:10D110000DFE41F2184358434FF47A73B0FBF3F01D
:10D1200030823AE0022F07D0032F0AD1002005F009
:10D13000FDFD4E4B187030E0002005F0F7FD307516
:10D140002BE02AD93A1F9210337D0132D2B2013B33
:10D1500002EB8303DBB2102B1FD8F91EC2F10102D0
:10D1600001EB8202D2B2012A0BD0042A11D1002095
:10D170005E1E05F0DBFD3E4B002298553D4B9A5557
:10D1800007E03D4A5E1E0020935505F0CFFD3B4B66
:10D1900098553B4A136801331360314B2A2C18BF52
:10D1A0009A7807F101074FF000000CBF01225440AC
:10D1B0002F7068700CBF5A759C7084E0687D0028E1
:10D1C00048D0304B13F8012D2F495A708B42F9D1BA
:10D1D000244A234C13785278402B85BF373B1B01E0
:10D1E0001B01DBB298BF03F0F003402A8CBF373A33
:10D1F000303AD2B21344AA78DBB29A4227D1212323
:10D200000B702249E0780B68012803F101031E4AE4
:10D210000B600AD002281CD172231370228A1C4B87
:10D220001A80628A1B4B1A8013E0672313700E4B1F
:10D230001B789F070ED5184B62681A60A2685A6067
:10D24000227B164B1A70E289154B1A8002E03F23AD
:10D250000B70002000236B7535E000BF3802002002
:10D2600024230020B8290020A8100020241000202A
:10D2700055100020451000202510002035100020FA
:10D280007C160020C80A0020B40A0020881600205E
:10D29000AA1000200C100020B0100020AE100020BA
:10D2A000AC1000206B78687D0E2B9FBFA54A591CDF
:10D2B0005170A54A98BFD454A24A18B993785C40DB
:10D2C000947000E00020003018BF0120F8BD9D4B95
:10D2D0000022997D082900F22C81DFE801F0050B7E
:10D2E0000F15202B475D6700B52C40F02281DA75C1
:10D2F000012239E0622C08BF022235E003229A7530
:10D300001C765C769C7614E104229A755A7E997E8E
:10D310002244D2B25A760A449A76DC7609E1052292
:10D320009A755A7E997E2244D2B25A760A449A76E7
:10D330009C83FEE006229A755A7E997E2244D2B2E0
:10D340005A760A449A769A8B02EB0424A4B2B4F576
:10D35000AC7F82BF7B4A0121D17500229C83DA8396
:10D36000002C40F0E68007229A75E2E05A7E997E12
:10D370002244D2B25A760A449A76DA8BB2F5AC7F5E
:10D380003EBF7049891881F820400132998B92B2D2
:10D390009142DA83E7D9CCE008229A755B7EA342FA
:10D3A00000F0C780674B0122DA750DE0674D9A7572
:10D3B00015F8012D6A70664A9542F9D1997E614A45
:10D3C000A14206D03F232B70624A53680133536059
:10D3D000AFE06148016801310160D07D10B13E23AA
:10D3E0002B70A6E021212970D17E062941D004D8D6
:10D3F000022907D0032923D0F8BD122959D030299A
:10D4000067D0F8BD5021546A297054494C60946A21
:10D410000C60116B4FF47A7491FBF4F1504C218045
:10D4200092F878114F4A19B1117841F0020102E0E7
:10D43000117821F002011170012283F8792169E04D
:10D440005321297092F82510CE0705D592F8242093
:10D45000D51E6A426A4100E0024602F0010183F8EB
:10D460007811002A56D13F490A7822F002020A7048
:10D4700050E04F21297092F82B10CC0705D592F877
:10D480002A20D11E4A424A4100E0024602F0010130
:10D4900083F8781122B933490A7822F002020A701F
:10D4A00093F84F10304A1170B3F84C102F4A118086
:10D4B00030E05621546B29702D490C8042F21074D3
:10D4C000916B91FBF4F12B4C2180012182F87A11B0
:10D4D00020E04921297092F82410274A102988BF9A
:10D4E00010211170254914780022A2420ED20E7A22
:10D4F000234D56554E7A234D5655CE7A224D5655CC
:10D5000011F80C6F214D56550132EEE720490A689B
:10D5100001320A6093F879310A4A002B3AD092F826
:10D520007A31BBB3002182F8791182F87A1118465A
:10D53000F8BD0020F8BD1279432A7FF494AD022291
:10D54000EA7090E524230020B8290020C80A0020B2
:10D55000B40A00201802002088160020B010002015
:10D56000AC100020A8100020AE10002052000020B7
:10D57000AA1000200C1000202410002044230020BA
:10D5800025100020351000204510002055100020E7
:10D590007C160020F8BD0449044B0968002218706D
:10D5A0005A6199611A777047B0290020180200204B
:10D5B000F8B5101A0D461F4606F028F90446781BE8
:10D5C00006F024F9174B079E196806F073F92146F7
:10D5D0000546204606F06EF929460746284606F01D
:10D5E00069F90146384606F05DF80AF0D3FA0E49AB
:10D5F00006F060F906F04AFB069B2946186004F124
:10D6000000400AF03BF9094906F054F9084906F0D0
:10D6100049F806F015FB0028BCBF00F50C40A0300F
:10D620003060F8BD4C0000202C7D8E3FA00CB3452F
:10D6300000A00C4644F25063984203DDA0F50C4074
:10D64000A0387047034B9842BCBF00F50C40A03097
:10D65000704700BFB0B9FFFFF7B50368174C184D0E
:10D6600023600B68174E63600068FFF79FFC95E826
:10D670000300154B0196009394E80C00FFF798FF08
:10D680003668124B60681E606B68114FC01A06F056
:10D69000BDF8104B196806F00DF906F0D1FA2A68AA
:10D6A000236878609B1A3B600B4B1E600B4B1B681A
:10D6B000DA880B4B1A8003B0F0BD00BF9828002019
:10D6C000B0100020A4280020A0280020E02800207E
:10D6D000A82800204C000020D82800201C0F002083
:10D6E000D428002070B50446407906F08BF81E4916
:10D6F00006F094F91D4D1E4E2860E07B06F082F87E
:10D70000194906F08BF9EE606860A07906F07AF8A6
:10D71000184906F083F9184D2860207C06F072F84D
:10D72000114906F07BF96860A07E06F06BF813499A
:10D7300006F074F9EE60A860E07906F063F80D4930
:10D7400006F06CF90E4D2860607C06F05BF8064927
:10D7500006F064F96860E07E06F054F8074906F0C8
:10D760005DF9EE60A86070BD0000C842B0280020DE
:10D770000000FA4400002041C028002000007A4444
:10D78000E428002010B50C4C23789B0713D50B4BD5
:10D790001B78042B0FD90A4A0A4B1068526818608C
:10D7A0005A60FFF703FC084B1A88084B1A8023784D
:10D7B00043F00103237010BDA8100020AE1000201C
:10D7C000B01000201010002080100020F42800204D
:10D7D000044B1A78044B0AB1044A00E0044A1A6068
:10D7E000704700BF82290020882900200000A04146
:10D7F0000000A0C1164B13B51B681B0325D5154BA4
:10D80000154C1B7815498DF80030154B20681B7896
:10D810008DF8013006F04EF806F038FA11498DF80F
:10D820000200606806F046F806F030FA8DF8030052
:10D83000A06806F02BFA0C4B8DF804001B780A2028
:10D8400069468DF80530FEF7D3FB02B010BD00BF6E
:10D850008C2900207E290020A029002000002041E2
:10D860009C29002000007A4482290020054A137870
:10D8700083F001031370044A00231360034A13600A
:10D88000B8E700BF822900209829002094290020B1
:10D89000094A137818441346C0B210F0800F18BF1D
:10D8A00080381070054A19781378994201BF002317
:10D8B0001370014A13707047F9280020F8280020DF
:10D8C00010B50A4B0A4A1B7842609C18094A04604A
:10D8D00012789A4225BFD31A0B60C3F1800300234C
:10D8E0002EBF4B600B604A6010BD00BFF9280020BE
:10D8F000FA280020F82800201FB5684602A9FFF783
:10D90000DFFF044B02981B6803440398184405B0DA
:10D910005DF804FB200E00202DE9F04F89B0019343
:10D9200000238246994602910392039A934205DAB4
:10D93000029A52F8232001339144F6E7019B4D46A9
:10D94000002B56D102F064F9002852D101987DE0F5
:10D950000222404E8DF81C201A0C4FF480578DF88F
:10D960001D2006201A0A8DF81E208DF81F3002F0A7
:10D9700073F97761062004F0CFFF374B012237613E
:10D98000D0461A7077612646002007A9042204F0C9
:10D990008DFF029F4FF0000B039B9B451EDABC4698
:10D9A00057F8042B4FEA8B03002A48D0B24236D3F3
:10D9B00032465AF803100020CDF814C0049304F046
:10D9C00075FF049BDDF814C05AF8032032444AF86E
:10D9D0000320DCF800309E1BCCF800601D4B4FF498
:10D9E00080521A611D4A2D1B13681C44019B146050
:10D9F00053B34DB3194B1B68DCB22A19B2F5807FC3
:10DA0000174A88BFC4F58074D26898BF2C469342E9
:10DA10009ED3144A00231370134A137014E000209D
:10DA2000D8F8001004F042FF57F8043CD8F8002062
:10DA3000F61A1344C8F80030002347F8043C0BF1F1
:10DA4000010B08F10408A7E7C5EB090009B0BDE820
:10DA5000F08F00BF000C01401D0E0020200E0020A2
:10DA60000C000020F8280020F928002030B50B4CCD
:10DA70000B4D22782B7885B09A420CD0684602A9CB
:10DA8000FFF71EFF0123684602A90222FFF744FFA9
:10DA900000232B70237005B030BD00BFF928002093
:10DAA000F828002030B50E4D0E4C2A78237885B02A
:10DAB0009A4211D0684602A9FFF702FF002302A98B
:10DAC00002226846FFF728FFFFF7E2FE20782B7856
:10DAD0001B1A5842584100E0012005B030BD00BF7C
:10DAE000F9280020F828002038B50E4C4FF4805556
:10DAF00045F2082002F0B0F86561062004F00CFF42
:10DB0000094B01222561C7201A70656104F004FFEA
:10DB1000064A002325611370054A1370054A1360F5
:10DB200038BD00BF000C01401D0E0020F828002069
:10DB3000F9280020200E002001480249FEF722BFEC
:10DB400000080040C825002001480249FEF71ABF1E
:10DB500000040040A02500204FF080400149FEF75E
:10DB600011BF00BF7825002001480249FEF70ABF17
:10DB7000002C01405025002001480249FEF702BF59
:10DB8000002C014050250020034B4FF4805208B177
:10DB90001A6170475A61704700080140034B4FF407
:10DBA000805208B15A6170471A61704700080140FD
:10DBB0002DE9F84F2E4E044637683846FCF79CFD99
:10DBC00005463846FCF725FD766880463046FCF76A
:10DBD00093FD83463046FCF71CFDD4F804900646BE
:10DBE0002946484605F066FEA76882464146384603
:10DBF00005F060FE0146504605F052FD2168824660
:10DC0000584605F057FE41460446484605F052FE88
:10DC1000314605F04FFE0146204605F043FD3146F2
:10DC20000446384605F046FE294605F043FE014607
:10DC3000204605F037FD0146504609F01FFE0D490C
:10DC400005F038FE0C4905F0E9FE0C4B196805F0AB
:10DC500029FD0B4905F0E2FE09F038FD83B21A04F4
:10DC600044BF00F5B47083B218B2BDE8F88F00BFAE
:10DC7000A02400200000E144DB0F4940C012002036
:10DC8000000020412DE9F04F87B00393994B804667
:10DC90001B889346980737D540F2E632109B96488A
:10DCA000DC89B0F900301B1B03F2F315954203D851
:10DCB000002BB8BF5B4201E04FF4FA73B0F90220C9
:10DCC00040F2E630121B02F2F314844203D8002A19
:10DCD000B8BF524201E04FF4FA729342B8BF134604
:10DCE0000522C3F5FA7393FBF2F30A22643B534314
:10DCF00098F81C20D2105343642293FBF2F3134490
:10DD000023EAE373DBB200E06423C1460093CB1C3B
:10DD100002930025029B022D13F8016F774F0293A7
:10DD20004FEA450A05D1B7F904301B365E43761138
:10DD300049E0734B37F9152033F9153003EB4202F4
:10DD4000CBF100039A4203DB5A451346A8BF5B465A
:10DD50006C4A32F90A40039A1B1B32F915402344DE
:10DD6000019305F039FA019B88B1674A1846545D62
:10DD700005F04CFD654905F051FE0146204604F0D2
:10DD80000DFE624905F096FD05F05AFF0346594A1B
:10DD90001288D10713D437F90A401B36664392071D
:10DDA0004FEA26160FD598F812409DF900206343DC
:10DDB0005343642293FBF2F306EB231603E098F837
:10DDC00008405C432611524B042433F90A3099F879
:10DDD000017093FBF4F4341B4E4E674306F10803C5
:10DDE000EB5C98F851205F430193642397FBF3F7B2
:10DDF000FF1172B13846049205F008FD06F10C01DE
:10DE000001EBC501049A736AFCF794F905F018FF59
:10DE10000746414B99F80B6019883E4B01FB04F211
:10DE200003F1280E5EF82500D21206FB02063B4ADB
:10DE3000B6F5001FA8BF4FF40016964203F1340058
:10DE4000B8BF164650F8252040F825404FF6FF7021
:10DE50000909B0FBF1F1A21A4A4303F1400103F1B1
:10DE60004C044EF8256051F825E054F8250044F89C
:10DE700025E098F85040921170444FEA850C7613D3
:10DE8000104441F825208CB1CDF810C0059305F061
:10DE9000BDFC059B224603F1580101EBC5015B6AFD
:10DEA000FCF748F905F0CCFEDDF810C099F8153004
:10DEB000BA195843019B013543431846642390FB2C
:10DEC000F3F0174B0012024423F80A2003F1080272
:10DED0004CF80270032D03F1140203F120034CF8F7
:10DEE00002604CF8030009F101097FF413AF07B099
:10DEF000BDE8F08F68110020C8290020881000209C
:10DF0000DC3300208429002000A501080000204106
:10DF1000C80F0020A0240020A40F00200000E0FF74
:10DF2000102500201FB5084B1B681B0309D58DF871
:10DF30000400039101230D2001A98DF80530FEF79F
:10DF400057F805B05DF804FB8C2900201FB5084B7D
:10DF50001B681B0309D58DF80400029100230D20D6
:10DF600001A98DF80530FEF743F805B05DF804FB14
:10DF70008C29002010B50A4A0A4B11689B68126868
:10DF80009142F8D1084A4FF47A70D2F89C4000FBD5
:10DF900004F2D31AB3FBF4F300FB013010BD00BF51
:10DFA000B029002010E000E0A024002038B504468D
:10DFB000FFF7E0FF0546FFF7DDFF401BA042FAD365
:10DFC00038BD10B504462CB14FF47A70FFF7EEFF60
:10DFD000013CF8E710BD024A136801331360704733
:10DFE000B029002010B50024044B53F8243003B1AD
:10DFF00098470134032CF7D110BD00BF80120020D8
:10E00000014B1B68184700BFC833002010B5002023
:10E01000FFF7F6FF074B00241C7005F001FB064BD1
:10E0200083F8A040C3F8A440A3F8A840C3F8AC40CC
:10E0300010BD00BFB0330020A024002010B510B9DF
:10E04000BDE81040E2E700230C225A430C4C1119A2
:10E05000125D824203D00133102BF5D110BD094B64
:10E06000D3F8AC0018B14A784078824206D2002238
:10E07000C3F8AC10A3F8A820C3F8A42010BD00BFBB
:10E0800000AC0108A024002010B540001428A8BF4F
:10E0900014200023074A022199540B449918142490
:10E0A000834201F8014CF5DBFF21D1540F20BDE87C
:10E0B0001040C3E71428002038B540F2DB15684350
:10E0C000134B10225A6108221A61851E0B24013C51
:10E0D00014F0FF0415D00E4B2846DA6882F01002C7
:10E0E000DA60DA6882F00802DA60FFF76AFF01207E
:10E0F000FFF786FF1920FFF764FF0020FFF780FF7E
:10E10000E5E7044A044B1A60044A054BDA6038BD5F
:10E11000000C0140EFBEADDEF04F00200400FA0518
:10E1200000ED00E0074B1A6832B15A681AB19A68DC
:10E130002AB9022200E0012243F8220070470F2092
:10E14000BAE700BF8012002003685B6918470368C4
:10E150001B6918470368DB68184703689B68184702
:10E1600003685B68184703681B681847B0F90230FA
:10E170002DE9F74F93421CBF0023037090F800A0D5
:10E1800004460E469146BAF1000F40F0AB801046AF
:10E1900005F03CFB864905F08DFB864905F08AFBBE
:10E1A0004FF07C5105F086FB09F0F0FA0146054678
:10E1B00005F080FB80498346284605F07BFB03463B
:10E1C00058461946019305F06DFA4FF07E5105F05F
:10E1D00069FA01464FF07E5005F020FC2946804642
:10E1E00005F068FB294605F065FB074601466060BF
:10E1F00005F058FAE7604FF07E572946A060276186
:10E20000284605F04FFA294605F054FB4FF08041AF
:10E2100005F046FA0146404605F04CFB019B606163
:10E220001946584605F03CFA394605F03BFA0146D6
:10E23000404605F03FFB40F2DC53A04627465546DA
:10E2400063651023A4F852301823A061A4F850305D
:10E250004FF09741D8F8100005F02CFB00218246C2
:10E2600005F0C6FC28B150464FF07C5105F018FA75
:10E2700004E050464FF07C5105F014FA05F042FDE1
:10E28000C7E90E014FF09741D8F8040005F012FBE2
:10E290000021824605F0ACFC28B150464FF07C517D
:10E2A00005F0FEF904E050464FF07C5105F0FAF914
:10E2B00005F028FD0135032DC7E9080108F1040820
:10E2C00007F10807C4D1A6F2DC531B042367E367F8
:10E2D0006367C4F88030A367C4F884300123A4F8CE
:10E2E00002902370D4F85490B4F95280C9EB06061A
:10E2F000636A06FA08F67343276A4FEAE67B206FE3
:10E3000007FB0B332667A7FB0667E26F1F44636CAE
:10E31000D4F840C053434FEAE27B0CFB0B3ED4F8E9
:10E320008010C4F88020ACFB02237344B61A67EB5C
:10E330000307E36AA26A43434FEAE07B02FB0B3E1A
:10E34000A2FB00237344B6185F41E36C656F4B4337
:10E350006067A06C4FEAE17B00FB0B33C4F88410CC
:10E36000A0FB01011944636B361A05FB03F3206B14
:10E370004FEAE57B00FB0B3367EB0107A0FB0501D0
:10E38000801919447941B4F95020A56705F076F950
:10E3900008F1FF3201239340E067C01841EBE371BD
:10E3A000424605F06BF9484403B0BDE8F08F00BF6A
:10E3B0006F12833ADB0F4940F404B53F2DE9F04179
:10E3C0000024234BE0B21E78B0420CD2214B33F82C
:10E3D0001010214B53F820301BB10B2801D8DB68FB
:10E3E00098470134EDE71D4B1B685B032ED50024D5
:10E3F0002346E2B2B24229D2174F4FEA840857F8B7
:10E40000242055689D4219D02846FEF77DFBEFF386
:10E410001283502282F3128811494FF0280EAA8CE1
:10E420000EFB001092B20132C0F8D420AA8ADBB2EF
:10E4300092B242F00102AA8283F3118857F80830A1
:10E4400000221B6801341A802B46D2E7BDE8F08118
:10E45000D0270020E40F0020D42700208C290020A2
:10E46000A024002008B50E4B1B6813F4805F0D4BF1
:10E4700014BFD3F85031D3F854319A880A4B197825
:10E480000023D8B2884204D2084820F81320013370
:10E49000F7E7FFF793FFBDE80840322091E500BFA2
:10E4A0008C290020A0240020D0270020E40F002089
:10E4B0000A4B30B51A680A4B02F48052D3F8504127
:10E4C000D3F8545100230AB1A18800E0A988054877
:10E4D00020F8131001330C2BF5D130BD8C2900200E
:10E4E000A0240020B227002070B5124D0024214640
:10E4F00005F25910702285F8584108F0DAFE2146DD
:10E50000D5F8CC310B4A0B4493F9020088B11E6850
:10E5100002F259140E5108199C88073184809B79A6
:10E520007029837192F8583103F1010382F8583150
:10E53000E6D170BDA0240020094B1A680E2303FB0E
:10E540000020437AFF2B07D0064A12789A4203D95B
:10E55000054A32F8130000E0808800B2704700BF1F
:10E5600014270020EC150020C82900202DE9F04FC9
:10E5700091B0FFF7FFFC8C4C0546D4F8D0614FF00A
:10E580000008831B1846019305F03CF9D4F8D41118
:10E59000029005F08FF9C4F8D0514546D4F8D871EF
:10E5A000824E97F800B00390814A0DF11C0A32F9AF
:10E5B000150005F02BF9039905F07CF94AF82500C0
:10E5C000BBF1000F2BD0584605F020F901464FF063
:10E5D0007E5005F023FA0246DFF8009211464FF014
:10E5E0007E50059205F05CF859F8251005F062F9A7
:10E5F00009F10C01049031F9150005F007F9059AAD
:10E60000114605F057F9DDF810C00146604605F0E7
:10E6100049F849F8250005F013FB708003E0654ACE
:10E6200032F81520728036F9022F0135032D02FBD6
:10E630000288B9D1642303FB08F85F4B5F481B884D
:10E6400007A95B4398FBF3F8A8F149081FFA88F87B
:10E65000FCF7D0F8B8F13B0F7D6810D9524BB3F9F5
:10E66000FC01D3F8F85105F0D1F80146284605F031
:10E67000DDFA534B68B31A7842F008022CE04FF0F1
:10E680007E51284605F00EF801464FF07E5005F009
:10E69000C5F981464FF00008DFF820B128465BF845
:10E6A000281005F007F9474A039032F9180005F0E1
:10E6B000ADF8039B0146184604F0F4FF494605F007
:10E6C000F9F84BF8280008F10108B8F1030FE3D17D
:10E6D000C4E71A7822F008022946D4F8F4011A7027
:10E6E00009F0CCF881462060D4F8F001D4F8F8B1F4
:10E6F00000F10045D4F8F401014605F0DBF8594675
:10E700008046584605F0D6F80146404604F0CAFF58
:10E7100009F040FA0146284609F0B0F82A49804637
:10E720006060484605F0C6F808F0D0FF274D26493E
:10E730002880404605F0BEF808F0C8FF244B6880EA
:10E740001B681B074CD5234807A9FCF753F8BD6885
:10E750004FF07E51284604F0A5FF01464FF07E5051
:10E7600005F05CF982464FF0000B1A4B284653F82F
:10E770002B10049305F09EF81749039031F91B0004
:10E7800005F044F8039A0146104604F08BFF514609
:10E7900005F090F8049B43F82B000BF1010BBBF143
:10E7A000030FE2D1184652E0A02400207010002090
:10E7B000C80F0020882600201C0000209026002082
:10E7C000A8100020721000204C3D0F448429002026
:10E7D000A4100020A0260020C81200207C260020C3
:10E7E0006C4D51462846FCF705F828686B680146D1
:10E7F000039305F05FF8039B82461946184605F01F
:10E8000059F80146504604F04DFFD5F808B082464D
:10E810005946584605F04EF80146504604F042FF6E
:10E8200009F0B8F90021824605F0D8F970B92868D6
:10E83000514605F0F3F851462860686805F0EEF897
:10E8400051466860A86805F0E9F8A8605148FFF7EC
:10E85000AFF9514B51491880029805F02BF84E4BF7
:10E8600008F10048054609F10049B3F90000CDF868
:10E870002C80CDF8289004F0C9FF494900F10040F0
:10E8800005F018F8DFF82C810C90B8F9000004F0BE
:10E89000BDFF0D90B8F9020004F0B8FF0E90B8F972
:10E8A000040004F0B3FF0AA90F900DA8FBF7A2FF24
:10E8B0007B78012B1AD13B4B3B4F1B7813F0040F95
:10E8C0000ED1D7F80C02402390FBF3F3C01A04F0EA
:10E8D0009DFF0F9904F0E6FE05F0B2F9C7F80C02AF
:10E8E000D7F80C02402390FBF3F001E02F4B18887F
:10E8F00004F08CFF01460F9804F0D2FED4F81412F5
:10E900000F90284604F0CEFE0146284605F086F812
:10E91000D4F81072054639460F9804F0C1FE01463E
:10E92000284604F0C7FF0146384604F0BBFE074600
:10E93000C4F810020D9808F0C9FED4F818522978CE
:10E94000FBF758FED4F81C321844C4F81C020E9889
:10E9500008F0BCFE2978FBF74DFED4F820321844AD
:10E96000C4F82002384608F0B1FE6978FBF742FE91
:10E97000D4F824320E4A184401991368C4F82402CA
:10E980001944D4F8283211600133C4F8283211B088
:10E99000BDE8F08F3000002080100020BD378635A4
:10E9A00035FA8E3CE1330020A02400201C0000201A
:10E9B000C43300207210002001380A4B042804D808
:10E9C000DFE800F00507090B0D00074A08E0074AD9
:10E9D00006E0074A04E0074A02E0074A00E0074A67
:10E9E0001A60704758000020A10C010885DC00085F
:10E9F000FD31010867090108D50501083900010842
:10EA000038B500240B4D6059254402F0BBFC696801
:10EA100011B10948FBF7CEFDA96811B10748FBF712
:10EA2000C9FD0748103402F0ADFCB4F5F07FE9D120
:10EA300038BD00BF04A5010855C401085BC4010826
:10EA400091CE010870B50546284608F076FC0646CA
:10EA500058B91A4B1A485A791A4BBDE8704003EB63
:10EA60008203D3F8DC11FBF7A5BD284616493246D0
:10EA700008F06CFC60B9154802F084FC144C54F8A2
:10EA8000041F19B11348FBF795FDF8E7124805E09C
:10EA90000024124B53F8241021B91148BDE87040EE
:10EAA00002F070BC2846324608F050FC01340028C1
:10EAB000EFD1024B0B4D5C71C6E700BFEC29002083
:10EAC00061C4010804A501086DC4010872C40108ED
:10EAD000E0A6010885C4010891CE0108E4A601085A
:10EAE00032C2010880BF0108F0B585B0044608F0C5
:10EAF00024FC082826D1621EE01D1F4912F8013FA0
:10EB000009681944497801F00301022908BF203B34
:10EB100082421370F1D1254604F1080715F8016B04
:10EB20001648314608F0FBFB20B12846314608F074
:10EB3000F6FB10B1F9F756F81CE0BD42EED12046C5
:10EB4000F8F714FA0E4802F01DFC00230D4A04A940
:10EB50001A4492F888210A440849595C0133082B69
:10EB600002F80C1CF2D10023074801A98DF80C30E3
:10EB7000FBF720FD05B0F0BD64000020C6D80108F9
:10EB800089C40108EC29002035CD01082A4B2B4C03
:10EB90001E6880B52068F9F7C9FB3046F9F7C6FB57
:10EBA000206841798D0703D441F00201FFF7CCFAC8
:10EBB000234B08221A61234D10221A612B689A03F5
:10EBC00041BF06236371E37923F0010344BF43F09F
:10EBD0000203E3712068FFF7C3FA90B1184F0823CE
:10EBE0007B61164B1868FFF7B8FA8046FEF7FCF910
:10EBF00008B102F035FF30464146FFF7B4FA08236A
:10EC00003B613046FFF7ACFA78B10D4F4FF010087A
:10EC1000C7F814803046D4F80090FFF79EFA0146FA
:10EC20004846FFF7A0FAC7F810802B689B03D1D5A0
:10EC3000FAF75EFECEE700BFCC270020CC260020EE
:10EC4000000C01408C2900202DE9F047054608F012
:10EC500074FB2F4E0446D6F8088090B92D4802F078
:10EC600091FB2D4B53F8241049B10123A34013EA23
:10EC7000080F02D02948FBF79DFC0134F1E7284832
:10EC800022E028462749224608F060FB58B926486A
:10EC900002F078FB254C54F8041F0029EFD01F48E0
:10ECA000FBF788FCF7E72B784FF000092D2B03BF0B
:10ECB000013504F1FF344FF0010A4FF0000A164B02
:10ECC00053F8297027B91A48BDE8F04702F05ABB3B
:10ECD00028463946224608F039FBA8B9012000FA37
:10ECE00009F0BAF1000F03D0FBF7F8FD114803E07B
:10ECF00040EA0800B060104802F044FB3946BDE825
:10ED0000F0470E48FBF756BC09F10109D7E700BFF1
:10ED1000EC2900208FC401084CA7010885C4010814
:10ED200091CE01086DC4010899C4010848A70108E3
:10ED300032C20108A5C40108AEC4010834CD0108DF
:10ED400010B5084802F01EFB074B00241C741C641D
:10ED5000064B1C70FFF7ACFB02F086FD044B1C60F9
:10ED600010BD00BFB6C40108CC260020E53300204A
:10ED7000CC27002070B5064600240A4BE518AA8867
:10ED800016420AD0E1580848FBF714FC2846002137
:10ED900002F089FA054802F0F5FA1434B4F5486F28
:10EDA000EBD170BDA0AD0108E2C4010891CE01080D
:10EDB00008B50848FBF7FEFBFEF796FE00F028FFBB
:10EDC00018B96420FFF7FDF8F8E70348BDE80840EC
:10EDD000FBF7F0BBECC40108F9C401082DE9FF41C1
:10EDE0000A48068885684488B0F80480C768FEF73A
:10EDF00083FDCDF800800290019731462A462346D4
:10EE00000348FBF7D7FB04B0BDE8F0810C000020FD
:10EE100001C50108F0B504788BB005460CB100249B
:10EE200036E04A4B19680E2303FB0411B1F91D515A
:10EE3000B1F91921B1F91B31009591F8205101F573
:10EE40008C70019591F8215101F59071029590F91E
:10EE50000700039091F902103D48049121460134C6
:10EE6000FBF7A8FB082CDCD16DE02D2B14D1072C6F
:10EE70001BDC284608F0B6FA0AAB661C03EB440418
:10EE800024F8100C15F8013F303B092BFAD9344611
:10EE90002B78002BE9D104E0A3F13002092A09D82C
:10EEA000E5E7082CBDF8182009D00BB0BDE8F0400C
:10EEB000F8F798BE202BF8D101352646E7E7072A58
:10EEC000F3D840F2DC55BDF81A00204BA0F2EE2139
:10EED00089B2A9421B68E8D8BDF81C10A1F2EE2443
:10EEE000A4B2AC42E1D8BDF81E7004B23EB2A64254
:10EEF000DBDB0DB2AE42D8DCA542D6DBBDF9244047
:10EF0000642CD2D1BDF8266034B2112CCDDCBDF812
:10EF10002050B42DC9D8BDF82240B42CC5D812B2A7
:10EF20004FF00E0E0EFB0233A3F81B116421A3F861
:10EF30001901A3F81D7183F8205183F8214183F84A
:10EF40001F1183F822610BB0F0BD00BFE00F00205D
:10EF50005EC50108F0B504468FB0204608F0EDF913
:10EF6000C5B21DBBAB4802F00DFAAB4C94F8D610FD
:10EF700009B9AA4853E049B294F8D42094F8D5309E
:10EF8000009194F8D710A648019194F9D81007344D
:10EF9000029194F9D210039194F8D3100491294668
:10EFA0000135FBF707FB102DE0D1E2E720469D4934
:10EFB000052208F0CBF90546B8B929469A487022CF
:10EFC00008F077F92846994B19680E2303FB0013C4
:10EFD00001300022082883F8232183F8242183F8B4
:10EFE000252183F82621F0D112E120469049042200
:10EFF00008F0ACF905462046002D4AD1202108F042
:10F000008EF9002800F00481461C304608F095F97E
:10F010002C460746874B53F824502DB986480FB02D
:10F02000BDE8F040FBF7C6BA30462946FAB208F010
:10F030008DF901340028EDD1774A164602F17001AE
:10F04000002382F8DA3082F8D63082F8D53082F8A0
:10F05000D43007328A42F3D1784901EBC40191F8E8
:10F06000A022934210DAD1F8A472C3EBC302B01805
:10F070003A44176800F1D401C0F8D4709088013385
:10F08000888092798A71E7E729466D48FBF792FA02
:10F090008FE06C49072208F059F905462046002DFB
:10F0A00049D1202108F03BF9064608F046F9C4B2E0
:10F0B0006CBB6548FBF77EFA214664480134FBF7D8
:10F0C00079FA0E2CF8D15548FBF774FA0024604801
:10F0D0002146FBF76FFA0025544A012311680E22DE
:10F0E00002FB0412D2F82321AB401342594B5A4978
:10F0F0005A4808BF19460135FBF75CFA0E2DEBD1D3
:10F1000046480134FBF756FA082CE0D180E030463F
:10F11000534908F06BF92C4600284CD0022C4FD0F4
:10F1200008F060F906AB43F824004D49002008F0D0
:10F130005DF90134F0E74A4908F058F9002460B15C
:10F14000082C38D008F04EF906AB43F824004449A7
:10F15000002008F04BF90134F1E7082C2BD1069B75
:10F160000F2B28D8DDF81CE0BEF1070F23D8089F2D
:10F170000D2F20D8099E06F16402C82A1BD80A9DCB
:10F18000FF2D18D80B98642815D80C99642912D82B
:10F19000884210DA0D9C032C0DD8324AC3EBC3030E
:10F1A000134483F804E05F719E71DD711872597227
:10F1B0009C722D4CD1E60FB0BDE8F040F8F712BDBF
:10F1C000069B072B20D807990D291DD80278722A93
:10F1D0000DD06E2A18D1154A0E20126800FB0323A9
:10F1E00001228A40D3F8231121EA020209E00F4AE2
:10F1F0000E20126800FB032301228A40D3F823115A
:10F200000A43C3F8232101E0F8F7ECFC0D4CA4E617
:10F210000FB0F0BD86C50108EC29002091CE010891
:10F22000B1C5010802C20108C02A0020E00F002079
:10F230002DC20108E4A6010832C2010804A5010894
:10F2400041C201087EC501085FC40108CDC501089F
:10F250009DC30108C6D101080CD10108D2C501081F
:10F26000D6C50108BC2A002080BF01082DE9F7435C
:10F27000047805468CB9324D95F8A312B5F8A02252
:10F2800095F8A2322F48009121460134FBF792F9FC
:10F29000102C05F10405EFD14FE008F0A3F80F287A
:10F2A000044636DC2846202108F039F8264EE4B220
:10F2B000D6F84480451CA4000027284608F092F8A0
:10F2C0005FFA87F9B9F1010F83B208D0B9F1020FE3
:10F2D0000BD0B3F5B47F25D2726C13530AE0FF2B29
:10F2E00020D8736C2344987004E0FF2B1AD8736CF9
:10F2F0002344D87028462C2108F011F8054608B19F
:10F30000013502E0B9F1020F0CD10137032FD4D13E
:10F3100013E00E480E4900220F2303B0BDE8F0436E
:10F32000FBF748B908EB04000021042207F0C1FFF5
:10F3300003B0BDE8F043F8F755BC03B0BDE8F08377
:10F34000EC290020D8C50108CC260020A1C1010865
:10F35000C0C101082DE9F04FAC498BB0044607F05D
:10F36000B1FFAB49002820460CBF0125072507F057
:10F37000A9FFA8490028204608BF022507F0A2FFE0
:10F38000002808BF0425E90740F1FB80A24801F0EE
:10F39000F9FF002001F002FEA04CA14801F0F2FFAD
:10F3A000A04801F0EFFF62799F4BA04803EB820376
:10F3B000D3F8DC11FBF7FEF89D48FBF7FBF8264677
:10F3C0000027D6F814800021404604F007FC20B145
:10F3D0009848FBF7EFF8002669E039469648D6F8DA
:10F3E00018B0D6F81CA0D6F82090FBF7E3F84046FA
:10F3F000002104F0FDFB10B1202001F0BBFF06A9A5
:10F400004046FAF75DFF01468C48FBF7D3F85846B3
:10F41000002104F0EDFB10B1202001F0ABFF06A9A4
:10F420005846FAF74DFF01468448FBF7C3F85046AB
:10F43000002104F0DDFB10B1202001F09BFF06A9A4
:10F440005046FAF73DFF01467C48FBF7B3F84846C3
:10F45000002104F0CDFB10B1202001F08BFF06A9A4
:10F460004846FAF72DFF013701467548FBF7A2F829
:10F470000C2F06F11006A4D1AAE749B294F8D420C3
:10F4800094F8D530009194F8D7106E48019194F912
:10F49000D8100734029194F9D210039194F8D31044
:10F4A000049131460136FBF785F8102E03D094F80D
:10F4B000D6100029E1D100260E2777430024624AA6
:10F4C0000123926CA3403A44D2F80A20134240F040
:10F4D000948001340E2CF2D10136082EECD15B4819
:10F4E00001F050FF4D4B5A4C9F6854F8041F19B15E
:10F4F0005848FBF75FF8F8E70E46574B53F826409D
:10F500004CB10123B3403B4203D054482146FBF7A2
:10F5100051F80136F1E7524801F034FF21463F4BE4
:10F520000AAA0B4493F8883113444E4A8A5C01318D
:10F53000082903F8102CF2D1002306A94A488DF8B7
:10F540002030FBF737F8494801F01CFF4848F8F72E
:10F5500089FF484801F016FF4548F8F749FB46483F
:10F5600001F010FF4248FFF781FE4448FBF722F804
:10F570004020FFF7FFFB424801F004FF3C48F8F74A
:10F580006DFEAA0726D53F4801F0FCFE3E4801F07B
:10F59000F9FE374801F042FD3C4801F0F3FE3448E3
:10F5A000F8F7A7FA3A4801F0EDFE3148F8F7A6FD62
:10F5B0003848FAF7FFFF2E48F8F728FC364801F0E4
:10F5C000E1FE2B48FFF726FC2C48FAF7F3FF8020DA
:10F5D000FFF7D0FB6B0716D5304801F0D3FE30485B
:10F5E00001F0D0FE224801F0F3FC2448FAF7E2FFD4
:10F5F0004FF48070FFF7BEFB05E0314622462948F4
:10F60000FAF7D8FF65E70BB0BDE8F08FECC501084D
:10F6100060CA0108F3C50108F9C50108EC290020FA
:10F6200007C6010819C6010804A5010825C6010876
:10F6300030C601083DC601084AC601085EC401087B
:10F6400035CD010852C60108CC26002071C601083C
:10F6500048A7010881C601084CA701088FC6010808
:10F660009CC60108C6D80108A8C60108B1C6010891
:10F6700080BF0108C0C60108CCC6010891CE0108B0
:10F68000DAC60108E7C60108FAC6010808C701087A
:10F6900012C7010821C701082FC701083BC701088D
:10F6A0004CC701085EC7010837B50622044603218E
:10F6B0006B461E20F4F756FB9DF801309DF80000C4
:10F6C000154D43EA002000B204F0A0F8296804F0C8
:10F6D000F1F804F0B5FA9DF8033020809DF802009F
:10F6E00043EA002000B204F091F8A96804F0E2F8BF
:10F6F00004F0A6FA9DF80530A0809DF8040043EAC6
:10F70000002000B204F082F8696804F0D3F804F035
:10F7100097FA608003B030BD3C00002010B5054C66
:10F7200023681869F9F706FC18B123681A69024BB7
:10F730005A6110BDB41200200004014038B50D4BD1
:10F740000D4D99680D4B1A681C465288114203D022
:10F75000FEF710FC286007E0FEF70CFC2B689842CF
:10F7600082BFC01A064B186023685A68054B5A615D
:10F7700038BD00BF000C01401827002014020020F3
:10F780000000002000040140084A13689B020BD5CA
:10F79000074B002119704FF6FE73064908680340B5
:10F7A0000B604FF400135360704700BF000002402D
:10F7B000E03300206C0002402DE9F047664D6B6895
:10F7C0006649581C0A788E4602F0FF060AB10346C5
:10F7D000F6E737466B60687CEB6895F81080AA7C8A
:10F7E00039B2202900F09C80DFF880C10CEB810346
:10F7F000DC789B783CF82110C3F1FF039BB2002B0F
:10F8000065D04FF03C0CB1FBFCF9C3F1FF0363433F
:10F810001B12B9F1050F5DD8DFE809F0030B1A29B7
:10F820003A4AE01A4143B1FBFCF0DAB21044C0B2EC
:10F8300051E0B1FBFCF00CFB101189B2DAB2C1F15E
:10F840003C01E31A4B43B3FBFCFC204694442CE000
:10F85000B1FBFCF00CFB1011E21A89B24A43B2FB77
:10F86000FCF25FFA83F84244D2B2204632E0B1FBA8
:10F87000FCF90CFB191189B2E01AC1F13C014843B3
:10F88000B0FBFCF05FFA83F84044C0B2224621E0AE
:10F89000B1FBFCF80CFB1811D8B289B2E31A01FBDA
:10F8A00003F2B2FBFCFC224684445FFA8CF412E0C3
:10F8B000B1FBFCF80CFB181189B2D8B2C1F13C01C4
:10F8C000E31A4B43B3FBFCF20244D2B203E02246FC
:10F8D000204600E044464FEA042C4CEA004C4CEA37
:10F8E000020C17234FF0010808FA03F806F117017C
:10F8F00018EA0C0FA1EB0301DFF8748014BF4FF07E
:10F9000011094FF0090989B213F1FF3308F801908A
:10F91000E8D218360137B6B2BFB2114BA0465FE746
:10F92000EB6001238EF8003040F22A33AA740D4AAE
:10F9300069810D4985F8108068742E815360002319
:10F940008B840B889BB243F001030B80136843F058
:10F9500001031360BDE8F08718270020E033002082
:10F96000282700206C00024000040040AA08002064
:10F97000C90A002001F0030301F0FC0101F18041FC
:10F9800001F5803110B59B008C680F229A4024EA63
:10F9900002028A608A68984002438A6010BDF0B50E
:10F9A000B1F800E000234EFA03F2D50725D58E7892
:10F9B0004FEAD30CF40648BFCC7806F00F0203F0F0
:10F9C000070748BF2243BF0050F82C500F24BC400B
:10F9D00025EA0404BA402243282E40F82C2005D101
:10F9E000C46801229A4024EA020205E0482E04D1AC
:10F9F000C46801229A402243C2600133102BD2D145
:10FA0000F0BD2DE9F0437A4A87B01368904693B170
:10FA10001A681AB17749886902438A619A88986896
:10FA2000ADF8002002228DF80320694604228DF8EB
:10FA30000220FFF7B4FF3220FEF7C3FA00211122A3
:10FA40001E20F4F7A5FB012160221E20F4F7A0FB85
:10FA50006420FEF7B6FA002402A8FFF725FE274629
:10FA600026460A25022101221E20F4F791FB3220AE
:10FA7000FEF7A7FA02A8FFF717FEBDF90820BDF9A7
:10FA80000A1014448A42A8BF0A46BDF90C300F443C
:10FA900093421E44A8BF134613F5805F09DD564A02
:10FAA000013DD36883F01003D360DBD14FF001092F
:10FAB00001E04FF000091E2000211222F4F768FB3C
:10FAC0000A25022101221E20F4F762FB3220FEF7F4
:10FAD00078FA02A8FFF7E8FDBDF90820BDF90A1081
:10FAE000A41A8A42A8BF0A46BDF90C307F1A934275
:10FAF000A6EB0306A8BF134613F5805F07DD3E4A59
:10FB0000013DD36883F01003D360DAD101E04FF0F8
:10FB10000009204603F07AFE0146384803F07EFFD4
:10FB2000374D20F000402860384603F06FFE014654
:10FB3000324803F073FF20F000406860304603F065
:10FB400065FE01462F4803F069FF20F00040A860E1
:10FB5000002170221E20F4F71BFB012120221E2011
:10FB6000F4F716FB1E2002210022F4F711FB64209B
:10FB7000FEF727FAB9F1000F04D14FF07E532B6046
:10FB80006B60AB60D8F80030194E1A7B62B31A7DF7
:10FB900052B3184900258A69012442F001028A61A2
:10FBA000187B197DFFF7E6FE1748FEF7BBFA3368AE
:10FBB000164A1B6904A8536104930C238DF8153071
:10FBC0008DF814508DF81640F9F784F9336801A8C0
:10FBD0005B7D8DF806508DF8043003238DF80530D9
:10FBE0008DF8074002F044FE07B0BDE8F08300BF87
:10FBF000B412002000100240000C014000406F468B
:10FC00003C00002001C05E461DF7000800040140D2
:10FC10000F4B73B518781C4698B105230D4D8DF820
:10FC200000304FF4805600238DF8013001A86E613A
:10FC30006946022202F03AFE2E619DF8050000F0AE
:10FC4000010000F00100207080F0010002B070BDE2
:10FC50001D0E0020000C0140064B70B506461C46E8
:10FC60001D68FFF7D5FF18B923685B1BB342F8D9AD
:10FC700070BD00BFB0290020F7B503238DF8043014
:10FC8000030C8DF805308DF80700030A06200F4697
:10FC900014468DF80630FFF7DFFF78B1084D4FF4BA
:10FCA000805601A904226E61002002F0FFFD384653
:10FCB0000021224602F0FAFD20462E6103B0F0BD7D
:10FCC000000C0140024640213C20F4F761BA70B5B7
:10FCD00000EB8000094CA0F1A1059C3825440444A8
:10FCE000074B15F8010F1E787040FFF7EBFFA54298
:10FCF000F6D13046BDE87040E4E700BF34A9010802
:10FD0000E633002010B5441E14F8010F10B1FFF7C0
:10FD1000DEFFF9E710BD024680213C20F4F738BA37
:10FD200010B5D420FFF7F7FF8020FFF7F4FFA820DD
:10FD3000FFF7F1FF3F20FFF7EEFFD320FFF7EBFFC8
:10FD40000020FFF7E8FF4020FFF7E5FF8D20FFF7D9
:10FD5000E2FF1420FFF7DFFFA120FFF7DCFFC82040
:10FD6000FFF7D9FFDA20FFF7D6FF1220FFF7D3FF06
:10FD70008120FFF7D0FFCF20FFF7CDFFD920FFF77D
:10FD8000CAFFF120FFF7C7FFDB20FFF7C4FF4020C9
:10FD9000FFF7C1FFA420FFF7BEFFA620FFF7BBFFC0
:10FDA000AF20FFF7B8FFA620FFF7B5FFAE20FFF7A3
:10FDB000B2FF2020FFF7AFFF0020FFF7ACFFB0201D
:10FDC000FFF7A9FF4020FFF7A6FF0020FFF7A3FFE2
:10FDD0001020FFF7A0FF4FF48064013C0020A4B284
:10FDE000FFF770FF002CF8D18120FFF794FFC820A7
:10FDF000FFF791FFAF20FFF78EFF012010BD08B580
:10FE00005038C0B2FFF787FF0020FFF784FFBDE83E
:10FE1000084010207FE710B504465039C8B2FFF7FC
:10FE20007AFF04EB4400400000F00E00FFF773FF80
:10FE300006206043BDE81040C0F3031010306AE7AD
:10FE4000012828BF01202DE9F04F0646734F1420EA
:10FE500000FB0671724BD1F8A4421E765C61714BB7
:10FE6000D1F8B422DD69B1F8AC822A43DA61A28804
:10FE7000B1F8AEA222F44072D1F8A852120489B0AF
:10FE8000120C4AEA0809A28003A9C5F810900222C0
:10FE90008DF80E0028460193ADF80C908DF80F20D8
:10FEA000FFF77DFD019B00971F464FF0080BAA68E6
:10FEB00018EA020F03D10A20FEF778F8F7E70A20C4
:10FEC000C5F81480FEF772F8C5F810800A20FEF716
:10FED0006DF8BBF1010BEAD1C5F814A00A20FEF7BA
:10FEE00065F8C5F814800A20FEF760F8C5F81080A0
:10FEF0000A20FEF75BF80222C5F810A0284603A9E5
:10FF00008DF80F201C228DF80E20ADF80C90FFF715
:10FF100046FD454A03A894423A690BBF42F40012D9
:10FF200042F480023A613A610BBF3A693A6922F4BD
:10FF3000001222F480023A61A38823F440731B0468
:10FF40001B0CA38023889BB243F001032380A58868
:10FF5000F8F752FE0599354B25F03F05B1FBF3F359
:10FF60002D042D0C1D43ADB2A5802288002522F062
:10FF700001021204120C22802D4A03A8B1FBF2F1F7
:10FF800000298AB208BF012242F400414FF4967260
:10FF900053434FF47A7293FBF2F301339BB2238401
:10FFA000A1832388009A9BB243F001032380238816
:10FFB00023F4816323F002031B041B0C23804FF402
:10FFC00080432381142303FB062696F8B1320124D3
:10FFD0008DF80C308DF80D508DF80E508DF80F40C7
:10FFE00002F046FC96F8B0329DF80F208DF80C30E8
:10FFF0008DF80D508DF80E501AB103A802F038FCA0
:020000040801F1
:1000000008E05A0903F01F039C4002F12003094A4B
:1000100042F8234009B0BDE8F08F00BF34A90108C1
:1000200018270020001002400054004040420F00FA
:10003000804F120000E100E02DE9F04F054690F8F6
:1000400050008DB008910592099318B13228A8BFCD
:10005000322000E0012003F0D9FB0146AA4803F05A
:10006000DDFCAA4B04461888002808BF012003F0D5
:10007000CDFBA749069003F01DFC01900199204695
:1000800003F010FB0146019803F0C8FCA14B079058
:100090001B889A0724D5A049B1F90030B1F90200B4
:1000A00083EAE37280EAE071A2EBE372A1EBE07114
:1000B00091420C46B8BF1446B4F5E17F12DA914282
:1000C00003DD0028D8BF404203E0002BCCBF184618
:1000D000584203F09BFB914903F0A0FC064603E065
:1000E000002601E04FF07E564FF0000903950024F2
:1000F000CDF8089063000493894B33F9140003F0A2
:1001000085FB884903F0D6FB03F09AFD03F07EFBE4
:10011000854903F0CFFB804B824633F9140003F08E
:1001200075FB7C4B07461B889B077ED0014603F07E
:10013000B9FA7E4B804633F9140003F067FB0146A1
:10014000404603F0AFFA03F07BFD059B5B4298420B
:1001500003DB059B8342A8BF0346754A0499885E6A
:10016000099A1B1A32F91400184403F04FFB804619
:1001700003F032F870B16F4B40466F4914F80390AA
:1001800003F04CFC0146484602F008FC6A4903F0C3
:1001900091FB8046287F03F035FB684903F08AFB1A
:1001A0008346287A03F02EFB0146404603F082FB8B
:1001B000634903F07FFB03F043FD81460BF10040F0
:1001C00003F03EFD814505DB584603F039FD484507
:1001D000A8BF484603F01AFBDFF888910290019906
:1001E000404603F067FB59F8241003F05BFA5549C9
:1001F0004FEA840B804603F0FBFC38B94046524975
:1002000003F014FD20B1DFF8408101E0DFF8348114
:1002100049F80B80A87C03F0F5FA0146404603F04C
:1002200049FB4A4903F046FB81463A4BB3F800B01C
:100230001BF0010F40F09880394B049ADFF81C81C5
:10024000D35E002BB8BF5B42B3F5206F4FEA840347
:100250000A9303DD002348F824302AE03C4938465D
:1002600003F028FB039B0B90587803F0CBFA0B9A12
:100270000146104603F0D2FB514603F011FA0199F2
:1002800003F018FB58F8241003F00CFA31498046AB
:1002900003F0AEFC38B940462F4903F0C7FC20B14B
:1002A000DFF8B48001E0DFF8AC802C4A0A9B42F80A
:1002B0000380039BD87A03F0A5FA284B53F8241047
:1002C00003F0F8FA264903F0F5FA1BF0020F804616
:1002D0004CD03846029903F0E3F90146304603F06A
:1002E000E9FA0146029803F0DDF94946074640461F
:1002F00003F0D6F90146304603F0DCFA01464846E1
:1003000003F0D0F9804631E083F9223EA40F0020AB
:10031000BD37863568110020881000200000E143B9
:10032000C80F00200000A03ECDCC4C40DC330020A4
:100330008429002000A50108000020410000A04001
:100340006F12033C0000F0C10000F0410AD7A33D4A
:100350000000A043000040C3000040433C270020B1
:100360000AD7233C34270020C846029F874B185DDC
:1003700003F04CFA0146504603F09CFA844903F01E
:1003800099FA0146384603F08BF995F85120034657
:100390003AB18049804B01EBC4011B68F9F7CAFEF2
:1003A00003467E4F504657F824100A9303F078F91D
:1003B000019903F033FB47F824A007F1080A5AF823
:1003C00024B01037594603F06BF90146079803F043
:1003D00071FA0146584603F065F983464AF824004D
:1003E000385D03F013FA0146584603F063FA6C498E
:1003F00003F060FA07460A9B4146184603F052F99B
:10040000394603F04DF907F061F9664A049B0492FE
:10041000D0520A9BDFF8B0B1184603F011FC4BF83C
:100420002400404603F00CFCDFF8A0A1DFF8A08117
:100430004AF8240007F1004003F002FC039B049AF1
:10044000013348F82400039317460CB9012451E600
:10045000089A554B9479B3F90430640028345C430E
:10046000524B6411B3F9040003F0D0F94FF07A5104
:1004700003F020FA07F02AF9201A03F0C7F9002C3C
:10048000B8BF6442322C0646494C02DD0023A3600B
:1004900025E0069803F0D4FB20F0030003F0B6F942
:1004A0000190687B03F0AEF90146304603F002FA92
:1004B000019B81463F49184603F0B0FA0146484681
:1004C00003F0F8F903F0BCFBA36818443A4B9842D8
:1004D000A8BF1846394B9842ACBFA060A360A36880
:1004E0006FF0FF005B13B3F5807FA8BF4FF48073FC
:1004F0009842B8BF184603F089F98146304603F0A8
:100500009FFBEB785843801103F080F92C4B044695
:100510001B78032B11D9B5F84E60B6F5FA7F0CD2D3
:1005200003F08EFB7342984203DBB0420346A8BF40
:100530003346184603F06AF9044695F8512032B163
:10054000154B20461F491B68F9F7F4FD0446494640
:10055000204603F0A7F803F073FB80B2B88000B226
:1005600003F054F907F0B2F8B880204603F068FBB6
:10057000CBF80800484603F063FB0023CAF80800E4
:10058000C8F808300DB0BDE8F08F00BF4827002044
:10059000A69B443BAC240020C42400204C27002010
:1005A000F7CC92381025002088100020C80F0020BA
:1005B000C824002000803B45FEFFFF0F020000F032
:1005C000D0270020BC24002018250020242500204E
:1005D000302500202DE9F04F89B00593BE4B002651
:1005E000B3F90290B3F90030B9F1000FB8BFC9F107
:1005F0000009002BB8BF5B429945B8BF99468046B9
:10060000B2463446B9F5FA7F04910392A8BF4FF47D
:10061000FA79019000960296B04D2B88990754D034
:10062000AD4B610033F91420AD4B33F9143003EBBB
:100630004202039B5B429A4203DB039B9342A8BFA7
:100640001346A84A8F5E059ADB1B32F914001F1867
:1006500002F0C2FD90B1A44B384613F804A003F099
:10066000D5F8A24903F0DAF90146504602F096F9AE
:100670009E4903F01FF903F0E3FA074698F80830A3
:1006800064227B4393FBF2F398F81C206FF0040A7A
:100690000AFB02FA534504DB02EB820A9A45A8BF23
:1006A0009A4642F21072924B53F82400384490421A
:1006B000A8BF10468F4A9042B8BF104643F82400A6
:1006C00098F812305843031302932D8805F0030362
:1006D000012B38D0804B884933F91430A6000093A1
:1006E000019B51F8247093F801E0844B33F9140016
:1006F00080EAE073A3EBE073B3F5206F16DC009A99
:1007000050235A4392FBFEF3042290FBF2F0181A96
:100710000744B7F57A5F7A4BA8BF4FF47A579F42E8
:10072000ACBF41F8247041F8243002E0002341F8C6
:1007300024308B597D2693FBF6F6019BDB7A7343BD
:10074000402693FBF6F6AA0712D5009A09FB06F598
:1007500009FB02F70298C9F5FA7303FB0A7703FB5A
:1007600000534FF4FA7297FBF2F193FBF2F505E0B8
:10077000EB0755BF354651460099029D5F4B042754
:1007800033F914305F4A93FBF7F3A25C6FF04F0725
:10079000534393FBF7F398F851204FEA440BCF18DB
:1007A00072B13846069203F031F85749574B01EBC6
:1007B000C401069A1B68F9F7BDFC03F041FA07462D
:1007C0004E4B534A3BF803003BF9021003B25B1A4D
:1007D000042193FBF1F102F1040E5EF824302BF8B2
:1007E00002000C3252F8240042F8243098F85020CD
:1007F00018444FEA840C08444EF8241082B1CDF816
:100800001CC0069203F002F84249404B01EBC401C0
:10081000069A1B68F9F78EFC03F012FADDF81CC08B
:100820003D4BDFF810E11B5D7A195843202390FB04
:10083000F3F3D21A2BF80E20384A5B424CF8023000
:10084000019B3748374901334CF801504CF8007090
:10085000019375460CB90124DEE61F4B0427B3F95A
:100860000440049B244E9B79D6F808E00F335B00CC
:100870006343224C5B11B4F90440002B94FBF7F75F
:10088000A3EB0707B8BF5B42322B98F80D400BDC97
:1008900004FB07E4244BA342A8BF2346234CA342F6
:1008A000ACBFB360B46001E00023B36098F80340CC
:1008B00004FB07F31E4C9B112478032C3DD9B8F898
:1008C0004E40B4F5FA7F38D26742BB4234DBA342D4
:1008D000A8BF234631E000BF881000206811002027
:1008E000DC3300208429002000A5010800002041FD
:1008F00060270020F0D8FFFFC8240020C80F002088
:1009000080C1FFFF48270020AC240020C424002021
:1009100068270020F82400205C27002030250020D4
:100920001825002024250020FEFFFF0F020000F004
:10093000D0270020102500203B46B4686FF0FF064A
:1009400044F34F34B4F5807FA8BF4FF48074B442B1
:10095000B8BF344683601E190023AE808C6093605C
:1009600009B0BDE8F08F2DE9F04F87B00393B44B89
:1009700081461D88029105F00205ADB2019295B144
:10098000B04BB3F90250B3F90030002DB8BF6D423F
:10099000002BB8BF5B429D42B8BF1D46B5F5007F36
:1009A000A8BF4FF40075CB460026A64BA64933F9E5
:1009B0001620A64B4FEA460A33F91630520083EA56
:1009C000E374A4EBE374B4F5206F4FEA860851F8A2
:1009D000260011DC042493FBF4F3D31A0344B3F58B
:1009E0007A5F9B48A8BF4FF47A538342ACBF41F86B
:1009F000263041F8260002E0002341F8263051F865
:100A000008709BF80B30FF119BF801405F438C4B43
:100A100054431B88BF119B074FEAA41456D08D4B3B
:100A20003AF903301A44019B5B429A4203DB019B73
:100A30009342A8BF1346884A3AF902209B1A039AA8
:100A400032F916201A44049202F0C6FB049A98B1B7
:100A5000824B10469B5D049302F0D8FE804902F061
:100A6000DDFF049B0146184601F098FF7C4902F027
:100A700021FF03F0E5F8024642F21070794958F878
:100A8000013013448342A8BF034677488342B8BF6E
:100A9000034648F8013099F8081099F81C004A43B9
:100AA00000EB8000D21141428A4203DB8242A8BFA0
:100AB0000246114699F81220641A53431B13FF1A79
:100AC0006F436C4303EB672701EB64245F4B042205
:100AD0003AF9033093FBF2F2644B9B5D534399F870
:100AE0005120A4EBA31472B12046049202F08EFEB2
:100AF0005F49604B01EBC601049A1B68F9F71AFBCA
:100B000003F09EF8044651495B4B3AF801003AF96C
:100B100003E002B2CEEB02024FF0040E92FBFEF2B3
:100B20002AF803009E440C3358F80EC058F803000E
:100B300048F80E206044104499F8502048F803C04B
:100B40008C467AB10591049202F060FE4B49494B04
:100B500001EBC601049A1B68F9F7ECFA03F070F890
:100B6000DDF814C0464BDFF834E19B5DE2194343E6
:100B70005B11D21A2AF80E2042484349434A5B428D
:100B800048F8004048F8017048F802300BF1010BBA
:100B900074460EB9012608E72A4B0427B3F904501E
:100BA000029B294E9B79D6F808E00F335B006B431C
:100BB000BCF904505B1195FBF7F7002BA3EB07077B
:100BC000B8BF5B42322B99F80D500BDC05FB07E5F3
:100BD0002F4BAB42A8BF2B462E4DAB42ACBFB360F0
:100BE000B56001E00023B36099F8035005FB07F3FB
:100BF000294D9B112D78032D0CD9B9F84E50B5F520
:100C0000FA7F07D26F42BB4203DBAB42A8BF2B4641
:100C100000E03B46B5686FF0FF0645F34F35B5F58C
:100C2000807FA8BF4FF48075B542B8BF354683605A
:100C30005E190023A6808D60936007B0BDE8F08F39
:100C40006811002088100020C8240020C80F002050
:100C500080C1FFFFDC3300208429002000A50108AB
:100C60000000204160270020F0D8FFFF4827002027
:100C7000AC240020C42400207C270020F82400207D
:100C80005C27002018250020242500203025002086
:100C9000FEFFFF0F020000F0D027002010250020EB
:100CA0002DE9F04F89B00593A74B0026B3F90280D8
:100CB000B3F90030B8F1000FB8BFC8F10008002B3D
:100CC000B8BF5B429845B8BF98468246B146B34626
:100CD0003446B8F5FA7F0492A8BF4FF4FA78029030
:100CE00003969A4D2B88990757D0022C55D0964BD6
:100CF000610033F91420964B33F9143003EB4202B0
:100D0000049B5B429A4203DB049B9342A8BF1346B9
:100D1000904A8F5E059ADB1B32F914001F1802F00F
:100D20005BFA90B18C4B384613F804B002F06EFDBC
:100D30008A4902F073FE0146584601F02FFE8749AA
:100D400002F0B8FD02F07CFF07469AF808306422F2
:100D50007B4393FBF2F39AF81C206FF0040101FB34
:100D600002FB5B4505DB02EB82029342A8BF134600
:100D70009B4642F210727A4B53F82400384490425A
:100D8000A8BF1046774A9042B8BF104643F82400E7
:100D90009AF81230584303130393298801F0030390
:100DA000012B01D1022C3DD1674B6F4D33F91490CB
:100DB000029BA00093F801E06C4B55F8247033F9C6
:100DC000146086EAE673A3EBE673B3F5206F1CDCD0
:100DD000022C14D0502303FB09F292FBFEF30422F1
:100DE00096FBF2F69E1B3744B7F57A5F604BA8BFBF
:100DF0004FF47A579F42ACBF2F502B5007E089EA3F
:100E0000E973A3EBE973642BE4DD00232B50564B0D
:100E10007D26C35893FBF6F6029BDB7A734340268C
:100E200093FBF6F68A0713D5022C11D008FB06F5C2
:100E300008FB09F70398C8F5FA7303FB0B7703FB6C
:100E400000534FF4FA7297FBF2F193FBF2F508E0CE
:100E5000CB0704D5022C02D0039D594601E035464C
:100E6000494663000193414B042733F91430414A4A
:100E700093FBF7F3A25C6FF04F07534393FBF7F339
:100E80009AF85120CF1872B13846069202F0BEFC93
:100E900039493A4B01EBC401069A1B68F9F74AF944
:100EA00002F0CEFE0746314B019A0198D15A344BDD
:100EB0000AB2C05E4FEA840C121A042092FBF0F2D0
:100EC0000198C15203F10801143351F824E053F89A
:100ED000240041F82420704410449AF8502043F82C
:100EE00024E082B1CDF81CC0069202F08FFC2549A7
:100EF000224B01EBC401069A1B68F9F71BF902F0BB
:100F00009FFEDDF81CC0204B204A1B5D0199584311
:100F1000202390FBF3F07B191B1A8B521C4B404291
:100F20004CF803701B4B01344CF803501A4B032C44
:100F30004CF80300029B03F1010302937FF4D1AE4E
:100F400009B0BDE8F08F00BF8810002068110020B4
:100F5000DC3300208429002000A501080000204186
:100F600060270020F0D8FFFFC8240020C80F002011
:100F700080C1FFFF48270020AC240020C4240020AB
:100F800090270020F82400205C2700201025002056
:100F900018250020242500203025002007B5064B09
:100FA00006490093064B074A01930748074BF9F798
:100FB00001FB03B05DF804FBD0BB0108C9C2010806
:100FC000A5BB0108C3C20108C4CC0108C4BB010809
:100FD00008B5037833B90C4B0C481978BDE80840C4
:100FE000F9F7E8BA06F0FEF902280CD8064B0C22F5
:100FF0001870074B02FB0030064B0230186001F0FE
:10100000A9F80548E5E708BDB0270020E4CC0108B1
:10101000943100200810002080BF010808B5037833
:101020003BB90B4B0B4893F8A817BDE80840F9F7FC
:10103000C1BA06F0D7F9022808D8054B83F8A807EB
:10104000F9F77EFCF9F71EFD0348E8E708BD00BF8D
:10105000EC290020E8CC010880BF010838B50378EE
:1010600003BB214B1B6801330F2B07D81F490C22F0
:1010700002FB031295681C462DBB00E01C460134A0
:101080000F2C01DD002400E005D818490C2202FBDA
:1010900004129568BDB99C42F1D11548BDE83840AD
:1010A000F9F788BA06F09EF90F28044605D80F4ACA
:1010B0000C2303FB00239D682DB92146BDE8384071
:1010C0000C48F9F777BA084B1C60FCF79FFF2146E4
:1010D0002A460948F9F76EFA0C235C43034B185D66
:1010E000BDE83840FCF7AABF4800002000AC01086A
:1010F000F5CC01080BCD010823CD010873B50378A9
:1011000013B9F6F76FFD3FE001AA204906F0CBF9CD
:1011100000240246264625469AB134B1012C08D156
:10112000104606F05FF9064603E0104606F05AF94D
:10113000054601AA0020154906F0B5F9013402461A
:10114000EAE70B2D03D9124812490C230CE0022CBC
:1011500011D1A6F57A73B3F57A7F08D90C480E49F8
:101160004FF47A724FF4FA63F9F724FA0CE00B4B60
:1011700003EB45035E80094B094803EB4503294611
:10118000B3F90220F9F716FA02B070BDD6C501080E
:10119000A1C10108C0C1010882C90108B02700200F
:1011A0003ACD010838B50D4C05462368834206D177
:1011B000F7F7E0F8204600214C2206F07AF8E36CBD
:1011C000AB4209D12846F7F7D5F8BDE838400448C6
:1011D00000214C2206F06DB838BD00BF6C11002014
:1011E000B8110020034B1A68D379591C1344D171EC
:1011F000187A70474811002010B5FFF7F3FF84B24A
:10120000FFF7F0FF04EB002080B210BD10B5FFF730
:10121000F3FF0446FFF7F0FF04EB004010BD10B5EC
:101220000446054B21461868FCF79DFF034B1B68DD
:1012300098796040987110BD4C1100204811002031
:1012400038B504460D462420FFF7E9FF4D20FFF78F
:10125000E6FF002C084C14BF21203E20FFF7DFFFE3
:101260002368002228469A71FFF7D9FF236893F874
:101270004900BDE83840D2E748110020014600206F
:10128000DEE710B50446C0B2FFF7C9FF200ABDE88B
:101290001040C4E710B5044680B2FFF7F2FF200CFF
:1012A000BDE81040EDE737B5828883680446100634
:1012B0000D4641BF29494FF4CC7091F8A81700FBA7
:1012C0000133D10542BF26490C20097802F03F02C4
:1012D00048BF00FB0133042A12D006D8012A0DD0E2
:1012E000022A2FD193F900102DE0102A0AD0202ACB
:1012F0000AD0082A26D1B3F9001024E0197822E098
:10130000198820E019681EE069461868F8F7D8FFC8
:1013100001461448F9F74EF9F5B1E06802F076FAA3
:101320006946F8F7CDFF01460F48F9F743F9206900
:1013300002F06CFA6946F8F7C3FF01460A48F9F76C
:1013400039F909E000210948F9F734F925B10848CD
:10135000E1682269F9F72EF903B030BDEC290020CD
:10136000B02700205EC4010857C401089DC30108CE
:1013700049CD0108024B0146D869FCF7F4BE00BF15
:10138000B027002010B5441E14F8011F21B1034BF3
:10139000D869FCF7E8FEF7E710BD00BFB0270020D2
:1013A0002DE9F04F037885B01BB96C48FFF7EAFFD1
:1013B000D0E006F017F805460628694C99BF694841
:1013C000294669480621F9F7F5F894F8202000230A
:1013D000D9B2914207D26549002051F82310013358
:1013E00009680880F4E7013DEDB272B6604F6DB256
:1013F00007EBC50149684FF001085E4E57F835907C
:1014000008FA01FA4FF480624FF400731FFA8AF170
:1014100072614FF0480B73613046C9F8141003A98C
:10142000ADF80C2001938DF80EB08DF80F80FEF70B
:10143000B6FA019B3046ADF80C3003A910238DF8A5
:101440000E30ADB28DF80F80FEF7A9FA484603A919
:10145000ADF80CA08DF80EB08DF80F80FEF79FFA56
:10146000E9007B185A6857F83530D00803EB800E36
:1014700053F8203002F00702A3659200E36523666B
:101480000F239340DB43E06DC4F854E01840E0655F
:10149000A06D0340A365E06D082393400343E3651B
:1014A000A06D08FA02F303433846A365B3685F05ED
:1014B000FCD4676DA36D08223B604FF40073C9F83C
:1014C00014A073612C4B1A6110225A6140F6B83394
:1014D000B268520513D4013BFAD14FF40073ADF852
:1014E0000C3018238DF80E302248012303A98DF803
:1014F0000F30FEF754FA236E3B6062B62AE0C9F85B
:1015000010A0E36D50F835E03B604318D3F804C0F9
:10151000DEF80C20012303FA0CF31343CEF80C3051
:10152000154B10221A61B268124B5205C2D5D9F878
:1015300008204FF4007C1AEA020F0F4A4FF0080E01
:1015400015BFC3F810C0C3F814C0C2F810E0C2F849
:1015500014E0E8E705B0BDE8F08F00BF50CD01080A
:10156000B027002097CD0108C3CD0108D427002063
:1015700094CC010800080140000C0140F7B529494E
:10158000294B0878294D1C68294B05EB80001A88E7
:10159000D0F8C010274B28481B7800914FF47A717F
:1015A000B4FBF1F1F9F706F8244B25481968254BEF
:1015B0000026B1FBF3F1F8F7FDFF234B1F68F3B2F0
:1015C00005EB8302D2F8D010E1B101249C403C42EB
:1015D00016D0220714D01D4A0B20D25C00FB032337
:1015E000124A1B4802EB8303D3F8F020F8F7E2FF1E
:1015F000022C05D1174B197A11B11748F8F7DAFF09
:101600000136DCE71548FFF7BDFE154B15481A8873
:10161000154B92B2198840F2D47303B0BDE8F04084
:10162000F8F7C8BFF4100020B029002000AC010872
:101630009410002050000020EECD01085C00002036
:1016400031CE010840420F00A410002054000020B9
:1016500041CE01080412002049CE010891CE0108B4
:10166000A60F00204DCE0108A40F00202DE9F04167
:101670000024804625460F4E4146A759384605F0BE
:1016800099FE58B139460C48F8F794FF30190021FB
:10169000FFF709FE0948FFF775FE01351434B4F56C
:1016A000486FE8D11DB9BDE8F04105486AE6BDE8DC
:1016B000F08100BFA0AD0108E6C4010891CE010889
:1016C00032C201082DE9F74F824605F036FE054685
:1016D00028B1012818D19AF800302A2B14D1584883
:1016E000FFF750FE0024574E5748A159F8F762FF04
:1016F00030192946FFF7D7FD14345448FFF742FE4E
:10170000B4F5486FEFD198E050463D2105F007FE53
:10171000002800F08D8003461D4613F8012D202A75
:10172000FAD0441C204605F05DFE81462046F8F7BD
:1017300031FD0746CAEB05054FF0000B142404FBEE
:101740000BF4DFF8208108F5D073E658019330469A
:1017500005F0F3FD8446314662465046CDF800C0A0
:1017600005F0F4FDDDF800C0019B002856D1EAB277
:10177000624553D11D194444D4F8AC0102F046F837
:101780000146384602F048FA002845D0D4F8B001A6
:1017900002F03CF80146384602F034FA00283BD00B
:1017A000B4F8A4319A0658BF4F46142202FB0B88A6
:1017B0001C0648BF2648D8F8A82142BF90F8A807C1
:1017C0004FF4CC7404FB0022D80542BF21480C24FE
:1017D000007803F03F0348BF04FB0022042B394686
:1017E0000BD004D8013B012B0CD817700AE0102B4A
:1017F00005D0202B05D0082B04D1118002E0176002
:1018000000E0176031461448F8F7D4FE284600215E
:1018100003B0BDE8F04F46E5104805E00BF1010BC1
:10182000BBF1A00F8AD10E4803B0BDE8F04FA9E587
:10183000504603B0BDE8F04F18E703B0BDE8F08FA5
:101840007FCE0108A0AD0108E6C4010891CE0108D1
:10185000EC290020B027002094CE01089FCE01087B
:1018600032C2010800AC010808B50748FFF78AFD3D
:10187000064BD869F6F75AFDFCF7F4FDF9F736F890
:10188000034A044BDA6008BDBFCE0108B027002030
:101890000400FA0500ED00E008B50548FFF772FD09
:1018A00000F09EFCF9F74CF8BDE80840DCE700BF0B
:1018B000CBCE010808B50448FFF764FDF9F740F8FE
:1018C000BDE80840D0E700BFE1CE010810B54B8865
:1018D000DC0641BF2F4B14791B6853F8244044BFEA
:1018E0002D4B43F820404B889B0641BF294B547930
:1018F0001B6853F8244044BF274B43F820404B88D3
:101900001C070ED5254B0C781B78B3EB141FA1BF19
:10191000204BD4781B6853F82440A4BF1E4B43F8D7
:1019200020404B889B070ED51D4B0C781B78B3EBE2
:10193000141FDFBF174B54781B6853F82440DCBFDB
:10194000154B43F820404B88DC070FD5154C0B781E
:10195000247803F00F03A342DFBF0E4B14781B68FB
:1019600053F82440DCBF0C4B43F820404B885B0706
:101970000FD50B780C4903F00F0309788B42A1BFF8
:10198000044B92781B6853F82220A4BF024B43F803
:10199000202010BD10270020AA080020231C0020B2
:1019A000211C0020201C0020221C0020254A00238E
:1019B000F0B515681C461A462348244903700B707D
:1019C0002E1976884EB92F5D3FB9037000230A7037
:1019D0004B7007781C461A460CE0360548BF0132AA
:1019E00004F1040403F1010348BFD2B2802CDBB23E
:1019F000E6D1EAE7E0B2B8420CD215F8240001348F
:101A000006099E4200F00F00A8BF731C9042A8BFB9
:101A1000421CEFE78A704B70C2F3470102F00102EB
:101A20000A444C1E0A490B480A70C3F3470203F0EC
:101A30000103134404700849501E084A08701370CB
:101A4000F0BD00BF24130020181C00202C2800200B
:101A5000221C0020201C0020231C0020211C002010
:101A6000924B2DE9F04FDA68914D1A612A6891B0D6
:101A7000DA60904A0295136843F0200313608E4B9E
:101A80001A78012A0CBF002201221A708B4B1A7897
:101A9000910740F14D838A490978042940F248832F
:101AA0008849097801F0040101F0FF0011B922F022
:101AB00001021A701B78DB0702D408B1FBF762FE43
:101AC0008149CA78531C052293FBF2F202EB820291
:101AD0009A1A7E4BCA701F7892000023DFF810829A
:101AE000DFF8109258F82310794C91FBF9FE04F1BD
:101AF000080040F823E0774844F8231000FB0E115B
:101B000042F2107091FBF0F004F1100680B226F85A
:101B100013004FF0140C04F114060CFB036C04F1D9
:101B20003C0A5AF823605CF802504CF80210761B0D
:101B3000314405264AF8231091FBF6F109FB0E11FA
:101B40004434012F44F823104FEA830B444605D157
:101B50000238B0F5797F98BF4BF808100BB9012314
:101B6000BCE7594E029BB2461868336DC01A01F0AB
:101B700049FE594901F052FF029B4FF07E511B680C
:101B80000746336502F034F808B94FF07E574B4BE7
:101B9000CAF854701B78514E13F00103504D12D007
:101BA0000DAA00924F4B0EAA01920CCB94E80300B1
:101BB000FBF7FEFC0D9A6421B2FBF1F20E9B328022
:101BC00093FBF1F300E033802B809AF858303E4DC0
:101BD000002B35D0696D4FF07E5001F01FFF074696
:101BE000EB6D2068C01A01F011FE394601F062FE6B
:101BF00002F026F82B6E86B2606836B2C01A01F089
